:020000040001F9
:10800000A805012071CB0100CD9A02005DCB0100D3
:108010005DCB01005DCB01005DCB01005DCB0100BC
:1080200000000000000000000000000029CD010059
:108030005DCB010000000000E1CC01005DCB010040
:10804000ADCE0100ADCE0100ADCE0100ADCE010040
:10805000ADCE0100ADCE0100ADCE0100ADCE010030
:10806000ADCE0100ADCE0100ADCE0100ADCE010020
:10807000ADCE0100ADCE0100ADCE0100ADCE010010
:10808000ADCE0100ADCE0100ADCE0100ADCE010000
:10809000ADCE0100ADCE0100ADCE0100ADCE0100F0
:1080A000ADCE0100ADCE0100ADCE0100ADCE0100E0
:1080B000ADCE0100ADCE0100ADCE0100ADCE0100D0
:1080C000ADCE0100ADCE0100ADCE0100ADCE0100C0
:1080D000ADCE0100ADCE0100ADCE0100ADCE0100B0
:1080E000ADCE0100ADCE0100ADCE0100ADCE0100A0
:1080F000ADCE0100ADCE0100ADCE0100ADCE010090
:10810000ADCE0100ADCE0100ADCE0100ADCE01007F
:10811000ADCE0100ADCE0100ADCE0100ADCE01006F
:10812000ADCE0100ADCE0100ADCE0100ADCE01005F
:10813000ADCE0100ADCE0100ADCE0100ADCE01004F
:10814000ADCE0100FFFFFFFF81F0004102E000BF64
:1081500083F0004330B54FEA41044FEA430594EA07
:10816000050F08BF90EA020F1FBF54EA000C55EA42
:10817000020C7FEA645C7FEA655C00F0E2804FEA13
:108180005454D4EB5555B8BF6D420CDD2C4480EAF5
:10819000020281EA030382EA000083EA010180EA25
:1081A000020281EA0303362D88BF30BD11F0004F73
:1081B0004FEA01314FF4801C4CEA113102D04042A9
:1081C00061EB410113F0004F4FEA03334CEA1333E4
:1081D00002D0524263EB430394EA050F00F0A780FC
:1081E000A4F10104D5F1200E0DDB02FA0EFC22FAF7
:1081F00005F2801841F1000103FA0EF2801843FAEB
:1082000005F359410EE0A5F120050EF1200E012ADB
:1082100003FA0EFC28BF4CF0020C43FA05F3C01819
:1082200051EBE37101F0004507D54FF0000EDCF192
:10823000000C7EEB00006EEB0101B1F5801F1BD33B
:10824000B1F5001F0CD349085FEA30004FEA3C0C3F
:1082500004F101044FEA445212F5800F80F09A8035
:10826000BCF1004F08BF5FEA500C50F1000041EB39
:10827000045141EA050130BD5FEA4C0C404141EB3D
:108280000101013C28BFB1F5801FE9D291F0000F38
:1082900004BF01460020B1FA81F308BF2033A3F1E7
:1082A0000B03B3F120020CDA0C3208DD02F1140CDE
:1082B000C2F10C0201FA0CF021FA02F10CE002F119
:1082C0001402D8BFC2F1200C01FA02F120FA0CFC12
:1082D000DCBF41EA0C019040E41AA2BF01EB04515B
:1082E000294330BD6FEA04041F3C1CDA0C340EDC59
:1082F00004F11404C4F1200220FA04F001FA02F39C
:1083000040EA030021FA04F345EA030130BDC4F159
:108310000C04C4F1200220FA02F001FA04F340EA4E
:108320000300294630BD21FA04F0294630BD94F0FF
:10833000000F83F4801306BF81F480110134013DE6
:108340004EE77FEA645C18BF7FEA655C29D094EA57
:10835000050F08BF90EA020F05D054EA000C04BFD5
:108360001946104630BD91EA030F1EBF00210020C0
:1083700030BD5FEA545C05D14000494128BF41F05F
:10838000004130BD14F580043CBF01F5801130BDC3
:1083900001F0004545F0FE4141F470014FF000004E
:1083A00030BD7FEA645C1ABF194610467FEA655CFF
:1083B0001CBF0B46024650EA013406BF52EA0335A1
:1083C00091EA030F41F4002130BD00BF90F0000F8F
:1083D00004BF0021704730B54FF4806404F13204CB
:1083E0004FF000054FF0000150E700BF90F0000F84
:1083F00004BF0021704730B54FF4806404F13204AB
:1084000010F0004548BF40424FF000013EE700BF7A
:1084100042004FEAE2014FEA31014FEA02701FBF0A
:1084200012F07F4393F07F4F81F06051704732F03C
:108430007F4208BF704793F07F4F04BF41F4002193
:10844000704730B54FF4607401F0004521F00041F1
:108450001CE700BF50EA010208BF704730B54FF07B
:1084600000050AE050EA010208BF704730B511F07C
:10847000004502D5404261EB41014FF4806404F1B4
:1084800032045FEA915C3FF4D8AE4FF003025FEA3A
:10849000DC0C18BF03325FEADC0C18BF033202EBBE
:1084A000DC02C2F1200300FA03FC20FA02F001FA18
:1084B00003FE40EA0E0021FA02F11444BDE600BFBB
:1084C00070B54FF0FF0C4CF4E06C1CEA11541DBF6A
:1084D0001CEA135594EA0C0F95EA0C0F00F0DEF835
:1084E0002C4481EA030621EA4C5123EA4C5350EA1A
:1084F000013518BF52EA033541F4801143F480136B
:1085000038D0A0FB02CE4FF00005E1FB02E506F0FB
:108510000042E0FB03E54FF00006E1FB03569CF050
:10852000000F18BF4EF0010EA4F1FF04B6F5007F56
:1085300064F5407404D25FEA4E0E6D4146EB0606C8
:1085400042EAC62141EA55514FEAC52040EA5E5051
:108550004FEACE2EB4F1FD0C88BFBCF5E06F1ED8FB
:10856000BEF1004F08BF5FEA500E50F1000041EB32
:10857000045170BD06F0004646EA010140EA0200DF
:1085800081EA0301B4EB5C04C2BFD4EB0C0541EA01
:10859000045170BD41F480114FF0000E013C00F316
:1085A000AB8014F1360FDEBF002001F0004170BD3A
:1085B000C4F10004203C35DA0C341BDC04F1140453
:1085C000C4F1200500FA05F320FA04F001FA05F2DF
:1085D00040EA020001F0004221F0004110EBD370AC
:1085E00021FA04F642EB06015EEA430E08BF20EAD8
:1085F000D37070BDC4F10C04C4F1200500FA04F37B
:1086000020FA05F001FA04F240EA020001F000410C
:1086100010EBD37041F100015EEA430E08BF20EA7F
:10862000D37070BDC4F1200500FA05F24EEA020EC7
:1086300020FA04F301FA05F243EA020321FA04F0F6
:1086400001F0004121FA04F220EA020000EBD370AD
:108650005EEA430E08BF20EAD37070BD94F0000FAD
:108660000FD101F00046400041EB010111F4801FE1
:1086700008BF013CF7D041EA060195F0000F18BF92
:10868000704703F00046520043EB030313F4801FCE
:1086900008BF013DF7D043EA0603704794EA0C0F88
:1086A0000CEA135518BF95EA0C0F0CD050EA41069E
:1086B00018BF52EA4306D1D181EA030101F000411B
:1086C0004FF0000070BD50EA410606BF1046194643
:1086D00052EA430619D094EA0C0F02D150EA01364F
:1086E00013D195EA0C0F05D152EA03361CBF104690
:1086F00019460AD181EA030101F0004141F0FE412F
:1087000041F470014FF0000070BD41F0FE4141F4B2
:10871000780170BD70B54FF0FF0C4CF4E06C1CEAB2
:1087200011541DBF1CEA135594EA0C0F95EA0C0F67
:1087300000F0A7F8A4EB050481EA030E52EA033522
:108740004FEA013100F088804FEA03334FF0805543
:1087500045EA131343EA12634FEA022245EA111570
:1087600045EA10654FEA00260EF000419D4208BF21
:10877000964244F1FD0404F5407402D25B084FEACE
:108780003202B61A65EB03055B084FEA32024FF47A
:1087900080104FF4002CB6EB020E75EB030E22BFD7
:1087A000B61A754640EA0C005B084FEA3202B6EB97
:1087B000020E75EB030E22BFB61A754640EA5C0046
:1087C0005B084FEA3202B6EB020E75EB030E22BFD6
:1087D000B61A754640EA9C005B084FEA3202B6EBD7
:1087E000020E75EB030E22BFB61A754640EADC0096
:1087F00055EA060E18D04FEA051545EA16754FEAF8
:1088000006164FEAC30343EA52734FEAC2025FEA15
:108810001C1CC0D111F4801F0BD141EA00014FF0A4
:1088200000004FF0004CB6E711F4801F04BF014375
:108830000020B4F1FD0C88BFBCF5E06F3FF6AFAE91
:10884000B5EB030C04BFB6EB020C5FEA500C50F121
:10885000000041EB045170BD0EF0004E4EEA1131A4
:1088600014EB5C04C2BFD4EB0C0541EA045170BDAB
:1088700041F480114FF0000E013C90E645EA060EEF
:108880008DE60CEA135594EA0C0F08BF95EA0C0F1D
:108890003FF43BAF94EA0C0F0AD150EA01347FF465
:1088A00034AF95EA0C0F7FF425AF104619462CE73C
:1088B00095EA0C0F06D152EA03353FF4FDAE10469F
:1088C000194622E750EA410618BF52EA43067FF4F0
:1088D000C5AE50EA41047FF40DAF52EA43057FF480
:1088E000EBAE12E74A0011D212F5001211D20DD5EB
:1088F0006FF47873B3EB62520ED44FEAC12343F0A6
:10890000004343EA505323FA02F070474FF000004F
:10891000704750EA013002D14FF0FF3070474FF0FE
:10892000000070474FEA4102B2F1E04324BFB3F5C3
:10893000001CDCF1FE5C0DD901F0004C4FEAC002D6
:108940004CEA5070B2F1004F40EB830008BF20F0BA
:108950000100704711F0804F21D113F13872BCBF74
:1089600001F00040704741F480114FEA5252C2F1C9
:108970001802C2F1200C10FA0CF320FA02F018BF12
:1089800040F001004FEAC1234FEAD32303FA0CFC65
:1089900040EA0C0023FA02F34FEA4303CCE77FEAF4
:1089A000625307D150EA01331EBF4FF0FE4040F43E
:1089B0004000704701F0004040F0FE4040F40000ED
:1089C000704700BF80F0004002E000BF81F000412E
:1089D00042001FBF5FEA410392EA030F7FEA226C65
:1089E0007FEA236C6AD04FEA1262D2EB1363C1BFF5
:1089F000D218414048404140B8BF5B42192B88BF64
:108A0000704710F0004F40F4000020F07F4018BF86
:108A1000404211F0004F41F4000121F07F4118BFA6
:108A2000494292EA030F3FD0A2F1010241FA03FC4E
:108A300010EB0C00C3F1200301FA03F100F0004336
:108A400002D5494260EB4000B0F5000F13D3B0F1FE
:108A5000807F06D340084FEA310102F10102FE2A6D
:108A600051D2B1F1004F40EBC25008BF20F00100DD
:108A700040EA03007047490040EB0000013A28BF7C
:108A8000B0F5000FEDD2B0FA80FCACF1080CB2EBFF
:108A90000C0200FA0CF0AABF00EBC250524218437D
:108AA000BCBFD0401843704792F0000F81F4000122
:108AB00006BF80F400000132013BB5E74FEA4103F5
:108AC0007FEA226C18BF7FEA236C21D092EA030F61
:108AD00004D092F0000F08BF0846704790EA010FDB
:108AE0001CBF0020704712F07F4F04D1400028BF08
:108AF00040F00040704712F100723CBF00F50000EA
:108B0000704700F0004343F0FE4040F4000070471F
:108B10007FEA226216BF08467FEA236301464202CB
:108B200006BF5FEA412390EA010F40F480007047DE
:108B30004FF0000304E000BF10F0004348BF404284
:108B40005FEA000C08BF704743F0964301464FF0C0
:108B500000001CE050EA010208BF70474FF000031C
:108B60000AE000BF50EA010208BF704711F000435D
:108B700002D5404261EB41015FEA010C02BF84462D
:108B80000146002043F0B64308BFA3F18053A3F58C
:108B90000003BCFA8CF2083AA3EBC25310DB01FAD3
:108BA00002FC634400FA02FCC2F12002BCF1004F57
:108BB00020FA02F243EB020008BF20F001007047E8
:108BC00002F1200201FA02FCC2F1200250EA4C003C
:108BD00021FA02F243EB020008BF20EADC70704782
:108BE0004FF0FF0C1CEAD0521EBF1CEAD15392EA90
:108BF0000C0F93EA0C0F6FD01A4480EA010C40026C
:108C000018BF5FEA41211ED04FF0006343EA5010C5
:108C100043EA5111A0FB01310CF00040B1F5000F07
:108C20003EBF490041EAD3715B0040EA010062F1B6
:108C30007F02FD2A1DD8B3F1004F40EBC25008BFA0
:108C400020F00100704790F0000F0CF0004C08BFBE
:108C500049024CEA502040EA51207F3AC2BFD2F18B
:108C6000FF0340EAC250704740F400004FF0000399
:108C7000013A5DDC12F1190FDCBF00F000407047D3
:108C8000C2F10002410021FA02F1C2F1200200FA11
:108C900002FC5FEA310040F1000053EA4C0308BFD8
:108CA00020EADC70704792F0000F00F0004C02BF29
:108CB000400010F4000F013AF9D040EA0C0093F0A4
:108CC000000F01F0004C02BF490011F4000F013BFE
:108CD000F9D041EA0C018FE70CEAD15392EA0C0F6C
:108CE00018BF93EA0C0F0AD030F0004C18BF31F0D7
:108CF000004CD8D180EA010000F00040704790F0AD
:108D0000000F17BF90F0004F084691F0000F91F050
:108D1000004F14D092EA0C0F01D142020FD193EA16
:108D20000C0F03D14B0218BF084608D180EA01009E
:108D300000F0004040F0FE4040F40000704740F07A
:108D4000FE4040F4400070474FF0FF0C1CEAD05248
:108D50001EBF1CEAD15392EA0C0F93EA0C0F69D0A4
:108D6000A2EB030280EA010C49024FEA402037D00F
:108D70004FF0805343EA111143EA10130CF0004006
:108D80008B4238BF5B0042F17D024FF4000C8B42F6
:108D900024BF5B1A40EA0C00B3EB510F24BFA3EBD6
:108DA000510340EA5C00B3EB910F24BFA3EB9103A6
:108DB00040EA9C00B3EBD10F24BFA3EBD10340EA00
:108DC000DC001B0118BF5FEA1C1CE0D1FD2A3FF646
:108DD00050AF8B4240EBC25008BF20F001007047FB
:108DE0000CF0004C4CEA50207F32C2BFD2F1FF039E
:108DF00040EAC250704740F400004FF00003013ACF
:108E000037E792F0000F00F0004C02BF400010F472
:108E1000000F013AF9D040EA0C0093F0000F01F086
:108E2000004C02BF490011F4000F013BF9D041EAA8
:108E30000C0195E70CEAD15392EA0C0F08D14202DB
:108E40007FF47DAF93EA0C0F7FF470AF084676E7AE
:108E500093EA0C0F04D14B023FF44CAF08466EE787
:108E600030F0004C18BF31F0004CCAD130F0004255
:108E70007FF45CAF31F000437FF43CAF5FE700BFAD
:108E80004FF0FF3C06E000BF4FF0010C02E000BFD6
:108E90004FF0010C4DF804CD4FEA40024FEA410378
:108EA0007FEA226C18BF7FEA236C11D001B052EA2E
:108EB000530C18BF90EA010F58BFB2EB030088BFF4
:108EC000C81738BF6FEAE17018BF40F00100704763
:108ED0007FEA226C02D15FEA402C05D17FEA236C45
:108EE000E4D15FEA412CE1D05DF8040B704700BF8C
:108EF000844608466146FFE70FB5FFF7C9FF002823
:108F000048BF10F1000F0FBD4DF808EDFFF7F4FF5B
:108F10000CBF012000205DF808FB00BF4DF808EDF4
:108F2000FFF7EAFF34BF012000205DF808FB00BF17
:108F30004DF808EDFFF7E0FF94BF012000205DF839
:108F400008FB00BF4DF808EDFFF7D2FF94BF0120EA
:108F500000205DF808FB00BF4DF808EDFFF7C8FFE3
:108F600034BF012000205DF808FB00BF4FEA40023B
:108F7000B2F1FE4F0FD34FF09E03B3EB12620DD947
:108F80004FEA002343F0004310F0004F23FA02F0B1
:108F900018BF404270474FF00000704712F1610F58
:108FA00001D1420205D110F0004008BF6FF000402F
:108FB00070474FF0000070477BB972B90029BEBFFF
:108FC00000204FF0004106E008BF00281CBF6FF0F2
:108FD00000414FF0FF3000F057B8ADF1080C6DE9DB
:108FE00004CE002909DB002B1ADB00F02BF9DDF899
:108FF00004E0DDE9022304B07047404261EB410127
:10900000002B1BDB00F01EF9DDF804E0DDE9022394
:1090100004B0404261EB4101524263EB43037047AD
:10902000524263EB430300F00DF9DDF804E0DDE9A3
:10903000022304B0404261EB41017047524263EBAE
:10904000430300F0FFF8DDF804E0DDE9022304B09B
:10905000524263EB4303704753B94AB9002908BF32
:1090600000281CBF4FF0FF314FF0FF3000F00CB86C
:10907000ADF1080C6DE904CE00F0E4F8DDF804E091
:10908000DDE9022304B07047704700BF4FF0FF3C9A
:1090900006E000BF4FF0010C02E000BF4FF0010CF2
:1090A0004DF804CD4FEA410C7FEA6C5C4FEA430C6B
:1090B00018BF7FEA6C5C1BD001B050EA410C0CBFBA
:1090C00052EA430C91EA030F02BF90EA020F00201C
:1090D000704710F1000F91EA030F58BF994208BF83
:1090E00090422CBFD8176FEAE37040F00100704740
:1090F0004FEA410C7FEA6C5C02D150EA013C07D197
:109100004FEA430C7FEA6C5CD6D152EA033CD3D0E1
:109110005DF8040B704700BF8446104662468C46DB
:109120001946634600E000BF01B5FFF7B7FF00280E
:1091300048BF10F1000F01BD4DF808EDFFF7F4FF37
:109140000CBF012000205DF808FB00BF4DF808EDC2
:10915000FFF7EAFF34BF012000205DF808FB00BFE5
:109160004DF808EDFFF7E0FF94BF012000205DF807
:1091700008FB00BF4DF808EDFFF7CEFF94BF0120BC
:1091800000205DF808FB00BF4DF808EDFFF7C4FFB5
:1091900034BF012000205DF808FB00BF4FEA410CFE
:1091A0007FEA6C5C02D150EA013C0AD14FEA430CE1
:1091B0007FEA6C5C02D152EA033C02D14FF000001E
:1091C00070474FF0010070474FEA410212F500125C
:1091D00015D211D56FF47873B3EB625212D94FEAFE
:1091E000C12343F0004343EA505311F0004F23FAE8
:1091F00002F018BF404270474FF00000704750EA3D
:10920000013005D111F0004008BF6FF000407047F9
:109210004FF00000704700BF4FEA40024FEA4103A1
:109220007FEA226C02D15FEA402C08D17FEA236CEE
:1092300002D15FEA412C02D14FF0000070474FF09D
:10924000010070472DE9F04786468C460846089E87
:10925000154674461946002B40F0C1808542B2FA8B
:1092600082F245D94AB1C2F1200300FA02FC9540CE
:1092700094402EFA03F343EA0C0C4FEA154EA8B2C1
:10928000230CBCFBFEF80EFB18CC08FB00F943EAEC
:109290000C43994528D9EB1808F1FF3704D29945BA
:1092A00002D9A8F102072B44A3EB0903A4B2B3FB34
:1092B000FEFC0EFB1C330CFB00F044EA0344A0420E
:1092C00014D92C190CF1FF3304D2A04202D9ACF10D
:1092D00002032C44241A43EA07401EB1D440002361
:1092E00034607360BDE8F0874746DDE76346F1E729
:1092F00092BB431B01214FEA154EAFB2200CB3FBCA
:10930000FEFC0EFB1C330CFB07F840EA03439845B8
:1093100061D9EB180CF1FF3004D2984502D9ACF1B9
:1093200002002B44A3EB0803A4B2B3FBFEFC0EFB2C
:109330001C330CFB07F744EA0344A7424DD92C1910
:109340000CF1FF3304D2A74202D9ACF102032C4442
:10935000E41B43EA0040C0E7C2F12003954094407B
:1093600020FA03F12EFA03F34FEA154E9040AFB204
:109370000343B1FBFEFC0EFB1C10190C0CFB07F8A1
:1093800041EA0041884522D969180CF1FF3004D226
:10939000884502D9ACF102002944A1EB08019BB237
:1093A000B1FBFEFC0EFB1C110CFB07F743EA01436B
:1093B0009F420ED9EB180CF1FF3104D29F4202D923
:1093C000ACF102012B44DB1B41EA004193E760460C
:1093D000E3E76146F7E76046A4E76346B8E7834200
:1093E00006D916B9002108467CE7C6E900E0F9E78E
:1093F000B3FA83F78FB9834201D3724508D8BEEB25
:10940000020460EB030301209C461EB9002169E7BA
:109410003846FAE7C6E9004CF8E7C7F1200CBB4034
:109420000EFA07F522FA0CF42EFA0CF1BA401C439E
:1094300020FA0CF3B8404FEA144901431FFA84FEA6
:10944000B3FBF9F809FB18300B0C08FB0EFA43EAE2
:1094500000439A4540D9E31808F1FF3004D29A45F9
:1094600002D9A8F102002344A3EB0A0389B2B3FB9B
:10947000F9F809FB183308FB0EFE41EA03418E455B
:109480002CD9611808F1FF3304D28E4502D9A8F116
:109490000203214443EA0040A1EB0E01A0FB029825
:1094A0004145CE46434602D306D14D4504D201384C
:1094B000B9EB020E68EB0403002EA7D0B5EB0E0249
:1094C00061EB030101FA0CFC22FA07F3F9404CEAC4
:1094D0000303C6E9003199E74046C5E74346D9E7AB
:1094E00010F8012B11F8013B012A28BF9A42F7D04E
:1094F000D01A7047034613F8012B002AFBD1181A23
:109500000138704700000000032973B50546144672
:1095100071D8002A40D0072A5CD15A681C681346CB
:109520003948D117C4FB0031012B71F1000225DB52
:1095300000F56E1000F65D70181841F1000130A3BF
:10954000D3E90023FFF738FD80B202281ED004289B
:109550001ED008281ED0102833D103232B492A6996
:1095600051F82310284611615268232114693022D2
:10957000A4461B0102B0BDE870406047244818189B
:1095800061F100011EA3D3E90023DBE70023E5E737
:109590000123E3E70223E1E71A881E4B33F8021B9D
:1095A0008A420BD12E692021736828469B680DF1F1
:1095B00007029847002807DA02B070BD01340B2C6F
:1095C000ECD16FF01500F7E79DF80720130704D4DE
:1095D000082C05D16FF08500EEE70A2C08BF09249E
:1095E000736802F00F0242EA041220212846DB6869
:1095F000D2B29847E0E702B0BDE8704005F070BC19
:109600003AA395000000000040420F00CCC50020A6
:10961000632EB5FFF4F402002DE9F04198460023D3
:1096200086B0CDE9043304230D4617460646019360
:10963000002800F0B580002900F0B280062104A8BF
:1096400012F041FC044648B103460121584A5948EA
:1096500012F099FD204606B0BDE8F081014604AA4B
:10966000304612F00BFC044648B10346524A012131
:10967000504812F088FD04A812F04FFCEAE76A4651
:10968000012104A812F0FBFC044610B103464B4A2A
:10969000EDE7009BB3B1042B1AD0052B0CBF0923B7
:1096A000FF232B70032101AB02AA04A812F013FDC3
:1096B000064678B10346424A01213E4812F063FD56
:1096C0003446D8E7002300202B706860A860D2E7FA
:1096D0000723E6E7019B002BF4D018336B4403F813
:1096E000100C02A9384614F098FD0222314602A857
:1096F0000EF08CFC2B78C0B2092B06D10F2824D990
:109700006FF0150423462F4AB1E70F28F8D8072B2E
:1097100022D12D4B2D4F33F81000D8B1FEF766FE45
:1097200021A3D3E90023FEF7CBFEFFF7FBF80421CA
:1097300068600DEB010302AA04A8019112F0CBFCB2
:10974000064660B10346224AB6E7224B224F33F861
:109750001000E2E72148EAE76FF07F04D2E7019BBF
:1097600002A918336B4403F8100C404614F055FD61
:109770000222314602A80EF049FCC3B20F2B07D9D2
:109780000121174A0B4812F0FEFC6FF0150472E736
:10979000581CC0B2FFF7D0F93946FFF721FA95E718
:1097A0006FF0150456E700BF7B14AE47E17A244002
:1097B000A410030014EB0200CD100300F610030008
:1097C00018110300441103002AF502000AD7A33F31
:1097D000681103000AF502000AD723400AD7A34004
:1097E0009311030000000000F8B506460F4600F094
:1097F0003BF81B4B04460D4693F90030013312D061
:109800003046394614F0C1FC68B13046394610A3E1
:10981000D3E90023FFF7B8FC40B110F0BEF90024F3
:109820002223104D036020462946F8BD0AA3D3E940
:10983000002330463946FFF789FC0028F3D010F0AA
:10984000ACF92223002400250360ECE7AFF300808D
:10985000EF39FAFE422E864051302DD5104987C08F
:10986000CBC700200000F07F2DE9FF4721F0004228
:10987000A94F04460D46BA424FEAD1762FD9A74FD9
:10988000BA4212D88EA3D3E90023FFF77DFCF0B9CA
:10989000204629468CA3D3E90023FFF757FC002874
:1098A00000F09C80002400250CE0C1F31303024665
:1098B000034305D00B46FEF74DFC04460D4601E080
:1098C000002EEFD12046294604B0BDE8F08780A3E2
:1098D000D3E9002310461946FEF7F2FDEDE7904B61
:1098E0009A4240F2A7808F4B9A4277D88E4BF40071
:1098F000C6F1010A03EBC603AAEB060AD3E900236B
:10990000FEF726FC894B804689462344D3E9003480
:10991000CDE90034DDE9002340464946FEF718FC56
:1099200004460D4622462B4620462946FEF7C8FD32
:1099300006460F4668A3D3E90023FEF7C1FD68A3DE
:10994000D3E90023FEF704FC32463B46FEF7B8FDA0
:1099500065A3D3E90023FEF7FDFB32463B46FEF745
:10996000AFFD63A3D3E90023FEF7F2FB32463B468B
:10997000FEF7A6FD60A3D3E90023FEF7EBFB32461A
:109980003B46FEF79DFD02460B4620462946FEF764
:10999000DFFB02460B4606460F4620462946FEF7E9
:1099A0008FFDCDE90201BAF1000F5AD100224FF02C
:1099B000804330463946FEF7CBFB02460B46DDE9D5
:1099C0000201FEF7A7FE22462B46FEF7C1FB024628
:1099D0000B4600205649FEF7BBFB6EE7554B204671
:1099E000294603EBC60646A3D3E90023FEF768FD2C
:1099F000D6E90023FEF7AEFBFFF7E6FB8246FEF753
:109A0000F5FC06460F4640A3D3E90023FEF758FDB8
:109A100002460B4620462946FEF79AFB80468946B9
:109A2000304639463AA3D3E90023FEF749FDCDE994
:109A300000016FE7404B9A420ED825A3D3E90023DB
:109A4000FEF788FB00223A4BFFF79EFB38B100225D
:109A5000374B204629462EE74FF0000A62E7824640
:109A600060E732463B4600204FF08041FEF770FB36
:109A700002460B46DDE90201FEF74CFE02460B46AC
:109A8000DDE90001FEF764FB42464B46FEF760FB52
:109A900002460B4600202649FEF75AFB6FF47F7200
:109AA000924502DB01EB0A5107E70AF57A7A0022B8
:109AB0004FF0B87301EB0A510EE700BFAFF300801F
:109AC000EF39FAFE422E864051302DD5104987C01D
:109AD0009C7500883CE4377ED0A4BE726937663E30
:109AE000F16BD2C541BDBB3E2CDE25AF6A56113F9E
:109AF00093BDBE166CC1663F3E5555555555C53F85
:109B0000FE822B654715F73F0000E0FE422EE63F40
:109B1000763C7935EF39EA3D412E8640FFFFEF7FF5
:109B2000422ED63FB1A2F03FE8EB0200D8EB020094
:109B30000000F03FF8EB0200FFFF2F3E00000000A6
:109B4000B1F5801F02460B462DE9F04F0D4687B058
:109B500024DA21F00044044308D10022002300202D
:109B6000C949FEF7D7FD07B0BDE8F08F002904DA38
:109B7000FEF7EEFA00220023F3E70022C34BFEF7C4
:109B80009FFC0B460D4602466FF03501C0488542EA
:109B900006DD10461946FEF7DDFAE4E70021F5E799
:109BA0002C15C5F3130510460022A4F2FF340C4413
:109BB00005F5152101F6647101F4801686F07F51D8
:109BC00004EB165481F4401141EA05031946B14BE8
:109BD000FEF7BEFAAB1C82468B46C3F3130300228A
:109BE000022B53DC0023FFF7A7FAD0B1002C00F0C2
:109BF00020812046FEF7FAFB06460F468EA3D3E9E6
:109C00000023FEF75DFC04460D46304639468CA322
:109C1000D3E90023FEF754FC02460B4620462946B2
:109C2000B9E789A3D3E9002350465946FEF748FC1B
:109C300002460B4600209849FEF78AFA06460F4670
:109C400052465B4650465946FEF73AFC02460B46E2
:109C500030463946FEF734FC06460F4614B9324604
:109C60003B46A0E02046FEF7C1FB8046894672A332
:109C7000D3E90023FEF724FC04460D46404649463E
:109C80006FA3D3E90023FEF71BFCA5E04FF0804350
:109C9000A5F5C226FEF75EFA02460B465046594627
:109CA000C5F5D725FEF736FDA6F27A465135CDE942
:109CB000000120463543FEF799FBDDE90023CDE99D
:109CC000020110461946FEF7FBFB02460B46CDE9A2
:109CD0000423FEF7F5FB804689465DA3D3E9002304
:109CE000FEF7EEFB5CA3D3E90023FEF733FA42460E
:109CF0004B46FEF7E5FB5AA3D3E90023FEF72AFA09
:109D000042464B46FEF7DCFB57A3D3E90023FEF7A0
:109D100021FADDE90423FEF7D3FB55A3D3E90023A1
:109D2000CDE9040140464946FEF7CAFB52A3D3E9F8
:109D30000023FEF70FFA42464B46FEF7C1FB50A345
:109D4000D3E90023FEF706FA42464B46FEF7B8FB7E
:109D500002460B46DDE90401FEF7FCF9002D8046C2
:109D6000894648DD00224C4B50465946FEF7A8FB79
:109D700052465B46FEF7A4FB02460B4606460F46DC
:109D800040464946FEF7E6F9DDE90023FEF798FB79
:109D90008046894664B902460B4630463946FEF78E
:109DA000D7F902460B4650465946FEF7D1F9DAE696
:109DB00021A3D3E90023DDE90201FEF781FB04467C
:109DC0000D461FA3D3E90023DDE90201FEF778FB6E
:109DD00042464B46FEF7BEF902460B463046394630
:109DE000FEF7B6F952465B46FEF7B2F902460B465D
:109DF00020462946D9E702460B4650465946FEF70B
:109E0000A7F9DDE90023FEF75BFB06460F46002CB1
:109E10003FF425AF08A3D3E90023DDE90201FEF7F3
:109E20004FFB04460D4606A3D3E90023DDE90201FA
:109E300029E70020002196E60000E0FE422EE63FE2
:109E4000763C7935EF39EA3D555555555555D53F51
:109E500044523EDF12F1C23FDE03CB966446C73F59
:109E6000599322942449D23F935555555555E53F72
:109E70009FC678D0099AC33FAF788E1DC571CC3F7D
:109E800004FA97999999D93F000050C300005043B4
:109E9000FFFFEF7F0000F03F0000E03FF8B502F168
:109EA000080323F0070300AFADEB030D054668463A
:109EB000144614F08EF900236E460DF804308AB073
:109EC0006A460849D661C2E9051507491162074982
:109ED00042F8101F4FF42351054802F0D5F8BD4653
:109EE000F8BD00BF50F502000002010304000002AB
:109EF00024EB02002DE9F04389B00B7806460C46AE
:109F000002AF092B00F2D680DFE813F00A00400010
:109F10004400C000D400D400D400C700D400CE0058
:109F2000CD6935B12B46644A012164480EF0BBFD72
:109F300028E00321624A61480FF001FD614B07F1FF
:109F40000C0493E80700604B84E807007C606C46D3
:109F50008AB0BB6002AA5D4B53615D4B93610523E0
:109F6000D3614FF4007313845A4B42F8103F4FF4FF
:109F7000135152482B4602F087F83046A546391D4A
:109F800010F0E2FC1C37BD46BDE8F083CB69524AB5
:109F90000321CAE74A69CB690321009247484F4A27
:109FA0000FF0E0FCD4F81480B8F1800F12D9DFF87C
:109FB000309149463046A8F1800210F072FD051E2E
:109FC00027D028DBA8EB0508B8F1800FF1D86FF097
:109FD000790901E04FF0000942463046404910F04F
:109FE00063FD0546B8B9237B012B06D1238B304690
:109FF000BB8107F10C0110F059FCB9F1000F16D02C
:10A0000063698022012100922C48364A0FF0AAFC95
:10A01000B8E76FF00405237B012B06D1238B304674
:10A02000BB8107F10C0110F041FC002D17DB6269C8
:10A030002B492D48FFF732FF05222C49284814F000
:10A04000F4F810B911F0F1FE9CE7062228492448E3
:10A0500014F0EBF8002895D111F0EAFE92E715F123
:10A060007A0FCDD02B460121224A14480EF01BFD59
:10A070000321214A11480FF062FC304610F03CFCED
:10A08000034600283FF47EAF1C4A4DE7CB690BB175
:10A090001B4A49E78B881B4A7AE7CB690BB11A4AFE
:10A0A00042E78B88194A73E7CB69002B3FF46AAF0C
:10A0B000174A39E7174A6BE755F5020024EB02000F
:10A0C0006DF5020080EB02000100D20483F502006E
:10A0D0009DF5020004000001A3F50200C0F5020096
:10A0E00076DD0020DEF502002DF6020038F60200D3
:10A0F0003EF6020045F6020065F6020082F6020016
:10A100009BF60200B1F60200C6F60200DCF6020081
:10A11000F1F6020009F702002DE9F0434FF00508BF
:10A1200089B0DFF8749000AF064614461D46C7E9B3
:10A1300005233974C7F80890C7F80C8004217818F3
:10A1400003F000F97B682A46BB83BB7F214623F0DE
:10A15000030312486C46BB77FFF7A0FE8AB06A463D
:10A160000F4BC2F81C80C2E905394FF40073138409
:10A170000C4B42F8103F00234FF413510A4801F0F2
:10A1800083FF07F10801A546304610F04BFB24374A
:10A19000BD46BDE8F08300BF27F702002DF702009F
:10A1A0003AF702000400000124EB02002DE9F04F11
:10A1B00001269DB002AF07F11408044610F0D9FA49
:10A1C00054220021404614F011F83B46424600213B
:10A1D000C7E9076645480FF0E2FC054688B103462B
:10A1E0003146434A43480EF05EFC434A31464148FB
:10A1F0000FF0A5FB6FF0090528466C37BD46BDE89A
:10A20000F08F4FF0080A3E68DFF8F09039482EB31F
:10A21000B369082B4AD1F36939495B6801204B6067
:10A2200045F6073308804B803E1D1023324604312B
:10A2300003F08CFAE94688B002AB324AC3E905263E
:10A240004FF400729A831A462F4B42F8103F0023B6
:10A250004FF4E651274801F017FFCD4638680FF05C
:10A26000A0FC274B17216363284B4046A364284A70
:10A270000AF0AAFA034668B30121264A1D480EF0E7
:10A2800012FC2548E062FFF735F9042284F85E20CD
:10A29000224A0023E26480222149C4E90E33C4E942
:10A2A00015122063226584F82430A5E7EB468AB0B6
:10A2B00002AAC2E90593182313620523C2F81CA061
:10A2C00042F8103F00234FF4215101F0DDFEDD463E
:10A2D00036689BE787F823000F231421114ACDF835
:10A2E00000800D480DF0A4FCCBE700BF4FF7020043
:10A2F0005DF7020024EB020074F70200B1F70200E0
:10A3000038DD00209BF7020003000001F59E0100EC
:10A31000D4F70200DCF7020062DD002076DE0020C8
:10A32000F6DD0020FDF702002123012110B5074AC8
:10A330000748FFF7F1FE034630B1BDE810400321A6
:10A34000044A05480EF0BFBB10BD00BF06F802006E
:10A3500070D3002028F8020024EB020098B50446D0
:10A360000321224A224800AF0EF0ABFB23781BB139
:10A37000032B20D0BD4698BD237A012B19D0052B85
:10A38000F8D11C4B6C4688B06A461B49C2E90513DC
:10A390004FF400739383194B42F8103F00234FF49E
:10A3A000E651134801F070FEA54615480CF03AFA44
:10A3B000E0E7144BE6E7217A134A144B6C4688B069
:10A3C000012908BF13466A461149C2E905134FF433
:10A3D00000739383094B42F8103F00234FF4E6517A
:10A3E000034801F051FEA546C4E700BF7FF8020014
:10A3F00024EB02005CF802008BF80200030000016D
:10A4000078C9002043F8020070F802007AF80200D0
:10A41000ABF802002DE9F047002582B0624C032121
:10A42000624A634802AF0EF04CFB2E46A146DFF8AD
:10A430008481DFF87CA194F8543053B1B4F85230E1
:10A44000B4F8562003210092504642460FF08AFA93
:10A45000013501360C2E04F10C04ECD12B460321FE
:10A46000554A53480EF02FFB0122E8214E480BF0CD
:10A470006BFB804640B103460121504A4C480EF028
:10A4800022FBBD46BDE8F08799F85030DB07F8D5D0
:10A4900011F0CBFCD9E9000100220023FDF75AFEA0
:10A4A0006D4688B002AC0426A246454BC4E90601BD
:10A4B00063614AF8106F4FF40351434652463C48DB
:10A4C00001F0E2FDD9E90201AD4600220023FDF7CB
:10A4D00041FE88B03B4BC4E90601636126614FF43D
:10A4E000035143465246324801F0CEFDAD460021AD
:10A4F000D9F81000FEF76CFA88B0334B6361FDF7B2
:10A5000087FF2661C4E906014FF4035143465246D2
:10A51000274801F0B9FDAD468AB099F8384099F85E
:10A52000390099F83A10B9F83C3002AA5362062370
:10A53000DFF898C0C2E90701C2E905C442F8103F3C
:10A54000234C43464FF44351194801F09DFD94F8C4
:10A550000080AD46B8F1000F93D113F028FC88B00D
:10A560000DF108094FF47A721A4BC9F81430A0FBA8
:10A57000020302FB0131C00B4FF47A72002340EA60
:10A580004140C90BFEF718FD4A46C9E9060142F8E9
:10A59000106F4FF403514346054801F075FD012348
:10A5A000AD4623706DE700BF30CA0020B8F8020046
:10A5B00024EB0200C5F80200D5F80200F6F802000C
:10A5C00019F902002FF9020045F902005DF90200B5
:10A5D000F6DE002081F90200072805D0092808D0FE
:10A5E000012808D1FFF716BF034A032103480EF0E4
:10A5F00068BA034AF9E770479EF9020024EB0200AB
:10A60000B0F90200F8B500AF6C4688B06A46724BEC
:10A610005361724B93614FF400739383704B42F814
:10A62000103F00234FF4E6516E4801F02DFDA54682
:10A6300005F068FF20B101216B4A6A480EF041FA2B
:10A6400003216A4A67480EF03CFA05F0B3F8034666
:10A6500060B1674A012163480EF035FA0121654A6D
:10A6600060480EF02EFA0020BD46F8BD0321624A74
:10A670005C480EF026FA614811F069FD034608B106
:10A680005F4AE7E74FF0FF324FF0FF335D480CF0D1
:10A69000EDF8544803215C4A0EF013FA5B480BF0C6
:10A6A000E3FBC8B15A4A01214E480EF00AFA594854
:10A6B00005F052FF20B10121574A4A480EF001FA35
:10A6C0005648FFF773FD0346002838D0544A01214D
:10A6D00044480EF0F8F9C6E70321524A41480EF00B
:10A6E000F0F90BF051FB044608B14F4ADBE711F0DB
:10A6F0009CFB00214FF480300CF09EFD204611F0B1
:10A7000097FBD4E701340AD03C230321474A35485C
:10A710000EF0D9F94FF4F01000210CF08DFD03215B
:10A72000434A30480EF0CDF93C4810F039F8034662
:10A7300040B1404A01212B480EF0C5F9E2E704463A
:10A740003D4DECE7294635480EF0AFF90346F8B920
:10A75000324E304610F06DF90246012128460FF0C6
:10A7600017FB002816DA0FF018FA344A03680121A3
:10A770001C480EF0A8F90321314A1A480EF0A1F93D
:10A78000264810F0B9F803460028BBD02D4AD1E77F
:10A790002D4A9CE7304610F027F9034620B110F10E
:10A7A0000B0F01D0294AE2E7EB88D90706D53046DE
:10A7B00010F056F9034608B1254AD8E7B5F9063036
:10A7C0001A0705D5234A012106480EF07AF9D2E787
:10A7D0009B06BED5204AF6E7CBF90200E7F9020056
:10A7E0000300000124EB0200FBF9020020FA020042
:10A7F0003BFA02000DFB02006DFA02005DA30100AE
:10A8000087FA020078C90020B0FA0200D9A5010039
:10A81000C9FA0200CB8A02002BFB020070D3002091
:10A8200054FB0200EAFA0200F8FA020079FB020087
:10A8300097FB0200BFFB020068D30020EFFB020081
:10A8400043FC02005DFC0200D9FB020003FC020095
:10A850001AFC020032FC02003AFC02002DE9F04F23
:10A8600091B0009302F004030293C2F3C2030133D8
:10A87000840705460E46DDF868900392059340F084
:10A88000BB81041D30B1072909D86FF01B0011B03E
:10A89000BDE8F08F01F00706341DC6F10806009BE5
:10A8A0004FF000084FF0040A591E4FF0FF3347469F
:10A8B0000193C3465346CDF810800DB1009A226033
:10A8C0000598002800F3E8809848009A824203D354
:10A8D00097488242C0F0E080039AA4EB050E9207ED
:10A8E0004FEA9E0000F103810F2F00F2B180002D8E
:10A8F00000F0058107F140020DEB020C019A0CF803
:10A90000200C0CF8102C049801300490E7E07A2811
:10A910005DD84B280ED8472859D829282DD8252866
:10A9200052D054D820287AD02338D0F1000B4BEBEA
:10A93000000B74E04C382E2849D8DFE800F070484E
:10A94000484848484848484848484B484848484884
:10A9500048484859484B4B595959704B6D487048B5
:10A96000184B184848827F4B48484B487F000020CE
:10A970004FF0000B4FF0040A38E001222A38C0B231
:10A9800002FA00F010EA0E0F49D110F0625C2FD1EC
:10A9900010EA020B43D06046013C5444B4FBFAF485
:10A9A0000AFB04F4002D61D0A3EB050CA444B445CC
:10A9B0003FF66BAF002868D1042B47D159F8043B10
:10A9C0002360042304342AE0019A013A01924FF0F3
:10A9D000000B24E011F8010C6C2834D1002011F890
:10A9E000023C83466C2BC5D14FF0080A5346D3E78F
:10A9F00009F1070929F00709073424F00704F9E8E9
:10AA000002AB35B106982044B0423FF63EAFC4E9F0
:10AA100000AB4FF0000B08344FF0080A534611F812
:10AA2000010F002878D0BBF1000F7FF470AF25280C
:10AA3000F5D14FF0010B019B013301934FF0040A54
:10AA4000ECE7584694E700208346A5E7082B02D0A0
:10AA50006FF015001BE709F1070929F00709F9E86C
:10AA60000223C4E9002308230834D8E768B9042B7B
:10AA700002D109F10409A4E7082BE9D109F107097A
:10AA800029F0070909F10809EDE7059A013A05924D
:10AA900059F8042B009210E7039A900720D54FF045
:10AAA000010CA4EB050E4FEA9E00BEF5007FCFD24D
:10AAB0000F2FCDD8F5B107F140020DEB020E019A30
:10AAC000C0B20EF8200C0EF8102CBCF1000F3FF4B1
:10AAD0001AAF60F07F000EF8200C08F10108013772
:10AAE000C5F108024FF6DA7E0434069297E74FF07C
:10AAF000000CDAE7BCF1000F01D00136EFE7029855
:10AB000002360028EBD10098CDE90631FEF7F2FCC1
:10AB1000DDE906310644E2E7631BB3F5806F97D2A7
:10AB200045B9A6F10804E018B1E600BFD8E6020076
:10AB30004C1F0300029A9B0828602B709DF8103070
:10AB4000C2B1EB7085F80280B8F1000F05D0002289
:10AB500008A8C5F1010C97420ED14FF0000AC5F1CB
:10AB600001030DF1200901930DF1300B574512D16E
:10AB7000601B8CE66B70E5E710F8013B190608D501
:10AB800004EB0C0EB64503F07F033FF67EAE04F8EF
:10AB9000013B0132DFE7B8F1000F03D099F9002043
:10ABA000002A17DB029BD3B11AF80B2004F8012B03
:10ABB0000022019B98182044B0423FF666AE99F8F7
:10ABC0000000009904F8010B2046039213F001FBEA
:10ABD000039A14440AF1010A09F10109C6E799F838
:10ABE000002055F822300093029B009845F822304F
:10ABF000FEF780FC421CDCE76FF00D0047E600BF6B
:10AC00002DE9F04F97B000AFD7F880B03B62CBF39F
:10AC1000C0030446894690F802A0FA62BB6141B9BC
:10AC2000457800780AEB800020444D4517D8A0EB0A
:10AC30000409E378FB61BAF1000F02D01BF0010FA9
:10AC400016D1FB6953BBFB6A1BB1494620463A6AE1
:10AC500098474D4628465C37BD46BDE8F08F461CF8
:10AC60003046FEF747FC0130304409F10109DCE7CA
:10AC7000626823787A62FA6A9900796104EB830149
:10AC8000002A40F001810E464FF000084D4601EBCE
:10AC90000A094E454CD101EB0A0610E01BF0020FE9
:10ACA000D1D023789A007A61626804EB83017A62DA
:10ACB000FA6A002A77D14D46904601EB0A061BF04E
:10ACC000050F0CBF02230123FB62FB6906EB430A5D
:10ACD0000BF00203BB625645BCD016F8021B16F8F7
:10ACE000013C54F82390AF4B994502D3AE4B9945A4
:10ACF00036D3BB69002B40D0786A0EF0CBF9002820
:10AD00003BD0E9468AB06A46A84B53617B6AC2E9E8
:10AD100006314FF400731384A54B42F8103F002313
:10AD20004FF41251A34801F0AFF9023DCD46D2E7EE
:10AD300016F8013BF96254F82300FEF7DBFBD7F865
:10AD40008430F96A01304BB1D7F8883098453EBF5E
:10AD5000D7F8843023F8180008F10108054498E773
:10AD6000BB6923B1786A0EF095F90028C9D11BF0B0
:10AD7000010F05D1FB6AED1AADE7BB6A002BAAD023
:10AD80004846FEF7B7FBD7F8843053B1D7F8883080
:10AD900098453FBFD7F88420431C22F8183008F1AB
:10ADA0000108054497E7BAF1000F73D01BF00406C1
:10ADB00073D0D046002607F1480052463B61B96285
:10ADC00013F007FAB96A3B6901EB0A02BA62FA6941
:10ADD000F9695200FA60BA6A02EB41023A610BF07B
:10ADE0000202BA603A69B96A8A4258D162781BF0A5
:10ADF000020F18BF00217A6208BF4FEA5801B2184B
:10AE00001BF0010FD2B240F09F801BF0040F14BF63
:10AE100040460020BB616270A070E17020463A6A33
:10AE20007969FB6A9847051EFFF614AFBB69414676
:10AE300023707B6A3A6A6370FB6984F802A0E3704E
:10AE400007F14800FB6A9847B0F10008C0F2B480EF
:10AE50007B69A9EB0A01C91AFB683A6AC91AD7E9E2
:10AE60000A0398470028C0F2A9804FF0000BA844BD
:10AE700008EB000507F1380AB34567D300213A6AA9
:10AE80000846FB6A9847E5E656464FF0000807F18A
:10AE9000380092E75646D04696E7B04694E7BA6A3D
:10AEA00012F8021B12F8015CBA6254F825003D4A00
:10AEB000904202D33C4A90421ED3BA6932B1786ABA
:10AEC0007B600EF0E7F87B6800288BD1BA6802BB84
:10AED00008F1280207F1300C08F10100944407F151
:10AEE000580208F1020852FA80F00CF8101C5FFAC0
:10AEF00088F800F8105C75E7BA693AB1786A7B6047
:10AF00000EF0C8F87B6800287FF46CAF1BF0010FCF
:10AF100009D006F1280207F13000711C161806F856
:10AF2000205CCEB25EE71BF0040F3FF45BAF08F18C
:10AF3000280207F1300008F1010102EB000808F8CF
:10AF4000105C5FFA81F84DE7002063E71BF80A30D8
:10AF500054F8239087F83730D7F88430FBB133F8B2
:10AF60001B8001213A6AFB6A07F1370098470028E5
:10AF700024DB0544B8F1000F06D14846FEF7BAFAC3
:10AF800000F101081FFA88F8414648463A6AFB6A10
:10AF90009847002812DB05440BF1010B6CE7D7F84A
:10AFA0008480DEE7D8E602004C1F03008BFC020021
:10AFB00004000001CCEA020045464BE6054649E69E
:10AFC000014B1860704700BF80C5002030B50025D8
:10AFD00087B0CDE903010446009503A9054805950E
:10AFE00000F010F9DDE904309842B8BF255407B0ED
:10AFF00030BD00BFE3900200032808B506D90EF06B
:10B00000CCFD092303604FF0FF3008BD2822044B1C
:10B0100002FB0033D3E8AF3F002BF0D00020F4E771
:10B02000E0D3002070B504460E461546FFF7E4FF56
:10B0300000280DDB28236343064AD1184968316094
:10B0400015B10C3313442B6028235C43105970BD99
:10B050000020FCE7D8D3002070B500254FF0FF3367
:10B060004FF0FF3217480BF0F7FA174BD3E8AF2F2A
:10B070007AB10135042D03F12803F7D10EF08DFDCF
:10B0800017234FF0FF3503600E480BF05DFB284699
:10B0900070BD28246C43D3E8EF0F0130C3E8E10F03
:10B0A0000029F8D1094E331932515A6004F10C00CD
:10B0B000304412F013FC04F12000304412F00FFD74
:10B0C000E2E700BFD0C80020E0D30020D8D30020A2
:10B0D00010B40446104628225443084B1A1919513B
:10B0E000506040B1C26832B10C34234440F20512C2
:10B0F00010BC0EF02DB810BC704700BFD8D3002094
:10B100002823434330B50D4908330B44D3E8AF2F10
:10B1100092B1541ED3E8EF5F954204D1C3E8EC4FDF
:10B12000BCF1000FF6D1F1D1012A05D128235843F3
:10B1300000230A180B50536030BD00BFD8D3002045
:10B14000F0B5024601680A270020074E0B461C781E
:10B150000131355D6D0701D41360F0BD07FB00437D
:10B16000A3F13000F2E700BFD91D03002DE9F84F2D
:10B1700015469A46D378224A6F2B12F803B08046C0
:10B180000F460BF0030B29D024D8582B0CBF1026E8
:10B190000A26DDF828903246002340463946FDF75E
:10B1A0005BFF092AD4B21ED83034B045E4B277F13F
:10B1B000000709F8014D01D3D14511D82B789B0622
:10B1C00005D5082E15D1AB7843F00803AB7048467F
:10B1D000BDE8F88F03F0F703702BD7E70826D8E710
:10B1E00080460F46D7E7BBF1010F0CBF3734573409
:10B1F000DBE7102EEBD1AB7843F01003E6E700BF9E
:10B20000D91D03002DE9F04F8A4616461C4600253D
:10B2100097B00390307808B928464AE3731C252874
:10B22000049307D05146039B98470028C0F24183FE
:10B230000135F0E11822002110A812F0D7FF737831
:10B24000252B00F0A380002398469E469C46184676
:10B25000711C0F4611F8012B2B2A00F0C68000F25A
:10B26000BD80202A00F0C480232A00F0C4802BB1C6
:10B270009DF8483043F040038DF84830B8F1000F96
:10B2800005D09DF8483043F020038DF84830BEF1DA
:10B29000000F05D09DF8483043F010038DF848307A
:10B2A000BCF1000F05D09DF8483043F008038DF83D
:10B2B000483028B19DF8483043F004038DF84830F9
:10B2C0009DF8483003F04401442903D16FF38613FD
:10B2D0008DF848309DF848302A2A43F080030997BA
:10B2E0008DF8483040F08C809DF8493043F00103E0
:10B2F0008DF849307B1C1A782E2A0CBF01210021C1
:10B300009DF8492061F341028DF849200CD15A1C67
:10B3100009925A782A2A40F083809DF84920023306
:10B3200042F004028DF849201A786C2A00F0A480BB
:10B3300000F28680682A00F08C806A2A00F0A580DE
:10B340004C2A00F0AA801A4612F8013B782B04928E
:10B350008DF84B309DF8492000F217816D2B00F2DB
:10B36000A980692B00F21181572B00F2BE80412B7E
:10B3700003D0453B022B00F2088104229DF84A309D
:10B3800062F302038DF84A300123CAE0B21C049232
:10B390008DF84B309DF84930D90740F1FD8054F8C5
:10B3A000048BB8F1000F07DA9DF84820C8F10008B7
:10B3B00042F004028DF848205A0740F1F68054F814
:10B3C00004BBBBF1000F80F2F5809DF849306FF3AC
:10B3D00041038DF849304FF0FF3BEBE02D2A0DD0B3
:10B3E000302A7FF444AF012333E74FF0010C30E7FC
:10B3F0004FF0010E2DE74FF001082AE7012028E762
:10B4000009A8FFF79DFE099BBB423FF474AF9DF86E
:10B4100048201390C00F60F341028DF848206AE77E
:10B4200009A8FFF78DFE9DF848301490C3F3400241
:10B4300042EAD07262F341038DF84830099B73E70A
:10B44000742A26D07A2A7FF47EAF06219DF84920FF
:10B450000CE05A78682A9DF8492006D1012161F351
:10B46000C6028DF8492002336DE7022161F3C6025E
:10B470008DF84920013366E75A786C2A9DF84920F7
:10B4800001D10421EBE70321F0E705219DF84920D4
:10B49000ECE707219DF84920E8E7BDF8482022F4B1
:10B4A000F04222F0020242F4804242F00202ADF881
:10B4B0004820DFE76E3BD9B201238B4040F2824146
:10B4C0000B4238D113F0240F52D1DF075DD5032191
:10B4D0009DF84A3061F302038DF84A3002F0780398
:10B4E000A3F14000434243411BE00120A3F1580176
:10B4F000C9B200FA01F111F4624F7FF43EAF40F699
:10B50000010739421DD111F4043F3ED09DF84A3065
:10B5100060F3020302F07802402A8DF84A3034D0FA
:10B5200000239DF84820C2F340010B4363F341021E
:10B530008DF848202EE702219DF84A3061F302037E
:10B54000E8E702209DF84A1002F0780260F3020159
:10B55000402A8DF84A1002BF9DF8481041F00101C1
:10B560008DF84810632BDBD1131E18BF0123D8E7D9
:10B5700003219DF84A3012F0780F61F302038DF831
:10B580004A3014BF01230023CBE79DF8483043F035
:10B5900001038DF84830C3E79DF94820002AACBF6D
:10B5A0004FF0FF38DDF84C8006E79F077FF513AFBB
:10B5B000DDF850B00023CDE913339DF84A309DF8F3
:10B5C000491003F00703012BC1F3C30133D1CB1E94
:10B5D000042B04D8DFE803F021464621210023682C
:10B5E00001294FEAE372CDE910321CD19DF94030B8
:10B5F000DA17CDE9103204349DF8483013F0030710
:10B6000050D032465146049B03980DF0B0FD0028FF
:10B61000C0F24F810544049EFCE554F8043BDA1760
:10B62000CDE91032E8E70229E5D11AB243F3C0337D
:10B63000CDE91023DFE7022B24D1CB1E042B04D845
:10B64000DFE803F018101018180001294FF000026D
:10B6500054F8043B14D00229CDE91032CCD19BB26E
:10B660001093C9E7073424F00704F4E80223CDE976
:10B670001023C1E754F8043B109300231193BBE758
:10B68000DBB2CDE7042B08D1073424F00704D4E95A
:10B6900000230834CDE91023AEE7032BACD154F8D6
:10B6A000043BDDE79DF84B007828B4D862281DD80C
:10B6B00025283FF4B7AD5828ADD1DDE910010DF1D3
:10B6C0003E03009312AA0AABFFF750FDBBF1000F37
:10B6D000814680F29880B9F1000F9CD00DF13E06B2
:10B6E000A6EB0903002F50D001334EE06338152834
:10B6F00091D801A252F820F079B70100DDB701001E
:10B7000017B6010017B6010017B6010017B6010001
:10B71000DDB7010017B6010017B6010017B601002A
:10B7200017B6010067B8010001B8010029B801008F
:10B7300017B6010017B6010051B7010017B6010096
:10B7400001B8010017B6010017B6010001B80100E9
:10B75000BBF1000FDDF840900ADB5946484612F075
:10B7600089FDB9F1000F3FF456AF09EB000676E012
:10B770004846FDF7BFFEF8E7109B00278DF82830FC
:10B7800001230DF129060DF128099DF84A1011F049
:10B790001002069200F081800233139A134405923E
:10B7A0004A0644BF14995B18B8F1000F40F38E802D
:10B7B000A8EB03089DF848305807C3F3800B00F14D
:10B7C0008580590678D53FB151463846039B984746
:10B7D00000286EDB5F46013530236EE01E075ABF3E
:10B7E000C3F300135F012B27DDE91023002BBFF605
:10B7F00064AF524263EB43032D27CDE910235CE78E
:10B8000000275AE700279DF848100DF13E03A3EBEF
:10B8100009036FF386119B458DF848107FF65BAFE7
:10B82000ABEB0303139356E7109880B30DF13E067C
:10B830000AAB0021009612AAFFF798FCBDF84A3027
:10B84000BBF1000F03F0EF0343F4F04343F01003A8
:10B850008146ADF84A30D5DA00283FF4DCAE002747
:10B86000A6EB090391E7109B07293FF6D4AEDFE86A
:10B8700001F00C04060C08080C0C1D70CBE61D80B2
:10B88000C9E6EA17C3E90052C5E61D60C3E6314EBA
:10B8900007460523A6F1050977E7080748BF0133E6
:10B8A0007BE7184607935146039B98470028079B60
:10B8B00004DA17B0BDE8F08F2023C34659460029AB
:10B8C0000BF1FF3BEDDC4544D8466D1A37B15146CC
:10B8D0003846039B98470028EBDB01359DF84A303A
:10B8E000DA0601D41B0706D551463020039B984742
:10B8F0000028DEDB0135069B3BB151469DF84B002D
:10B90000039B98470028D4DB0135059F2F4406E0B0
:10B9100051463020039B98470028CADB01357B1B2A
:10B92000002BF5DC33464A46514603980DF01FFCC8
:10B930000028BEDB0544A844A8EB0503002B7FF7D5
:10B940006AAE51462020039B98470028B1DB0135A1
:10B95000F2E700BF44FD02002DE9F047058B0446E5
:10B960002807904611D4022905F0070540F0CC8045
:10B9700020460DF067FE78B10138218B042811D8DC
:10B98000DFE800F0C2106D85950001290CBF45F07D
:10B99000100545F02005258388F31188BFF36F8FCC
:10B9A000BDE8F08701F0070AAA4500F0A58000274E
:10B9B000B9463E46A368002B00F0BC8041F0080168
:10B9C000218388F31188BFF36F8FA168002900F0ED
:10B9D000BA800D68002900F0B680334652462046F2
:10B9E000D1F80480C047002D76D02B6829461D462B
:10B9F000F0E701F007035A1F012A1BD8002221F0AB
:10BA00000701062B276889B2C4E9002209D13B4609
:10BA100003E0628B013262831B68002BF9D141F095
:10BA20000201204621830DF00DFE00287AD041F05E
:10BA3000200176E0042B0AD121F0070189B22046CB
:10BA400021830DF0FFFD10B141F020012183218BF6
:10BA500001F0070AAA454FD00027B946AAE7236993
:10BA600021F0070141F00601062DD3F80090218353
:10BA70002DD1B9F1000F3FD041F00801218388F3A7
:10BA80001188BFF36F8F20463949C84729E021F05C
:10BA90000701236941F0040189B2042DD3F8049011
:10BAA0002183E6D000274FF0040A3E4682E721F0CA
:10BAB0000701236941F0050189B2052DD3F80890EB
:10BAC0002183D6D000274FF0050A3E4672E70027B3
:10BAD0004FF0060A3E466DE72B4687E7B9F1000FA7
:10BAE000D1D1EFF31188202383F31288BFF36F8F36
:10BAF000238B23F008032383258BEA062ED525F01C
:10BB00001003238305F007056669218B002EBFF61D
:10BB100070AF00232768C4E9003321F0070141F02A
:10BB200001012183218B4FF0000901F0070AAA458A
:10BB30007FF440AF002F9CD041F00801218388F3AF
:10BB40001188BFF36F8F002FC8D03D683946334648
:10BB5000524620460DF0A2FD2F46F4E7AB067FF5D6
:10BB60001BAF25F02003238305F0070500E700BF86
:10BB7000C99602002DE9F047044607464FF0010937
:10BB8000DFF8508014B93846BDE8F08794FAA4F580
:10BB9000B5FA85F509FA05F32E0108EB05156FEAEC
:10BBA000030A24EA03042B7B002BEBD058F8063061
:10BBB0001B694BB94644736804222846196807EA92
:10BBC0000A0700F04DFADDE7284698470028D9D14A
:10BBD000F0E700BF64EB020030B5002289B00F49E6
:10BBE0000F4812F02BF9002200230024CDE9062390
:10BBF0000E230C4DCDE903344FF440722846CDE9B5
:10BC00000144094B094900940BF066F8084928469D
:10BC100011F06FFF204609B030BD00BF35BC0100F8
:10BC2000A8CF002018CB00200DBF010068E4002041
:10BC300045FD020001480AF0F5BD00BF60C90020C3
:10BC40002DE9F04780461F480F460DF0F6FD0646E9
:10BC5000002830D000252846BDE8F087237B6BB153
:10BC60002368DB680BB12046984723681B69D3B96A
:10BC7000636804222046196800F0F2F90136103496
:10BC80004C45EBD3B8F1000FE5D0002DE2D02846AB
:10BC9000FFF770FF0546002FF7D000214FF4A47086
:10BCA0000BF0CAFAF1E7204698470028E0D00AFADC
:10BCB00006F31D43E2E705464FF0010A024CDFF8A8
:10BCC0000C90DDE788D4002064EB020074EB0200E6
:10BCD000014B53F8200070471CEC020008B50346E6
:10BCE00008462BB1044A136000F05EFC002008BD3A
:10BCF0006FF01500FBE700BF84C5002010B5044CB1
:10BD0000237813B903480AF08DFD0123237010BD79
:10BD1000F7DE002060C9002010B5044606480DF08B
:10BD20008CFD3CB1054BD3E8EF1F0139C3E8E21F9E
:10BD3000002AF8D110BD00BF80D4002084D4002098
:10BD400000200146034BD3E8EF0FC3E8E21F002AAF
:10BD5000F9D1704780D4002070B5FFF7F1FF054698
:10BD6000074C084EB44200D370BD63685B792BB1B9
:10BD700023685B6813B12946204698471034F1E7E1
:10BD800064EB020074EB020010B5044C0449204639
:10BD90000DF000FB034B1C6010BD00BF3CC8002031
:10BDA00008EC020078D4002008B50023074A4FF4BD
:10BDB00000411370064A07481360074A1360FFF7F3
:10BDC0008DFFBDE80840FFF7DFBF00BFF8DE0020B1
:10BDD00080D400203798020084D40020014600223D
:10BDE000002301480DF0F7BA3CC8002001480DF0CF
:10BDF0008DBB00BF3CC80020024B014618680DF007
:10BE0000D9BB00BF78D4002001480DF00EBC00BFA4
:10BE10003CC8002070B5264B1878002847D0FFF7A3
:10BE2000E5FF054670B1234BD3E8EF1F0139C3E8A6
:10BE3000E21F002AF8D1204C204EB4422DD32846D0
:10BE4000FFF7DAFF1E4B1F4C1B68002B19DD11F0AA
:10BE5000AEFF4FF47A72A0FB020302FB0131C30B69
:10BE600043EA4143D4E900209B1A40F2E9324FEA09
:10BE7000D13161EB0001934271F1000101D3FFF771
:10BE80006BFFD4E9003213F57A7342F10002C4E982
:10BE90000032BDE87040FFF7B7BF63685B7923B13C
:10BEA0002368294620461B6898471034C5E770BDB3
:10BEB000F7DE002084D4002064EB020074EB020063
:10BEC00080D40020A0CF002070B50D4D297861B935
:10BED0000120FFF7B5FE0B4C0B4EB44206D3FFF723
:10BEE00099FF0028FBD101232B7070BD63685B793B
:10BEF0001BB1236820469B6898471034EDE700BFCC
:10BF0000F8DE002064EB020074EB020000212DE952
:10BF1000F0470846FFF794FE044648B340F26768CE
:10BF20004FF000090BF0A6F91A4B186030B11A4B0C
:10BF30001B68092B02DD19480AF074FC0025184F14
:10BF4000DFF858A044B12046FFF714FE044618B9A4
:10BF50004FF0FF384FF0FF39FFF75CFF064628B976
:10BF6000B5B942464B4650460AF080FC3546E9E7F3
:10BF70004FF0FF384FF0FF39D4E72B689B691BB1B6
:10BF800000222846114698471035BD42F5D3E8E710
:10BF9000044DFAE77CD4002084D4002060C900203E
:10BFA00074EB020064EB020013B518480DF045FC79
:10BFB000174B1B7873B1EFF31184202383F312889E
:10BFC000BFF36F8FFFF726FF84F31188BFF36F8FE6
:10BFD00002B010BD0F4B1B68002BF9D050B90022E6
:10BFE00000230D48CDE900234FF4004200230BF05D
:10BFF000A9FBEDE70928EBD1074811F02BFF074813
:10C0000002B0BDE810400AF00DBC00BF84D400208F
:10C01000F8DE00207CD40020A8CF002060C90020DA
:10C0200010B5064B04461B6898472146A06004489B
:10C030000DF04DFABDE81040FFF7B6BF84C50020F3
:10C040003CC80020044A054B9B1AB1EBD30F34BF08
:10C0500052F8310000207047C4EA020064EB02008D
:10C06000084B10B4C31A44681B1101332371436891
:10C070009A7101224368196043685A7110BCFFF736
:10C080003DBE00BF64EB02002DE9F04F8FB0C1F35D
:10C090004A2804AF0D469146B8607B600C0DB8F19C
:10C0A000000F63D000264FF0040B4FF00A0A07F18F
:10C0B0001403C7F80C80C7E907667E620193CDF8C8
:10C0C00008B0CDF800A007F11C0332464846F968D5
:10C0D000FEF796FDB0F5006F03461CD36C468AB0A0
:10C0E000D9F8041004AB26481A46C3E9050140F20A
:10C0F000FF71D9614FF400711984224B42F8103F4F
:10C100004FF4125133462048FFF7BEFFA5462C37A7
:10C11000BD46BDE8F08FC0F30A0804F117001844CB
:10C1200020F0070080083B60FFF758FE68F35325B6
:10C13000044690B13B6800F11001C7E9083607F1E9
:10C140001403F961CDE900A3CDF808B048460F4AC1
:10C15000F96807F11C03FEF753FD68F353252A46DF
:10C1600020467B68B9680DF09AFBD0E704F1170010
:10C1700020F007008008FFF731FE0446EDE700BF1E
:10C180005AFD020004000001FCEA0200739802005C
:10C190002DE9F04F87B00446DDE9105ADDE9126958
:10C1A0000F4693469846A6B31021334652460020C8
:10C1B000CDF80090CDF81490FEF750FB014605F144
:10C1C00017000844144B04F007040BF0070BE400BD
:10C1D00020F0070003EA412344EA8B1480081C4343
:10C1E0000391FFF7FBFD44EA0554054640B13EB11B
:10C1F000334652460399CDF800901030FEF72EFBDF
:10C20000434622463946284607B0BDE8F04F0DF0B8
:10C2100046BB3146D3E700BF00FE0F00406820B1A7
:10C22000034BC01A40F3CF0070474FF0FF30704708
:10C23000C4EA02000EB403B503AB53F8042B014665
:10C24000044801930DF0A8FB02B05DF804EB03B0C5
:10C25000704700BFC1990200CA0605D48B064CBFC7
:10C2600002490349FFF7E6BF704700BFB919030051
:10C27000B81903002DE9F04F89B09A46149B9DF838
:10C280004CB00693159B04460593169B0D469046AD
:10C29000179E0493BBF1000F00F09D8006F480739D
:10C2A00007930DF0E4FA06F00209024600283ED09A
:10C2B00020469249FFF7BEFF0746B9F1000F08D0AC
:10C2C00016F0440F35D12A4620468D49FFF7B2FFBC
:10C2D000074406F0010353B18A4B204653F82B2044
:10C2E000894B8A49002A08BF1A46FFF7A3FF06F4C4
:10C2F0008073002B49D006F00803002B63D1B8F1FE
:10C30000000F66D0424620468149FFF793FF05465D
:10C31000069B3D44002B6DD1049B002B73D1F3078A
:10C3200000F1E58031462046FFF796FFD9E0074649
:10C33000C3E7784B18680028CAD0774B4FF47A7956
:10C340001B684FF46161B5FBF3F5B5FBF0F300FB3F
:10C35000135509FB05F5B3FBF1F2B5FBF0FE4FF009
:10C360003C0C01FB123100FB1E55B1FBFCF309FB39
:10C3700005F5B5FBF0F50CFB131120460091CDE956
:10C3800001E56649FFF756FFA2E706F00803EBB1A7
:10C39000634B204653F82B206249FFF74BFF0546BD
:10C3A000B8F1000F05D0424620465949FFF742FF39
:10C3B0000544BAF1000FABD0524620465A49FFF768
:10C3C00039FF0544A4E74FF0000AE1E706F008054D
:10C3D000E6E745469CE7BAF1010F069B06D1002B24
:10C3E00065D1049B002B7CD000250CE0002BF8D0FD
:10C3F0004E485DE04E48069B22464E490CF019FE21
:10C40000049B002B69D0DFF83081DFF83091049F66
:10C410003146102F204628BF10274FF0000AFFF7A3
:10C420001BFF554546DC059B494620461A78FFF719
:10C4300001FF4FF0010A1AF0070F03D141462046D1
:10C44000FFF7F8FE57453CD9059B4946204613F8AF
:10C450000A20FFF7EFFE0AF1010ABAF1100FEAD144
:10C460004FF0000A20463649FFF7E4FE5246059B8E
:10C4700020469A5C334B995C11F0970F08BF2E222F
:10C480003149FFF7D7FE0AF1010ABAF1100F1DD0AA
:10C490001AF0070F03D141462046FFF7CBFE574560
:10C4A0005246E4D841462046FFF7C4FEEBE7204859
:10C4B0005D46A0E741462046FFF7BCFE0AF1010AAF
:10C4C000AFE720462149FFF7B5FEC4E7059B3B4493
:10C4D0000593049BDB1B049399D1BBF1000F7FF400
:10C4E0001EAF204609B0BDE8F04F0DF05CBA204603
:10C4F000054A0649FFF79EFE14E700BF9EFD0200B5
:10C50000A2FD02002CEC020099FD0200580B030072
:10C51000C7FD020090D400208CD40020ABFD0200A7
:10C5200040EC0200CBFD0200D1FD0200EF990200B9
:10C53000C199020099990200DEFD0200D6FD0200B9
:10C54000E0FD0200D91D0300B30E0300DCFD020074
:10C5500042F20F7373B58B4228BF0B460568044641
:10C56000052168460D4A0CF0DCFD06466368284646
:10C570000B225B680A490DF001FA6368324669468E
:10C5800028465B680DF0FAF963681B2228465B6851
:10C5900004490DF0F3F902B070BD00BF40F802008D
:10C5A000FEFD0200E2FD020000210123064A904246
:10C5B00006D8064A01B901231360054B186070477D
:10C5C000012140085B00F2E740420F008CD40020BC
:10C5D00090D40020F8B50D460446064F4618B442E4
:10C5E00001D12846F8BD14F8011BBB6801485B68FF
:10C5F0009847F4E7F8E70200014B0360002070471A
:10C6000088EC020008B504480CF07EFDBDE8084047
:10C6100002480CF079BD00BF44FE020079FE020022
:10C620002DE9F04706460C4600AF002936D0D1E987
:10C630000012E9468AB06D46A3684FF0050AA84685
:10C640001F48C5E90723C5E9050148F810AF0023D5
:10C6500042464FF421511B48FFF716FDD4E903125F
:10C66000CD466369AD461848C5E90723C5E905010C
:10C67000C5F810A0002342464FF421511148FFF79E
:10C6800003FDCD46E3690121104A0E480DF060F923
:10C69000A36901210E4A0B480DF05AF9012E07D16A
:10C6A000EFF305830B4A31460648103B0DF050F975
:10C6B0002146304609F022FEBD46BDE8F08700BFA6
:10C6C000A7FE020044EB0200D6FE020005FF0200B6
:10C6D00014FF020042FF020030BFFFF7FDBF00BFA2
:10C6E000074A936893F90E10002907DB52699342B9
:10C6F0001FBF044A536843F080535360704700BF24
:10C70000F4DC002000ED00E070B52A4C06460D4632
:10C7100029482A490DF0E1F9A36ADB0647D52648E6
:10C7200027490DF0DAF91120A36A1C0704D5224825
:10C7300024490DF0D2F912201E4CA36A990712D594
:10C7400021491D480DF0C9F9636BA26A120609D58B
:10C7500001211E4A18480DF0FBF81EB1A36A23F010
:10C760008003A3621320134CA36ADE0704D512488A
:10C7700017490DF0B2F91420A36A9C0604D50E489F
:10C7800014490DF0AAF915200A4B9A6AD10658BF30
:10C790009A6A9A6A920642BF5A6A22F400525A6210
:10C7A0009A6A42F0FF029A6200232B7070BD10203B
:10C7B000BAE700BF00ED00E044EB020055FF0200C5
:10C7C0006BFF02009EFF0200B1FF0200C9FF0200E2
:10C7D000DFFF0200FEFF020010B5244C244925486B
:10C7E0000DF07BF9A36A99013ED5224822490DF04C
:10C7F00074F91E20A36ADA0104D51E481F490DF002
:10C800006CF91F20194CA36ADB0204D519481C4996
:10C810000DF063F90220A36A1C0304D515481949D9
:10C820000DF05BF92120114CA36A590304D511487E
:10C8300015490DF052F92220A36A9A0304D50D4838
:10C8400012490DF04AF92320084CA36ADB0304D5F2
:10C8500008480F490DF041F92420A36A6FEA034309
:10C860006FEA1343A36210BD1D20C3E700ED00E093
:10C870002D00030044EB02004500030058000300B4
:10C88000720003009C000300BA000300DF000300F5
:10C89000F900030070B5294C06460D462848294981
:10C8A0000DF01BF9A36AD9043CD5254826490DF0A3
:10C8B00014F91720A36A1A0504D5214823490DF05D
:10C8C0000CF918201D4CA36A9B0512D51C48204961
:10C8D0000DF003F9A36BA26A100409D501211D4ACA
:10C8E00017480DF035F81EB1A36A23F40043A36284
:10C8F0001920124CA36A590504D5114816490DF0A8
:10C90000ECF81A20A36ADA050ED50D4813490DF08C
:10C91000E4F81B20094A936A43F47F43936200239F
:10C920002B7070BD1620C5E7A36A9B04F2D504489E
:10C930000B490DF0D2F81C20ECE700BF00ED00E041
:10C9400044EB0200240103003A0103009EFF0200B1
:10C950004B0103006401030079010300940103000B
:10C96000FEFF02002DE9F0478AB0694B0446D3F878
:10C9700004A089461646002500AFCAF3080885F3CF
:10C980001188BFF36F8F02F07F43B3F17F4F1ED149
:10C99000D3071CD4500603D4110708D4012508E09E
:10C9A0005C495D480DF099F816F0040600D04C463D
:10C9B00000250023FB71A8F10303092B00F28680F8
:10C9C000DFE803F0077C7F798484848484822C46AA
:10C9D000EFE7524950480DF080F800234C4EFB71B0
:10C9E000F36A9A0705D54E494B480DF076F80023B7
:10C9F00029E0F36A002B01DA4A49F5E7F36A5B00A4
:10CA0000F5D5494944480DF068F87369A26943F4C3
:10CA100080737361BFF34F8FBFF36F8F736932F809
:10CA2000022C23F480737361BFF34F8FBFF36F8FBA
:10CA30004DF602739A4228D1236801213B4A3648B9
:10CA40000CF086FF2368FA79DAB907F1080604F1D9
:10CA5000200C324620686168083403C264451646DB
:10CA6000F7D17A6A002D4ED0C2F3080121B96FEADE
:10CA700052226FEA42227A62184607F10801FFF754
:10CA8000CFFD2837BD46BDE8F087B36ADBB22BB1D6
:10CA90000120F91DFFF738FE0346D4E7B36A13F40B
:10CAA0007F4F04D00120F91DFFF7F4FEF4E7B36ACD
:10CAB000B3F5803F9BD3FFF78FFEEDE70020F91D14
:10CAC000E8E70020F91DEFE719498DE7194A6E469E
:10CAD0001AF4F87F8AB0184B18BF13466A461749F4
:10CAE000C2E90513A8F11003D3614FF40073138456
:10CAF000134B42F8103F00234FF411510648FFF743
:10CB0000C3FAB54673E722F4FF7222F00102B2E7DE
:10CB100000ED00E0DA01030044EB0200FD01030038
:10CB20001402030035020300430203006202030003
:10CB30007E020300C1010300AC010300A202030056
:10CB400004000001044B5A6942F010025A615A690C
:10CB500042F480625A61704700ED00E0EFF3088014
:10CB6000EFF3098101B57246FFF7FCFE01BD00BF7E
:10CB7000002080F31488BFF36F8F002080F30A88B1
:10CB800080F30B880FF079FB00200E490860BFF39B
:10CB90004F8F0D4880F3088800F02CF8202080F398
:10CBA00011880A484FF40061401880F30988EFF3B8
:10CBB00014800221084380F31488BFF36F8F00F0C4
:10CBC00009F9000094ED00E0A805012068EC0020C0
:10CBD000002318460649D1F89020C2F30722934259
:10CBE00000DB7047C1F89830C1F8A0000133F6E7C8
:10CBF00000ED00E010B572B6002484F31388FFF74F
:10CC0000E7FF23464FF0FF300C4A03F120010133C8
:10CC1000102B42F82100F8D100234FF0FF30074AD3
:10CC200003F160010133102B42F82100F8D162B604
:10CC3000BFF34F8FBFF36F8F10BD00BF00E100E067
:10CC4000084B9B6883420BD1EFF3058343B1064B3E
:10CC50005A6842F080525A605A6A22F400425A627C
:10CC600011F048B8F4DC002000ED00E06FF00A019C
:10CC7000084A9368D967084998674B6843F080531E
:10CC80004B60002383F31188BFF36F8F9368D86FD5
:10CC9000704700BFF4DC002000ED00E00E4A93680E
:10CCA00083F88100EFF31183202383F31288BFF30D
:10CCB0006F8F4FF00061536920F0FF009360074AC7
:10CCC0005160002193F8812010439A6F996782F395
:10CCD0001188BFF36F8F7047F4DC002000ED00E097
:10CCE00010498A6882F881E04FF030001044EFF379
:10CCF000098C80E8F01F74467046FFF7CFFFA64608
:10CD000008498A68864602F1300090E8F01F8CF3EB
:10CD1000098802F1000004B50CF0E9FEBDE804400A
:10CD200070470000F4DC00201EF0040F0CBFEFF38E
:10CD30000880EFF30980816911F8021C0229FFD0F5
:10CD400001B50CF0BFFE01BD40B2002807DB012396
:10CD50004109034A00F01F00834042F82130704728
:10CD600000E100E040B200280CDB01220649430943
:10CD700000F01F008240203341F82320BFF34F8F83
:10CD8000BFF36F8F704700BF00E100E0054B420921
:10CD900053F82220012300F01F0003FA00F0104096
:10CDA000704700BF00E100E040B2002801F101013E
:10CDB000ACBF00F16040064B4FEA4111C9B2ABBFB6
:10CDC00000F5614000F00F0080F80013195470471F
:10CDD00014ED00E00B4A08B50B4B22F07F029A607D
:10CDE000BFF34F8FBFF36F8FD3F8882022F4700208
:10CDF000C3F8882009F06CFB0AF0DAFA00F04AF870
:10CE000009F0A6FB0080010000ED00E042F8203CA4
:10CE1000009B0D4942F81C3C019B21F0010142F8A6
:10CE2000183C029B42F8081C42F8143C4FF08073F7
:10CE300042F8043C002383674FF43C43203A0265E8
:10CE4000C0F88030704700BF3D9102000B4B0E468A
:10CE500098601546836E83F30B882C4686F3098809
:10CE60004FF00000064B984720464FF000014FF06E
:10CE700000024FF00003034C204700BFF4DC002009
:10CE8000F79A02003D9102001022014B1A6170478F
:10CE900000ED00E0002320210348C2180133412B9C
:10CEA00082F80013F9D1704700E100E008B5EFF314
:10CEB0000583064A103B02EBC30152F83300496870
:10CEC0008847BDE80840FFF70BBC00BFACE8020094
:10CED0001FB5094C094A23460121094800F012F9FF
:10CEE00000230393074B0121E41A01A80193029444
:10CEF00000F012F904B010BD0000042080C500202D
:10CF000088EC020030CA002010B50C7A0B6804F0DF
:10CF10001F0223F01F031A43CB68640923F01F0389
:10CF2000054943EA440343F00103C1F89800C1F8FE
:10CF30009C20C1F8A03010BD00ED00E010B50A4BF8
:10CF4000D3F89030C3F30723013B984208D901215D
:10CF50000346064A06480CF0FBFC6FF0150010BDB6
:10CF6000FFF7D2FFFBE700BF00ED00E0B9020300CE
:10CF70001CEB02002DE9F04F8946144606464FF09F
:10CF80000008514D85B0C84527DAD6F804A0BAF19B
:10CF9000000F44D0BAF11F0F17D91AF01F0F14D188
:10CFA000D6F800B01BF01F0F0FD158460CF0C6FD8D
:10CFB00007460AEB0B0001380CF0C0FD874210D089
:10CFC0006FF01507414A3B4601E04346404A0121C4
:10CFD00040480CF0BDFC6FF01504204605B0BDE8DC
:10CFE000F08F17F1160FEDD0BC42EBDDC5F898704D
:10CFF000D5F89C10C5F89870D5F8A03021F01F0125
:10D0000043F01F0BD6E900321A44994202F1FF3A6D
:10D010001DD1D34507D13146F8B20CF098FD08F187
:10D0200001080C36AFE73146C5F89870D5F89C304A
:10D0300022F01F0203F01F031343C5F89C30E0B237
:10D040000CF085FD10F1160FC5D0441CE7E7C5F8BC
:10D050009870D5F8A020013B23F01F0302F01F02B7
:10D060001343D3453146E0B2C5F8A030E8D00CF008
:10D070006EFD10F1160FAED0C5F89870D5F89C2053
:10D080009DF808300BF1FF3B62F304038DF8083084
:10D09000D5F8A0309DF808205B0863F347128DF89F
:10D0A0000820D6E900321344009323F01F035B44A9
:10D0B000A3EB0A03013023F01F036946C0B20393B8
:10D0C000FFF73CFFBEE700BF00ED00E002030300F6
:10D0D000DF0203001CEB02000522044BC3F894207E
:10D0E000BFF34F8FBFF36F8F704700BF00ED00E0BD
:10D0F000BFF35F8F0022024BC3F89420704700BF3C
:10D1000000ED00E010B5034C2278FFF733FF2070EC
:10D1100010BD00BFFADE00202DE9F74F294D8A46E9
:10D1200006464FF00008AB46274FD0451BDAD6F82D
:10D130000490B9F1000F3FD03168084601910CF01E
:10D14000FDFC0199044609EB010001380CF0F6FCE6
:10D1500084424FF014021D4B08D002FB08F36FF01D
:10D1600015024BF8032003B0BDE8F08F14F1160F41
:10D170002C60F8D01978A142F5DD02FB08B0C7F8A1
:10D180009840C7F89840D7F89C4000F10801007B10
:10D1900064F304000871D7F8A0000C79400860F32C
:10D1A00047140C71D7F89C1021F01F016960D7F863
:10D1B000A01021F01F01296108F1010814350C3677
:10D1C000B3E700BFC0D4002000ED00E0FADE00208D
:10D1D000F0B54149414CD1F890302568C3F307239D
:10D1E0009D4287B075D80020FFF782FF3C4BC1F805
:10D1F000C030854216D13B4C01A82570FFF7FCF9E1
:10D2000000250646384FAE4213D10020237832491C
:10D21000D1F89020C2F30722934254DBFFF75CFF62
:10D2200000202FE0616801EB0011FFF76DFE013077
:10D23000DFE70199280101EB0513DA683A40B2F5FE
:10D24000001F21D0B2F5800F2BD0B2F5801F38D14E
:10D250005A689B680958013B22F01F0003440120D3
:10D26000844623F01F0340EA4C10CDE902218DF8DB
:10D27000100002A920780593FFF760FE00281DDA50
:10D280006FF0150007B0F0BD5A689B680958013B64
:10D2900022F01F0003444FF0020C012023F01F0373
:10D2A000E1E75A689B680958013B22F01F000344DC
:10D2B0004FF0000C062023F01F03D4E7237801333E
:10D2C000237001359FE7C1F89830C1F8A000013301
:10D2D0009EE74FF0FF30D5E700ED00E094EC020050
:10D2E000AAFF4400FADE00200000F0FF014B1860A6
:10D2F000704700BF90C5002010B5074C2368C218C6
:10D300000648C0F1005101F580218A4236BF2260F3
:10D310004FF0FF30C01810BDD4D4002028120120D7
:10D320000122024B0020C3F84025704700900340C3
:10D3300020B1034B800143F001031847704700BF41
:10D34000D0EB0200F7B506460D460D488AB2836859
:10D3500031461B689847002810DA00240CE02F1B88
:10D36000042F28BF04270EF0F9FA3A46019001A9CC
:10D37000301910F02EFF3C44A542F0D803B0F0BDA8
:10D38000E4E702002DE9F04105460E461746104C31
:10D39000DFF84080444507D30CF0FFFB6A230360AD
:10D3A0004FF0FF30BDE8F0812368AB4200D063B995
:10D3B0003A4631462846A368984730B13A46314646
:10D3C0002846E368BDE8F04118471034E2E700BFA3
:10D3D000B4EA0200C4EA02002DE9F04F4FF0000861
:10D3E00046469DB0CDE9060108A814461D4610F03A
:10D3F000E0FCDDE90823DDE9069BCDE904230DAB64
:10D400000A93CDF80C80BBF1000F22D1002E6ED014
:10D41000B5F1FF3F08BFB4F1FF3F17BF4FF47A7279
:10D420004FF0FF34A4FB024302FB05331CBFE40BA7
:10D4300044EA4344079B4FF4827200934146069BA3
:10D44000039801940CF0AFFB074638461DB0BDE8C9
:10D45000F08FD9F80000002829DB0CAA0BA9FDF7F2
:10D46000E1FD074618B34FF0FF324FF0FF330C9841
:10D470000CF0A8FB1CAB01930AAB00934FF4817234
:10D480004B4639460B980CF08EFB10F1780F824614
:10D4900012D10022002308A810F08BFCDDE908342B
:10D4A000CDE9043400240C980CF08EFB254609F1DC
:10D4B00008090BF1FF3BA6E71AF1120F0C980BD1EC
:10D4C000039B1BB10CF080FB0126F0E70B9BB846D9
:10D4D00003930CF079FBF7E70CF076FBBAF1000F41
:10D4E000E5DA0CF05AFBCAF10003036021E0DDE944
:10D4F000042308A810F081FCDDE9084522462B46EC
:10D50000DFF8C8800A990DAC091B891008FB01F1EE
:10D5100020460AF051F900F10B030B2B054604D805
:10D520002B4F1F4117F0010706D00CF036FB6D4260
:10D5300005604FF0FF3788E7B9460A94DDE90645F4
:10D540008DB9B9F1000F80D0002F7FF47EAFDDE9F7
:10D55000042308A810F051FCDDE908452B462543BB
:10D560002246CFD171E72068E680002827DB0CAA8D
:10D570000BA9FDF757FD824618B92023E380013738
:10D580001DE04FF0FF324FF0FF330C980CF01AFB08
:10D590000AAB514640F2031200930B9823460CF05D
:10D5A00002FB82460C980CF00FFB1AF10B0F09D00E
:10D5B000BAF1000F95D1B4F90630002BDFD1083451
:10D5C000013DBDE74FF00109F9E700BFCDCCCCCC60
:10D5D0007EF7FFFF014B1860704700BFD8D40020D2
:10D5E00010B4034C24682468A44610BC604700BFF4
:10D5F000D8D40020014B1B685B681847D8D40020A2
:10D600002DE9F0410D460646E8B1E1B10846FBF7C9
:10D6100071FF08281AD8104FDFF84080441C474596
:10D6200007D322462946301D10F0D3FD0020BDE867
:10D63000F081B74205D022462946381D10F0B9FDC9
:10D6400038B13C37EBE76FF01500F0E76FF05A00A8
:10D65000EDE76FF07700EAE7C0C90020FCC90020C1
:10D66000F0B54FF0FF324FF0FF33274885B00CF094
:10D67000E1FB0025254C264EB44205D3224805B0D7
:10D68000BDE8F0400CF0F4BBC4E9015523682573F4
:10D690001B689F6897B13B6883B104F1100010F0DC
:10D6A0001DF904F1240010F019F93B682046984751
:10D6B00094F8383023F0030384F83830237903BB1F
:10D6C0002046CDE901338DF80C300CF04CFC40B114
:10D6D000104A01A81368591C116008210E4A0BF06A
:10D6E00020FD9DF8043043B90C4A01A81368591C69
:10D6F000116008210A4A0BF014FD204601A9FFF72A
:10D700007FFF3C34B8E700BF0CC90020C0C900202F
:10D71000FCC90020E0D400204F030300DCD400202B
:10D720005603030038B5074C074DAC4200D338BD53
:10D73000032120460CF087FB10B920460CF0E1FBDA
:10D740003C34F2E7C0C90020FCC900202DE9F04FAD
:10D75000002489B0022883460E46CDE90644029291
:10D760005FD10B6804913BB94A6852B94FF6FF7319
:10D770004C89E11A4C424C4106A80146002213464E
:10D7800008E01C46F8E70D78013301350D70DDB275
:10D79000082D03D036F81350002DF4D00132082A9A
:10D7A00001F10101EBD14FF0FF374FF0010A0023E7
:10D7B00010F8012B524588BF5FB203F10103DBB2C1
:10D7C00088BF9246082BF3D199463A220023BAF13A
:10D7D000010F08BF4FF0FF37CDE900230022029868
:10D7E00000252B46B9F1040F5ED10199C95C0346AF
:10D7F00041BB302103F8021B0099417018460135E6
:10D80000EDB24D452B46EDDB029B98420BD0BBF1B0
:10D81000010F4FF0000340F09C8000F8013C02989B
:10D8200002E0012803D0002009B0BDE8F08F2E23CC
:10D830004FF004094FF0FF378246264601910093CE
:10D840000494CBE74FF0000C4FF00908CDF814C05A
:10D85000DFF804C1B1FBFCFE03910CFB1E11DDF8E7
:10D8600014E0C64503DCDDF80CE0E64509D3DDF83D
:10D870000CE0CDF81480BEFBFCFE0EF1300E03F878
:10D8800001EB4FF00A0E08F1FF38B8F1FF3FBCFB87
:10D89000FEFCDFD14FF0000119701B1A50FA83F023
:10D8A000009B00F8013BAAE774B1052D0CD906F1E5
:10D8B0000C0301933A2300F8013B2E234FF0040997
:10D8C0004FF0010B00938BE79F420DD102B915B9C0
:10D8D0003A2300F8013B3A2300F8013B0AF1FF33F9
:10D8E0002B440022DDB28AE712B13A2300F8013B53
:10D8F000049B33F8152052BA12F47F4FC2F307236A
:10D900005FFA82F816D00F2BD9B20AD90023612210
:10D910000CF036FB0123612241460CF031FB012261
:10D920006DE7092B04D83031C9B200F8011BF1E7CB
:10D930005731F9E7B8F10F0FEDD8B8F1090F94BFDF
:10D9400008F1300808F157085FFA88F800F8018BF1
:10D95000E5E7037063E700BF00CA9A3B2DE9F04793
:10D960000F6890F860503C4B3C4A064690F85E00C9
:10D970000537042814BF104618460F600C460CF0FB
:10D98000E2FBC5F34005034638B9D4E900209042D4
:10D9900096F85E1004D16FF00B031846BDE8F087CF
:10D9A000501C20601170D4E900829045F3D008F13A
:10D9B0000102226088F800302146B6F85C000CF0C5
:10D9C000B0FB03460028E8D106F12C000CF0BBFBAD
:10D9D00003460028E1D1306C6D00E8B1214696F88D
:10D9E00060A090F808900CF0AEFB0AF0010A034624
:10D9F0000028D2D1736C21465BB318460CF0A3FB10
:10DA000003460028C9D145F004054FEAC90345EA99
:10DA10004A1503F018031D43B06B38B121460CF0D2
:10DA200092FB03460028B8D145F08005F06B38B171
:10DA300021460CF088FB03460028AED145F0400596
:10DA400088F8005022463946BDE8F04710200CF017
:10DA500095BB0CF066FBD3E7BCEC0200C4EC020003
:10DA6000D0E900239B1A012B81BF054B1B88138033
:10DA7000036883BF0233436000206FF00B007047E0
:10DA80005C030300D0E900239B1A012B81BF054BE7
:10DA90001B881380036883BF0233436000206FF04C
:10DAA0000B0070475E030300142290F824305343A8
:10DAB000014AD358184700BFCCEC020030B41425FB
:10DAC00090F82440024B05FB043330BC5B681847D8
:10DAD000CCEC020010B4142490F82420024B04FB78
:10DAE000023310BC9B681847CCEC020070B41426BB
:10DAF00090F82450034C06FB0544E468A44670BC2F
:10DB0000604700BFCCEC0200084B70B5C31A0D464D
:10DB100007499B1004465943402206480CF0E2FF97
:10DB20002B4601462046BDE870401847F8D4002037
:10DB3000B76DDBB6BCE70200402373B50B4C009316
:10DB4000041B0B460D460A49A41061430646094AC8
:10DB500009480CF0F2FF011E05DA30462B4602B0F0
:10DB6000BDE87040184702B070BD00BFF8D4002077
:10DB7000B76DDBB6A3AB0200BCE7020010B5EFF354
:10DB80001184202383F31288BFF36F8F074A136831
:10DB900023F00201DB07116002D401200EF078FBB4
:10DBA00084F31188BFF36F8F10BD00BF48D50020EC
:10DBB00070B50022012104460520FFF7F5F80F4853
:10DBC00005F0F0F80E4B984215D105F0FBF82669E8
:10DBD0000C4930460BF085FD00280BDB0125356430
:10DBE0002469084904F11C000BF07BFD002801DBCF
:10DBF0000020E56470BD6FF00400FBE70DDD01005F
:10DC00000000AD0BE0EC02007FB500220123CDE95E
:10DC1000022304ABCDE90433094A6B46CDF800D0AA
:10DC2000CDF804D00CF0B6FF002805DB4FF480429D
:10DC30000023684608F01AFE07B05DF804FB00BF39
:10DC4000C1AB02000C22104B014602FB0033002046
:10DC500030B4D3E90E529863EFF31180202484F39B
:10DC60001288BFF36F8F1C6C04F0C00444F00204F0
:10DC70001C6480F31188BFF36F8F1DB12B4630BC3D
:10DC80000248184730BC7047F8D40020BCE70200B7
:10DC900010B4EFF31182202383F31288BFF36F8F48
:10DCA0001748016841F002040460C80707D482F3F2
:10DCB0001188BFF36F8F012010BC05F097B8114990
:10DCC000D1F80C04D1F80C14C907F0D5EFF311808A
:10DCD00083F31288BFF36F8F0B490B6C03F0C00303
:10DCE00043F002030B6480F31188BFF36F8F82F35C
:10DCF0001188BFF36F8F002010BCFFF7A3BF00BFD8
:10DD000048D5002000500040F8D4002010B1012870
:10DD100004D07047034B1B6C5B0701D1FFF792BF28
:10DD2000704700BFF8D400202DE9F04101220746DA
:10DD30003449D1E8EF3FC1E8E02F0028F9D133B9E9
:10DD4000314932484B60CB608A600BF0DDFC7B1EB2
:10DD5000012B28D8012F06D12D4BD3F81C3403F00A
:10DD60000303022B1FD00FF0BEFE0546E8B9294B76
:10DD70001B78D3B102220646254BC3F80823244C56
:10DD8000DFF89480D4F81824D4F81834D20315D5C9
:10DD900003F00303022B01D0012F0FD16DB386F3E3
:10DDA0001188BFF36F8FBDE8F081EFF31186202358
:10DDB00083F31288BFF36F8F0125E0E7C5B13046CA
:10DDC0000BF0ADFED4F81835DBB2012BDAD1D4F864
:10DDD0000421002AD6D00022C4F80421D4F804215A
:10DDE0000222C4F818252022C8F88021A360C9E7C0
:10DDF0000021212009F020FAE4E70222044BC3F8B5
:10DE00000423D0E7F4D40020E4D4002014D500206B
:10DE10000050004064E4002000E100E008B507483D
:10DE20000FF0ABFC38B10648FFF760FA0448FDF785
:10DE3000C7F8002008BD6FF01200FBE7F8E702000A
:10DE400045DE01000A2838B50446074D04D1AB6809
:10DE50000D2128465B689847AB6803485B68E1B2D0
:10DE60009847204638BD00BFF8E7020038B545683E
:10DE70002B69B3B11035284605F0ECFB044680B998
:10DE80000146284605F0AAFB084B98420BD12246D2
:10DE90002846074905F078FB224605213120FEF788
:10DEA00083FF002038BD6FF00400FBE70000AD0BDE
:10DEB000B5DE0100430970B507D10B4B596821B19C
:10DEC00001250C68094E854001B970BD8A682A4059
:10DED00002D030464B6898471CB1236821461C4647
:10DEE000F2E72346FAE700BF4CD50020D0E7020056
:10DEF0002DE9F04340F206354668D00648BF0320BE
:10DF0000337B02EA050558BFC2F3401087B001F029
:10DF10001F07B5F5837F144647EA43178DF80300C2
:10DF200041D00FD8062D18D007D8B5B1022D3CD05E
:10DF30006FF0150007B0BDE8F083B5F5807FF7D12D
:10DF400001250AE040F20222954230D0B5F5407F2B
:10DF50002FD0B5F5007FEBD1022522032BD501236D
:10DF600072688B409360326962BB07F01F037F09C0
:10DF700075D13D4A84F4803102EB8302D2F800323D
:10DF8000C1F30041C4F3404423F4E16344EA410493
:10DF900023F007031C4344EA800444EA0524C2F842
:10DFA00000420020C6E70725D7E70425D5E7052569
:10DFB000D3E70325D1E7630341BF012372688B4098
:10DFC000D360D0E71036394630460DF1020205F035
:10DFD000E9FA14F4403F80460CD1394630460EF041
:10DFE000F5F9224B9845DCD130469DF8021005F03A
:10DFF0003FFBD6E74FF0000901AB3946304603AA94
:10E00000CDE90439CDE90199CDF80C9005F028F956
:10E01000164B98428CD114F4003315D09DF8033080
:10E0200084F48034C4F300448DF80E3039464B46F6
:10E03000304603AA8DF80C508DF80D4005F00CFA0F
:10E040000A4B9842CDD073E7CDE9043339460DF140
:10E050000303304603AA039305F002F9F0E7803387
:10E0600052F82330FFDE00BF002584400000AD0BD6
:10E07000F0B5406801F01F04057B87B044EA451401
:10E080000569002D5FD0B2F5001F00F1100506D123
:10E09000214628460EF09CF9002007B0F0BD00276D
:10E0A000B2F5800F01AE0197776037D1B3F1007FF1
:10E0B00014BF052304238DF804300023CDE9046345
:10E0C0000393836823FA01F111F0010118D1B2F131
:10E0D000A07F15D104F01F03620903F1800338D13A
:10E0E0001D4A52F82330DB070AD40DF103063246ED
:10E0F0002146284605F056FA184B984219D0029648
:10E100002146284603AA05F0ABF8154B98421DD1CD
:10E1100001222146284605F0C3FABDE7B3F1C06FDE
:10E1200005D0B3F1007F14BF01230223C3E703230B
:10E13000C1E73146284605F0A7FA094B9842DED0E0
:10E140006FF00B00A9E76FF08500A6E76FF01500F0
:10E15000A3E751F82330FFDE002584400400AD0B17
:10E160000000AD0B08B5CA0743680AD4C1F34201E9
:10E17000012909D002290ED00121094A09480BF0D2
:10E18000DEFB6FF0150005E04FF0CC721B6800203D
:10E19000C3F8242508BD4FF0C8621B68F7E700BF2D
:10E1A000A9030300ECEA0200F8B5446800AFE36994
:10E1B000054606699847206A0CF069FD00281FDBB8
:10E1C00033462046124A04F1080105F0AFFB114B1B
:10E1D000984217D06C4688B02B686A460E49C2E94F
:10E1E00005134FF4007393830C4B42F8103F0C4817
:10E1F00000234FF4E251FDF747FF6FF00400A546FE
:10E20000BD46F8BD204605F0CBFB0020F8E700BF77
:10E2100061E201000000AD0BBB030300030000013D
:10E22000ECEA020070B5446823682046D3F808552C
:10E23000D3F80C6505F0C4FB3146284605F056FEC0
:10E240000546206A0CF023FD204605F0A9FB034B90
:10E250009D4214BF6FF00F00002070BD0000AD0B99
:10E260000378012B08D0022B08D04BB9054B0B6368
:10E2700001F1180008F0D6BA034BF8E7034BF6E7B4
:10E28000034BF4E70000AD0B0100AE0B0200AE0B38
:10E290000100AD0B2DE9F04F8DB002AFBA60142232
:10E2A0001D46D0F804B0D0F81080BBF818300646F0
:10E2B0000C46B8180021D8F834A0FB600FF096FF88
:10E2C0007D754FF0FF324FF0FF33404608F0CEFA35
:10E2D00008F118037B604FF000090022002308F1C9
:10E2E000180008F0C3FA4D46BB68994501D30024D5
:10E2F0003FE0207A020700F1AA80BB6809F101091A
:10E30000994521680AD2830708D4237D80EA030255
:10E3100002F0010203F004031A4307D025B901F00B
:10E320006043B3F1005F36D0002300E00123626850
:10E33000D7F80CE005EB020CF4451ED96C468CB006
:10E34000316802ABDA61FA684248C3E9082140F259
:10E3500003521A851A46C3E905053F4B42F8103FA0
:10E3600000234FF451513D48FDF78EFEA5466FF056
:10E370001B04404608F056FA22E0C00705D40AEB19
:10E3800005003B600FF025FF3B6862682A4495B2A8
:10E39000002B47D1CDB9002523683B626368227A00
:10E3A000BB6102F001013975BBF82410994210D20B
:10E3B0002B4A0091294801210BF0D4FA6FF01B047D
:10E3C00020462C37BD46BDE8F08F2B46C7F820A06D
:10E3D000E5E782F00202C2F340025846520107F11B
:10E3E000140105F00BFB1F4B984205D00B339842EC
:10E3F0000CD16FF00F04BCE74FF480420023786823
:10E4000008F034FA28B13046FFF70CFF6FF004042F
:10E41000AFE7D8F83030134A9342F7D1237ADB07BD
:10E4200002D400250C345FE73B6A9A45F9D12346B4
:10E4300008E0A91AD8688DB21AFA81F13B600FF092
:10E44000C8FE3B685A680C3B9542F2D2E9E76FF090
:10E4500085048EE7DB03030006000001ECEA0200FE
:10E46000A60403000000AD0B2DE9F0414568044609
:10E47000066928680FF081F918B96FF01200BDE83D
:10E48000F08130460FF02AFA7461AB68BBB9042200
:10E490000B2120466B7C0CF042FC0028EFDB0622AF
:10E4A0000B212046AB7C0CF03AFC0028E7DB012373
:10E4B0002046BDE8F0411A460B210CF030BC052384
:10E4C000062120462A7C0CF02AFC0028D7DBA8680D
:10E4D0000FF053F90028D0D0EB89A868297B43F4CA
:10E4E00080320127D0F810C013F0010FDCF80030A3
:10E4F00007FA01F714BF3B43BB43D0F808E0CCF860
:10E500000030DEF8003098470028B8DB01272B7B6D
:10E51000144A07FA03F3C6E90723A86806F11801AD
:10E520008368DB6913B96FF05700A8E73A4698474C
:10E530000028A4DB0C4BB362A868297B82680369BE
:10E540009669002EEFD01B688F401F4214BF4FF01A
:10E5500000734FF080634FF0A072B047002896DA46
:10E560008DE700BFAFAC02006DE50100262300225D
:10E570002DE9F04F044650F8100C91B0D0F80490FB
:10E580001146009306AB0CF0A6FB002805DA2046E6
:10E5900008F0CAFA11B0BDE8F08F0026234F97F8B3
:10E5A000008097F801A008F140036B4413F8273C62
:10E5B0001AEA030F13D0216931B1012354F8100C6A
:10E5C0000D6803FA06FB11BB08F101025346002156
:10E5D00054F8100CD2B20CF0A2FB0028D7DB0136A5
:10E5E0000E2E07F10207DAD1D9F8080099F80C507D
:10E5F0000669836805A95B6898470028C7D1059B11
:10E6000032685A400123AB401A42C3D0BFE78A6840
:10E610001BEA020203D04B680390984703981DB190
:10E620002B6829461D46CEE72B46FAE70F05030067
:10E630002DE9F04740F2FF15524E534FDFF84CC121
:10E6400000EB8101814202D10020BDE8F08704681F
:10E6500014F4804FC4F3C32EC4F3080340F0828047
:10E66000640CAB4208BF4FF0FF3316F80EE0192CD4
:10E670007BD8DFE804F00D131A1D7A7A7A7A7A7A59
:10E680007A204D7A7A7A7A7A7A7A7A7A5065686BD1
:10E69000C2F80C355C1C5CD10430D3E7C2F81435E9
:10E6A0005C1CF9D04FF0000910E0C2F80835F1E722
:10E6B000C2F81035F4E7C2F80835BEF1000FEFD10B
:10E6C0005C1CE9D04FF000094FF0060ED0F800A016
:10E6D0000AF40044002C16BF4FF00009C8464FF062
:10E6E000010803F01F045B0947D107EB8404D4F849
:10E6F0000032CAF3412A03EA0C0343EA8A0343EADD
:10E700000E2343EA090343EA4803C4F80032C3E78F
:10E71000C2F80C35D1E7C2F86035B3F1FF3F0468A9
:10E72000BAD0C4F30044A4B95FEA531820D101243D
:10E73000DFF854809C40C8F80C404FF00109C5E751
:10E74000C2F86435E9E7C2F86835E6E7C2F86C3527
:10E75000E3E75C090ED10124DFF82C809C40C8F867
:10E760000840EAE76FF015006FE76FF085006CE78F
:10E77000E460FFDE00239B60FBE70023803453F856
:10E780002430F6E72B05030000258440F0F8FCFF59
:10E7900038B570B14FF400450021064C0023E0FB72
:10E7A0000541054A2046FAF757FCBDE8384008F015
:10E7B00043BD38BD3F420F0040420F00F8B54468EA
:10E7C00000AF05460CF012FBA06A28B900212846CC
:10E7D0000CF081FBBD46F8BD0EF0CFFF0346B0B98B
:10E7E000A26A6C4688B011686A461548C2E90501FC
:10E7F0004FF400719183134942F8101F12484FF4EF
:10E80000E251FDF741FC6FF01200A546E2E7E38D0F
:10E81000A06A94F82C1043F400320124066913F026
:10E82000010F336804FA01F414BF2343A343D0F863
:10E8300008C03360DCF8003098470028C6DAC9E722
:10E8400033050300030000014CEB020017289FBFB3
:10E85000054B584300F5742000F510709ABF08600E
:10E8600000206FF015007047A086010010B5134C12
:10E87000A1421DDD124B98421ADCA04206DD9942EE
:10E8800006DD17236FF02100138010BD0023F9E788
:10E890006FF43A63A0F55B2018440A4BB0FBF3F029
:10E8A0001080584300F5742000F51070884202D99A
:10E8B0006FF01500E9E70020E7E700BF3F420F00D7
:10E8C000A05A3200A086010037B50D46212D114611
:10E8D0001C46406814D03A2D27D10A2A25D104229B
:10E8E000032100680DF107030CF012FA20B99DF81E
:10E8F0000720C4E90020002003B030BD1046F8E72F
:10E90000022A12D1052200680DF107030CF000FA6B
:10E910000028F1DB9DF80720002AEFD012F00A0F43
:10E9200014BF012200220248E3E76FF08500E3E70D
:10E9300020A1070070B50C2914464568036900F052
:10E94000928029398AB2142A00F29880142900F2A0
:10E950009580DFE801F00B5093811B939393939381
:10E96000939393939393937693707400188841F2E2
:10E97000883358434FF47A738012B0FBF3F203FBF1
:10E980001200584322606060002070BD9888FAF73A
:10E99000CFF801464FF08940FAF7D6F94FF07E5193
:10E9A000FAF714F8F9F734FD08F0ACFFF9F7BAFFFD
:10E9B0000646A88EFAF7BCF801463046FAF7C4F9C5
:10E9C00001463048FAF702F801464FF07E50FAF758
:10E9D000BBF92D49F9F7FAFF0546FAF7C7FA4FF0E8
:10E9E0007E512060284608F0C7FF2849FAF7F8F85A
:10E9F000FAF7BCFAC7E75A889B7A0D2B0ED80B2B77
:10EA00000ED8042B11D00020504348BF00F2FF3035
:10EA100080124FF47A7390FBF3F2B0E70F2BF2D130
:10EA2000E8684FF44873404202E04FF47A73286973
:10EA300090FBF3F0E8E71B7A00202360A3E75B7A02
:10EA4000FAE7EA68124B92FBF3F22260E86890FB67
:10EA5000F3F203FB120096E72A690D4B92FBF3F2E7
:10EA600022602869F3E7D8880A4B58430A4B90FB89
:10EA7000F3F000F5C02000F2AE50CAE76FF0850059
:10EA800083E700BF0FCF5B3B339388430024744977
:10EA900040420F0078783C0078ECFFFF2DE9F04F02
:10EAA000446887B020680EF068FE002800F05F819F
:10EAB00094F836300A22013305212068DBB20CF0CD
:10EAC0002EF90646002854D110254FF07E58DFF865
:10EAD000A4A2DFF8A49204F114076FF0004357F8E2
:10EAE000040F98420BD10235EDB2182DF5D16FF01D
:10EAF000004ADFF88892A24F04F124083EE0FAF7BA
:10EB00001BF85146FAF720F94946F9F761FF01462B
:10EB10004046FAF719F99B49F9F758FF8346A08E4A
:10EB2000FAF706F801465846FAF75AF8F9F770FC72
:10EB3000266BFAF759FE02460B463046CDE9022312
:10EB4000F9F744FCDDE90223F9F7BAFCF9F7CAFE4C
:10EB500006448302B3FBF6F303F0030200920321A1
:10EB60002A462068C3F387030CF0E8F8064600281D
:10EB7000B9D0304607B0BDE8F08F1A2558F8043FE9
:10EB800053450DD11A2DF8D162687F4811460DF119
:10EB900016030CF0AFFD163020D16FF01506E8E734
:10EBA00041F28832A9EB03035A434BBF774B784BB2
:10EBB0009B189B184CBF93FBF7F3B3FBF7F39BB287
:10EBC00003F00302009203212A462068C3F387035F
:10EBD0000CF0B4F806460028D4D0CAE70C22032172
:10EBE0009DF8163020680CF09AF806460028C0D12F
:10EBF000A268654811460DF116030CF07BFD163036
:10EC0000CBD00D2203219DF8163020680CF087F838
:10EC100006460028ADD1E2685E480DF11603A2F564
:10EC2000FA610CF0D6FC1630B7D0BDF816300321CF
:10EC300003F00102009220680822C3F347030CF09E
:10EC40007DF80646002894D1226953480DF1160339
:10EC5000A2F69E410CF0BDFC16309ED0BDF81630D9
:10EC6000032103F00102009220680A22C3F3470344
:10EC70000CF064F8064600287FF47BAF62694748D1
:10EC800011460DF116030CF035FD163085D0022229
:10EC90009DF81630114620680CF041F80646002811
:10ECA0007FF467AF0E22032194F8373020680CF010
:10ECB00036F8064600287FF45CAF0F22032194F853
:10ECC000383020680CF02BF8064600287FF451AF4E
:10ECD00001232422052120680CF021F80646002893
:10ECE0007FF447AF02460123052120680CF017F896
:10ECF000064600287FF43DAF012500952B462A46A5
:10ED0000052120680CF01AF8064600287FF431AF80
:10ED10002B460C22052120680CF001F8064600283D
:10ED20007FF427AF94F83A30BBB994F83B3033B155
:10ED300001230622032120680BF0F1FFA8B994F803
:10ED40003930002B3FF415AF012304220321206842
:10ED500007B0BDE8F04F0BF0E2BF2B465022032175
:10ED600020680BF0DCFF0028DFD0064601E76FF0DB
:10ED70001206FEE600007A4433938843AE0506008F
:10ED800078783C000FCF5B3BD8EF0200C4C3E1FFB3
:10ED90003C3C1E00CCEF0200C0EF0200A8EF0200D6
:10EDA00013B50A2A446833D1212917D03A292FD123
:10EDB0001B6820683BB901230522032102B0BDE88E
:10EDC00010400BF0ACBF0123002203210BF0A7FF82
:10EDD00000BB0123042203212068EFE7D3E90012DE
:10EDE0000D4B0E4803FB01220DF1060311460CF0FA
:10EDF00081FC10F1160F0DD0012202219DF8063082
:10EE000020680BF08CFF28B9012302460221E3E7BA
:10EE10006FF0850002B010BD40420F00A8EF020065
:10EE200070B5032904691CD80F4B58560F4B5E561A
:10EE30000F49B04202F1080201DD002070BD031D40
:10EE400004EB4303B3F9013025691B116B4393FBBA
:10EE5000F1F501FB153342F8085C42F8043C01303F
:10EE6000E7E76FF08500E9E7B9060300B5060300A0
:10EE700040420F0038B5056927216B6805F108028B
:10EE80001C680723A047041E06DA0221054A06482B
:10EE90000AF055FD204638BD2B7A13F00F0F18BF2E
:10EEA0000024F7E78A050300F4EA02003B2908B5CD
:10EEB00003D1BDE80840FFF7DDBF0329F9D00C29D5
:10EEC00007D105480221054A0AF039FD6FF0850097
:10EED00008BD6FF03C00FBE7F4EA0200A90503005F
:10EEE00008B50221034A04480AF029FD6FF08500A5
:10EEF00008BD00BFCA050300F4EA02002DE9F04195
:10EF000084B0D0F8048000AFD8F800300546066918
:10EF10009847041E17DB73680F2128469B68FA1D6B
:10EF20009847041E05DA384A012138480AF007FDDF
:10EF300009E0FB79332B0BD00121354A33480AF025
:10EF400007FD6FF0150420461037BD46BDE8F0817F
:10EF500098F80C20D3070BD544F6161142F28B4CCF
:10EF600049F22D2E2B4BC3E900C12B49C3E902E125
:10EF700094070AD573681E211C69802328461A4607
:10EF8000A047041E01DA254ACEE74FF00008072308
:10EF9000C7F8098087F80D803B72736820215C6890
:10EFA0002846062307F10802A047041E01DA1C4A7E
:10EFB000BAE7184B42461B68232133617368284621
:10EFC000DB689847041E01DA164AADE76C468AB042
:10EFD0006A4633691449C2E9088351610220042159
:10EFE0000623C2E9060142F8103F4FF4435143465D
:10EFF0000648FDF749F87368A546472220212846B0
:10F00000DB68984704469EE7F4050300F4EA020033
:10F010000C060300CCC5002094B6010023060300B3
:10F0200049060300690603009106030010B5436812
:10F03000046958680EF0A1FB38B906480121064A58
:10F040000AF07DFC6FF0120010BD044B00206360DD
:10F05000FAE700BFF4EA0200CE0603001CF002004B
:10F060002DE9F74306464FF0000800220121082051
:10F07000FDF79AFE0820FDF767FE776835693C6862
:10F080004146C4F800852E60D7F80C9001AA484686
:10F090000BF099FE002837DB019BD9F80020197985
:10F0A0001868FFF7C5FA00282EDB6B7A3169012B4F
:10F0B00003D0032B26D14FF01008AB7A032B21D1BC
:10F0C00095F80BC0BCF1000F02D0BCF1010F19D1B3
:10F0D0002A7A12B1022A15D10E226B687068B3F534
:10F0E000164F00687BD02DD8B3F5165F7AD016D8AE
:10F0F000B3F5966F78D00AD8B3F5967F77D0B3F58D
:10F10000167F77D06FF0850003B0BDE8F083B3F5CC
:10F11000166F72D0B3F5965FF4D15C4B3EE0B3F559
:10F12000E14F6DD007D8B3F5615F6BD0B3F5964F63
:10F13000E8D1574B32E047F6122E7345E2D14FF437
:10F1400000032BE0B3F5613F5ED013D8B3F5963FD3
:10F150005DD009D84DF6C02E73455AD0B3F5614F36
:10F16000D0D14FF46B0319E0B3F5E13FCAD14FF0B2
:10F17000EB7313E0B3F5612F4ED009D8DFF814E13B
:10F1800073454CD0B3F5E12FBCD14FF0E86305E0F7
:10F19000DFF804E17345B5D14FF08053C0F8243552
:10F1A000736848EA0C081B6842EA0802C3F86C2539
:10F1B0000B1DD5E9010183E803007B6899073DD564
:10F1C00005F1180003F0A0FE344B98422AD03448D1
:10F1D0000121344A0AF0B3FB6FF0040094E74FF4C6
:10F1E0001D03DBE7304BD9E74FF49E23D6E74FF4FE
:10F1F000A033D3E74FF41C33D0E74FF41D23CDE702
:10F200002A4BCBE72A4BC9E74FF06C73C6E7294B73
:10F21000C4E74FF46503C1E74FF07063BEE74FF0FA
:10F220008063BBE7287E04F10C0204F590710DF0B9
:10F2300028F801202B7E984003F056FD0823C4F8DF
:10F2400000353B7A53B9C4F81031D4F810316B69EA
:10F25000C4F834350123C4F8383523607B680020B6
:10F260009A075CBF4FF48073C4F804337B68DB06F5
:10F2700044BF4FF48003C4F804332B69C4F8443509
:10F280000123C4F84805A360E3603DE700B0130024
:10F2900000A04E0090D0030040420F000000AD0BD4
:10F2A0005CEB0200E60603000050270000C075007A
:10F2B00000F03A0000903A012DE9F04104460D4675
:10F2C00007690EF010FC4FF02008B0B92C4B1B78EA
:10F2D0009BB1642660680CF0EEFAF0B901200CF0E6
:10F2E000CEFF013EF6D10021212007F0A5FFF0E777
:10F2F00086F31188BFF36F8FF5E7EFF31186314680
:10F3000088F31288BFF36F8F60680CF0D4FA80B96D
:10F3100086F31188BFF36F8FEFE7EFF31186314665
:10F3200088F31288BFF36F8F60680CF0C4FA00286E
:10F33000DED03B691D70626838691368C3F8440504
:10F340000120C3F848050020C3F82001D3F820515C
:10F35000C3F858015268D3F85801D20608D50820DE
:10F3600062681268C2F800054FF48002C3F80423F3
:10F3700001229A6081F31188BFF36F8FBDE8F0819D
:10F3800064E400200123834070B5DC430B4AD2E8DB
:10F39000EF1F01EA0405C2E8E65F002EF7D14FF443
:10F3A000803282400648C0F80823BFF35F8FBFF366
:10F3B0006F8F0B4214BF0120002070BDF4D50020D8
:10F3C0000050014070B40E4922F07F46D1E900346C
:10F3D000D01AC31844F10004C1E90034A6F50013A3
:10F3E000B3F5400F09D2074B1B681A0A1B069C197C
:10F3F000054B42F10005C3E9004570BC08F0B2B806
:10F40000F0CF0020F8D50020F8CF0020D9B101239B
:10F410000D4A8340D2E8EFCF4CEA030CC2E8E1CFBB
:10F420000029F7D14FF48033084A8340C2F80433EF
:10F43000074BD3E8AF3FC340DB0742BF4FF4001296
:10F44000044BC3F800217047F4D500200050014060
:10F45000F0D5002000E100E00D4B1868010A00061D
:10F46000BFF35F8F0B4BD3F80435181841F100013F
:10F47000B3F5801F0AD2084BD3E90023904271EB09
:10F48000030303D210F1807041F10001704700BF07
:10F49000F8D5002000500140F8CF00202DE9F04FB2
:10F4A00085B016461F4604469DF840A0FFF76AFF48
:10F4B0000190FFF7D1FFB04271EB070352D23B4BF3
:10F4C000301A67EB0101984271F100014DD2384BBF
:10F4D00003EB0413D3E902239F4208BF964258D09E
:10F4E0004FF48038334908FA04F8204626F07F4B61
:10F4F000C1F848830CF026FA4FF00309584604F18E
:10F500005005AD00ADB205F1804504F5A87305F5D1
:10F51000A8350293029A20F07F4341F82230C1F8C7
:10F520004483D1F80435244AC01A033820F07F40C0
:10F5300090422ED9286868B1D1F80435A3EB0B00AE
:10F5400020F07F40B0F5000F039322D920460CF045
:10F55000F9F9039BBAF1000F07D109EB030009F198
:10F560000109D7E7BAF1000F09D06FF01505204661
:10F570000199FFF74BFF284605B0BDE8F08F012346
:10F580000E4AA340D2E8EF0F1843C2E8E10F00296A
:10F59000F8D107490E982301C8500F9B01EB0412C4
:10F5A0000025C2E902675360E1E700BF0100800067
:10F5B000E0CF002000500140FDFF7F00F0D500208B
:10F5C0007FB500254FF0FF304FF0FF31194C1A4B3B
:10F5D0000226C4F80833C4F84833184BC4F8085559
:10F5E000C3E902014FF480334FF40012C4F804332E
:10F5F000134B0121C4F804631520C3F880212A4667
:10F60000FDF7D2FB1520FDF79FFB01230D4AA360F8
:10F61000236013600C4B0D4A009328460023CDE96C
:10F620000155FFF73BFF3046FEF77EFB284604B04E
:10F6300070BD00BF0050014003000F00E0CF00206C
:10F6400000E100E0F4D50020C5F30100FFFF7F00DA
:10F650002DE9F7432E4BD3F8042390070BD5D3F8AD
:10F66000042142B10022C3F804212A4AD3F804310C
:10F67000136801331360264AD2F80433D90326D520
:10F68000254BD3E8EF1F21F00100C3E8E40F002C65
:10F69000F7D1CB0702D4D2F84031C3B100251C4CBE
:10F6A000C4F84051D4F84031FFF7D6FEEFF3118291
:10F6B000202383F31288BFF36F8F184BD3E90267BF
:10F6C000B042B94106D282F31188BFF36F8F03B005
:10F6D000BDE8F0834FF0FF38D3E900104FF0FF3959
:10F6E0001D60C3E902894FF48033C4F84833C4F87D
:10F6F0004051D4F8403182F31188BFF36F8F002955
:10F70000E5D0009032463B4628468847DFE700BFF9
:10F7100000500140F8D50020F0D50020E0CF0020B7
:10F7200030B5431C124C85B005D08442A8BF0446B6
:10F73000012CB8BF0124FFF78FFE0E4B0C4DD3E90F
:10F740000013401AB0F5000F0FD22218AA4228BFAA
:10F750002A46002052180849CDE90100009143F1E2
:10F760000003FFF79BFE05B030BD2A46F1E700BF5E
:10F77000FFFF7F00F0CF0020C5F3010008B5FFF7C1
:10F780006BFE024B1B68C01A08BD00BFF0CF002003
:10F7900070B50546054C064EB44200D370BDD4E9A1
:10F7A0000031284698470834F6E700BF341F0300AD
:10F7B000341F030070B5002201212A20FDF7F4FA5E
:10F7C0000B4806F081FC044628B101210346094A92
:10F7D00009480AF0BDF8094D094EB54201D320464B
:10F7E00070BDD5E90031204698470835F5E700BFE0
:10F7F00068F002001F0703003CEB0200341F030007
:10F80000441F0300F0B50F4B01461A680E4B0B2541
:10F81000002618461F46B84201D3013D04D11846C0
:10F82000013A19605A60F0BD04688C42FBD03CB1CB
:10F830004468141BA642BCBF034626460830EAE7CC
:10F840000346ECE7B8D60020C4D600200020054BC4
:10F85000C3E90000044BD3E8EF2FC3E8E10F002910
:10F86000F9D17047BCD60020B8D600202DE9F0476A
:10F8700088B005460E460DF079FF20B96FF06D0097
:10F8800008B0BDE8F0870EF092FA33680446002B0A
:10F890000F4604D107F04EFC6FF00A00F0E7BCBF42
:10F8A0004FF0FF3333600122002101A80EF099F8D8
:10F8B000E8460795EFF3118A202383F31288BFF3FC
:10F8C0006F8F07F0D7FCFFF79DFFDFF818914268B4
:10F8D000D9F800309A426CD10023434D00936B68F5
:10F8E000002B6DD1C5E900888AF31188BFF36F8FB3
:10F8F00033685A1C69D04FF4004E40F2E7300021C3
:10F9000023EAE37C4FF47A720023CCFB0E01F9F773
:10F91000A3FB02460B4601A806F0A8FFEFF3118AED
:10F92000202383F31288BFF36F8F00222B685BB113
:10F93000434554D10099002A4BD16A6829609A4204
:10F9400000D169600023009307F094FCFFF75AFF91
:10F95000D9F8003043608AF31188BFF36F8F0DF040
:10F9600005FF00288AD035686B1C27D00EF01FFADF
:10F970004FF47A7EA0FB0E320EFB0121A4FB0E4257
:10F980000EFB0722DB0BE40B43EA414344EA42440B
:10F990001B1B4FEAD1314FEAE57C61EBD231ED1A06
:10F9A0006CEB010CBCF1000FB8BF002535602DB920
:10F9B00072E743608AF31188BFF36F8F00205FE71F
:10F9C000C3F80080C5F804808EE74FF0FF3213467D
:10F9D000A1E711606968994208BF6A60B2E71A46F8
:10F9E0001B68A4E7B8D60020BCD6002030B4046859
:10F9F0002CB10D4B9C4202D3A8339C420BD30B4C31
:10FA00002378062B0BD85D1C2570074C03EB4303B2
:10FA100004EBC3030360006830BC0DF0E2BF6FF07D
:10FA20000B0030BC704700BF10D600200EDF002056
:10FA300002682AB1094B9A4202D314339A4206D380
:10FA4000074B1A7832B901221A70044B0360006820
:10FA50000DF044BF6FF00B00704700BFFCD50020D5
:10FA60000DDF002038B505460A4BD3E8EF1F013102
:10FA7000C3E8E21F002AF8D1074B1C6804B938BD5F
:10FA8000E369AB4201D005B113B9201D06F0CAFEEF
:10FA90002468F3E7B8D60020BCD600200146002237
:10FAA000002301480DF0E1BE14D7002001460148B3
:10FAB0000DF0E5BE14D700200146002200230148C6
:10FAC0000DF0D3BE28D70020014601480DF0D7BE67
:10FAD00028D7002008B54FF48062064906480DF08B
:10FAE0007BFEBDE808404FF40252044904480DF083
:10FAF00073BE00BF0FDF002014D70020E884002071
:10FB000028D7002010B5044B1C6804B910BD201D77
:10FB100006F088FE2468F8E7BCD6002070B50546DC
:10FB2000054C064EB44200D370BDD4E900312846DE
:10FB300098470834F6E700BF241F0300341F030072
:10FB4000014804F0D7BD00BF1DFB0100292800F0CB
:10FB500099800ADC01284FD0062800F09580002803
:10FB600000F08E804FF0FF307047B0F58D7F04D0ED
:10FB7000B0F5007FF6D11E2948E04B1E142BF1D8BA
:10FB800001A050F823F000BFDFFB0100DFFB010004
:10FB9000DFFB0100DFFB0100DFFB0100DFFB0100F9
:10FBA00065FB010065FB010065FB010065FB0100D1
:10FBB00065FB0100DFFB0100DFFB0100E5FB01004D
:10FBC000E9FB010065FB010065FB0100DDFB0100B5
:10FBD000EDFB0100F1FB0100F5FB01000E2100200F
:10FBE000116070470F21FAE71021F8E71121F6E7BD
:10FBF0001221F4E71321F2E736293FDC202907DC44
:10FC00001429ECD038DC0229E9D00429E7D0A9E78F
:10FC1000A1F12103152BA5D801A050F823F000BFB6
:10FC2000DFFB0100DFFB010065FB010065FB01005C
:10FC300065FB010065FB010065FB0100DFFB0100C6
:10FC400065FB010065FB010065FB010065FB010030
:10FC500065FB010065FB010065FB010065FB010020
:10FC600065FB0100DFFB0100DFFB0100DFFB0100A2
:10FC7000DFFB0100DFFB01001529C7E73D29C5E7D0
:10FC80001F29C3E72029C1E73729BFE74FF0FF321B
:10FC9000064B00201A609A611A639A641A669A6782
:10FCA000C3F89020C3F8A820704700BF40D70020B9
:10FCB0000B490346087880B90A49097839B1A2F599
:10FCC000807102290AD9A2F58872012A06D9013B5E
:10FCD000022B8CBF0020012070470020704700BF1E
:10FCE00090E300208FE3002070B400231825016802
:10FCF000084C05FB03F2A658B14206D1B0F9061034
:10FD00000832A01870BC07F0AFBD0133082BF0D14A
:10FD100070BC704740D700202DE9F3470746904656
:10FD20000C4679B300231A46C868834234D1802A2E
:10FD300071D800254FF0FF324FF0FF3338480BF0F9
:10FD400006FFA946374EE368AB422CD8002635465D
:10FD5000DFF8D0A0B14511DD85B96368384601935D
:10FD60002368A9EB060200930AEB060143460BF059
:10FD7000F2FE051EEEDD2E44B145EEDC28480BF008
:10FD8000E8FE05E009F009FF16234FF0FF35036098
:10FD9000284602B0BDE8F087A16801EBC3014968BD
:10FDA00001330A44C1E7A36806EB090003EBC5026F
:10FDB00053F8351052680EF00CFAA3684FEAC50AE2
:10FDC00053445B6801359944BDE7A3684FEAC60A0E
:10FDD00003EBC6035B683BB14FF00009A36803EB7C
:10FDE0000A025268914504D30136E368B342ECD865
:10FDF000CEE753F80A1063684944019323683846F4
:10FE00000093A2EB090243460BF0A5FE011E05DBA1
:10FE100089440D44E2E700263546E6E70D46B7E79C
:10FE200020C900200FE300204FF0FF324FF0FF33D6
:10FE300070B505460B480BF08AFE002318200A4ACD
:10FE400000FB03F156588C18013605D15550054872
:10FE50000BF07FFE204670BD0133082BF0D100244B
:10FE6000F5E700BFBCC8002040D7002038B5094DD9
:10FE700004464FF0FF3228464FF0FF330BF067FE89
:10FE800000234FF0FF32C4E900232846BDE8384084
:10FE90000BF05FBEBCC8002010B50446094B0A4AEF
:10FEA000186003680948DA61FDF794FB23680C3396
:10FEB000D3E8EF1F41F00801C3E8E21F002AF7D1A1
:10FEC00010BD00BF3CD70020DDFF010094F0020010
:10FED000F0B5A1F58173046887B0032B57D8DFE82C
:10FEE00003F0024077530127D2E9016113683A4ACF
:10FEF000B3F904300492ADF814308DF816703368FD
:10FF0000994204D109F049FE0C23036014E000F18A
:10FF1000080528460EF000F92B46002239463068C5
:10FF20000EF0D1F80823204600933C22394604AB5A
:10FF300005F012FA044610B14FF0FF340EE03368BA
:10FF400014333360CDE90200284602AA03A90EF05B
:10FF5000E8F8039B002B18BF6FF07704204607B02A
:10FF6000F0BDD2E900421368143313600023CDE9D9
:10FF7000033303AA04A908300EF0D3F8049B0BB195
:10FF8000039BE3800024E9E713684360FAE7032951
:10FF900012D0042918D1156835F4804303D009F034
:10FFA000FCFD1623036004212046C5F3803207B010
:10FFB000BDE8F0400DF0A4B9204600220DF0A0F9F4
:10FFC000840304F48044C9E709F0E7FD16239CE7A5
:10FFD0006FF05E04C2E700BFE9FC01002DE9F041CB
:10FFE0000D1E0746904612DA07F068F81C4E0123F2
:10FFF00033704246384625F04041FDF7C3F90023EF
:020000040002F8
:100000003370044607F06EF82046BDE8F0816B00BF
:1000100003D507F053F8134EE9E7FBF71DF8041E6C
:1000200009DB2946424638460CF0E9FC051E05DA94
:100030002046FBF765F84FF0FF34E5E7FFF7F4FEE5
:10004000014638B909F0A9FD0C230360284605F0E4
:1000500051F9EDE72046044AFBF73AF8D4E700BF30
:1000600090E300208FE300209CF002002DE9F04F88
:1000700014460E4600218BB00546202202A81F46DA
:1000800001910EF0B3F85CB163680293E3680493E6
:10009000A368039323690593236A03B1089302AC11
:1000A0004FF0FF324FF0FF333B480BF050FD31462D
:1000B0002246284601AB04F031FE064648B9804688
:1000C00081464FF0180A019D38604DB901980CF037
:1000D00078FC31480BF03DFD30460BB0BDE8F08FA9
:1000E00054200EF03DF8044600284FD0C0F8009090
:1000F000C0F820902B684360AB68C3606B68836076
:10010000EB680361D5F804B0BBF1010F15D10820ED
:100110000EF026F8E061002835D00823A3616B6952
:100120005A88A0F800B042805B684360B8F1000FC5
:100130002FD13C60A046ED69C7E7BBF1020F09D0A3
:100140000EF007F86FF0050638680BF0F3FC00239B
:100150003B60BBE718200EF003F8E06198B1C4F8EB
:1001600018A06A695388111D4380034602F1140CDC
:1001700023F804BB51F804EB614543F804EBF9D1D3
:10018000137D0375D2E720460DF0E3FF6FF00906FB
:10019000DAE7C8F80040CDE7E4C800202DE9F043D5
:1001A00089B007460C461546FAF756FF0646002E5C
:1001B00038681DDBFCB10DB32B6801AA082B18BFF2
:1001C00016230DF10809019349460CF092FDB0F198
:1001D00000080ADBFFF728FE074690B909F0DDFCAE
:1001E0000C230360404605F085F83046FAF788FF97
:1001F0004FF0FF3618E02246A146E5E72A46A94619
:10020000E2E764B15DB1B9F80020012A10D10823FA
:100210002B60BDF80A3022806380039B63603946FF
:100220003046164AFAF754FF304609B0BDE8F0836D
:10023000022A17D118232B60BDF80A3003AD638062
:1002400023460DF11C0C23F8042B2A4603CA6245F1
:1002500018605960154603F10803F6D19DF81C306B
:100260002375DCE709F099FC86230360404605F01E
:1002700041F83846FFF7FAFDB7E700BF9CF00200EF
:1002800007B5D0E90032012100920348034A09F082
:1002900069FB03B05DF804FB3CEB0200620703005E
:1002A00008B5034903480BF0BCFD6FF0150008BD0D
:1002B0008B070300DCEA020008B5034903480BF092
:1002C000B0FD002008BD00BFA6070300DCEA020065
:1002D00013B50B480469836801A95B689847002837
:1002E00005D008DA02B0BDE81040FFF7E5BF23688B
:1002F00001985840C00F003818BF012002B010BD4F
:10030000D0E7020010F0010210B50ED111F0010487
:1003100009D0192106480BF074FD044618B10549AF
:1003200005480BF07EFD204610BD0122F1E700BF1D
:10033000D0E70200BB070300DCEA0200002814BF7C
:100340004FF098624FF4001210B5114B19699B6879
:100350009C699CB1130206D50B68002BACBF4FF013
:1003600098624FF0307202F0C0631F21084802F417
:10037000C002A047044618B9204610BD6FF05704CC
:1003800001212346034A044809F0E2FAF4E700BFDA
:10039000D0E70200D1070300DCEA020038B5EFF332
:1003A0001185202383F31288BFF36F8F0E4C2378BF
:1003B000ABB90E4B984200D050B90020FFF7BEFFFA
:1003C00018B10B490B480BF02CFD00220A4B1A7098
:1003D0000123212223700948002306F047FC85F3FE
:1003E0001188BFF36F8F38BD92E30020D0E7020081
:1003F000F1070300DCEA020091E3002000D00020B6
:100400002DE9F041334F3B7853B10020FFF796FFC1
:1004100028B131493148BDE8F0410BF002BD3870D8
:10042000FFF756FF04462E4BD3E8EF2FC3E8E14F0A
:100430000029F9D12B4BDFF8B0801A7842BBD8F8ED
:100440000060A64219D0294B66401B680BB13146AB
:1004500098474FF0FF334FF0FF32254806F0FCF885
:10046000244B1D6835B1043D2B6831462046984722
:100470006D68F7E71E4806F067F9C8F8004054B108
:10048000BDE8F0414FF4A47200231B4806F0EEBB18
:1004900000221A70F1E7EFF31186202383F312880C
:1004A000BFF36F8F154B1D78012D05D086F3118892
:1004B000BFF36F8FBDE8F08128461C70FFF73EFF49
:1004C0003D7086F31188BFF36F8F0028F2D00C497E
:1004D000A0E700BF91E300200D080300DCEA020062
:1004E00030D80020ACC7002004D8002034D8002029
:1004F00008D800201CD8002000D0002092E3002063
:100500002608030010B54FF4003108480BF064FCD6
:10051000044620B9BDE810400F21FFF7F3BE04499F
:1005200004480BF07EFC204610BD00BFE0F0020046
:100530003E080300DCEA0200054BD3E8AF3F00B100
:100540000360044811B102685A400A6003607047B2
:1005500030D8002000D80020F8B5264B1860264877
:100560000DF0BCF9254926480BF036FC044628B1AD
:10057000244925480BF055FC2046F8BD234FBD68A3
:10058000AE691EB96FF057042149F2E703464FF4F4
:1005900000121F213846B04704460028F4D11D49F7
:1005A0001D4B4B604FF000438B60EB69F3B10122B0
:1005B000384698470446D8B9184919480DF083FAC7
:1005C0000122184B16481A700023002206F01AFB6D
:1005D00021462046FFF7B0FFFFF77AFE124BD3E823
:1005E000EF2FC3E8E10F0029C6D0F8E76FF05704FA
:1005F0000E49BEE734D8002008D8002010000100C2
:10060000E8F0020058080300DCEA0200D0E702002C
:100610007508030024D800209D0302000104020095
:1006200000D0002092E3002030D800209008030082
:100630000A4610B518B1BDE81040FFF731BE1921C8
:1006400005480BF0DEFB044618B1044904480BF0E2
:10065000E8FB204610BD00BFD0E70200BB07030047
:10066000DCEA020008B5064804F03EF8034620B173
:100670000121044A044809F06BF9002008BD00BFBD
:100680008D060200B8080300C4EA02002DE9F84311
:1006900004460026244DDFF8949000AF4D4521D349
:1006A000EEB12046F8F726FF0022411D0023204826
:1006B0000DF0DBF8054650BB6E4688B06A461D4B10
:1006C000C2E905344FF4007393831B4B42F8103F8B
:1006D0004FF4E45103461948FBF7D6FCB546BD4636
:1006E000BDE8F88395F8088018F0010F0BD1296850
:1006F00019B120460DF0CAFD28B118F0020F04D040
:1007000020466B6898470C35C8E70126FBE7214671
:1007100004300DF082FD294609480DF057F90948CB
:1007200006F002FADBE700BFCCC7002020C800209B
:1007300094C80020E508030003000001C4EA020099
:10074000A8C9002004C600202DE9F843134E144F19
:10075000DFF8508000220023304606F031F80546CD
:10076000B8B9BDE8F883237ADA070AD49B0708D41E
:10077000216819B148460DF089FD10B148466368FB
:1007800098470C34BC42EED3294640460DF077F82A
:10079000E0E7054C05F10409F4E700BFA8C9002013
:1007A00020C8002094C80020CCC70020094B1B5C47
:1007B00003F00303022B08BF2038C0B2A0F14103AD
:1007C000192B04D9A0F15F0358425841704701200A
:1007D000704700BFD91D0300A0F12C03DBB2112B21
:1007E0009DBF0348D84000F001000020704700BFC3
:1007F00001400200F8B505460024094E56F8047B76
:100800003846F8F777FE3946024628460DF00DFDCA
:1008100020B10134042CF1D10020F8BD0120FCE707
:10082000F0F002002DE9F0430468A3B0237880467D
:100830000E4615460094002B00F0CF80684B1B78C5
:10084000062B13D10020621C00921146074612F8B5
:10085000010BFFF7ABFF0028F7D107B100910B1B8D
:100860002246314628460BF090FB46E0013B082B20
:1008700043D8DFE803F064495AA20D421C3F05004B
:1008800022460021134612F8010B60B10121F9E75D
:1008900022460021534F134612F8010B385C10F02A
:1008A000440F40F0988001B100931B1BD8E76846C5
:1008B0000BF0D6FA0022009B4A481F4613F8011B92
:1008C000415C490710D102B100973B1B22463146DB
:1008D00028460BF05AFB3B783D2B07D17B783F2B0A
:1008E0000BD10237009708E00122E6E73F2B04D145
:1008F0000137F7E728460BF01EFB0020009BC8F8E5
:10090000003023B0BDE8F08327463A7810460BF05C
:100910009EFA3B46013708B9002AF6D122463146F5
:1009200028461B1B0BF031FBDCE727463A783B4699
:10093000222A07F10107F1D0002AF7D1EEE720467D
:100940000A2201A907F062FB0124019B0290009397
:10095000009B1878292825D020B303F10109FFF75F
:100960003BFFCDF8009008B9274619E00A2201A9FB
:10097000484607F04BFB22AB671C03EB840444F8AA
:10098000800C4846F8F7B6FDDDF80490044648466A
:10099000F8F7B0FD844206D0202FCDF8009002D0A9
:1009A0003C46D5E72746BB003146284602AA0BF055
:1009B0000FFB009B013300939FE70A22204602A908
:1009C00007F0A8FA0B4602990246009128463146E4
:1009D0000BF0C6FA91E701215DE74FF0FF3090E799
:1009E00094E30020D91D030010B50446F8F782FDFA
:1009F000012821D923781249CA5C02F00302022A95
:100A000008BF203B412B17D16378CA5C02F0030278
:100A1000022A08BF203B542B0ED1A27802F0F70324
:100A2000232B0BD0252A09D010460BF010FA10B951
:100A3000B2FA82F0400910BD0020FCE70120FAE77D
:100A4000D91D03002DE9F04107460468DFF89081C5
:100A500000293DD120780BF0EEF9624E054660B3D7
:100A6000062305222046604933700DF0DEFBF8B105
:100A7000052220465D490DF0D8FBC8B10B22204667
:100A80005B490DF0D2FB98B10A22204659490DF07E
:100A9000CCFB68B10B22204657490DF0C6FB38B19C
:100AA0000722204655490DF0C0FBB0FA80F56D09CC
:100AB00088F8005000203C604EE098F8003053B9B0
:100AC0002046FFF791FF002848D007233370F1E755
:100AD00098F800301BB10222424B1A70EAE7002955
:100AE00043DD224615781646284601320BF0AFF951
:100AF0000028F7D13046F8F7FDFC032830D92B4603
:100B00003F4A515D01F00301022908BFA5F120030E
:100B1000412B25D17378D15C01F00301022908BF74
:100B2000203B542B1CD1B378D15C01F00301022986
:100B300008BF203B2B2B0AD0252B11D1F378D25C98
:100B400002F00302022A08BF203B582B08D00922DA
:100B50006FF00100234B1A70BDE8F0810223B5E766
:100B600020780BF068F9002836D12278244B9B5C62
:100B70005B070AD42D2A08D02B2A06D0222A07D1B7
:100B80000322184B01341A7094E70422154BA4E792
:100B9000282A04D10122134B14441A708AE7104604
:100BA0000BF055F988B10F490B78042B0AD1224676
:100BB000144612F8010B0BF04AF90028F8D105236E
:100BC0000B7077E7082B3FF475AF1046FFF704FE74
:100BD00010B10822034B80E74FF0FF30BCE700BFA5
:100BE00093E3002094E300201C0903002209030082
:100BF00028090300340903003F0903004B090300DF
:100C0000D91D03002DE9F74F894616461F46804639
:100C1000002800F09980002A00F096805368002B8D
:100C200000F09280002410460BF060F942463368D1
:100C3000CDF804809F4228BF1F46454B1C70454B92
:100C40001C70114608780BF002F925460132044663
:100C50000028F6D105B101910025DFF8FCB0019B19
:100C60001A78002A50D0AF424ED91BF802202946EC
:100C7000120748BF013301A848BF0193FFF7E2FE06
:100C8000431C41D0023008BF00253246294601A846
:100C900008BFCDF80480FFF7C5FD013034D0019ABC
:100CA0001078FFF799FDB0B150780BF0D0F878B11B
:100CB0000135BD4241D0294601A8FFF7C3FE0130EE
:100CC00022D03246294601A8FFF7ACFD01301BD0E7
:100CD000019B01330193019A10780BF0B8F838B3F7
:100CE000013211789246084601320BF0B0F8002824
:100CF000F7D139B108460BF09EF818B95046FFF706
:100D000079FDA8B1CDF804A0019DC4B92B78CBB171
:100D10002846FFF76FFD002814BF00206FF00A007F
:100D2000B9F1000F01D0C9F8005003B0BDE8F08F51
:100D30000135BD4208BF012491E70446E4E76FF0A6
:100D40000600EDE72046EBE76FF01500EDE700BF8A
:100D500094E3002093E30020D91D030010B504465E
:100D600092B04822002168460DF040FA0D4B2168F0
:100D70001A6891421A4603D161685B6899420ED0A5
:100D800094E80300012382E803008DF8003002ABF1
:100D900094E8030083E80300684600F0EDFD12B01C
:100DA00010BD00BF3CD800202DE9F74F05230422D9
:100DB0006E460025CDE90023154FDFF85880DFF897
:100DC000589056F804BB154BBBF1040F14BF3C46BA
:100DD0004446204614BFCA469A46F8F78BFB0428BF
:100DE00010D121465046F8F77BFB58B122465946B0
:100DF0000B4803F085FC034620B10121094A0A484B
:100E00000BF0A3F915B103B0BDE8F08F0125D8E7C9
:100E10004CE4002051E4002038E400203DE40020B0
:100E2000760903008709030014EB020008B50B489C
:100E300003F066FC034638B10121094A09480BF06A
:100E400084F96FF00D0008BD074803F059FC002835
:100E5000F9D003460221054AF0E700BFB1090300BB
:100E6000BC09030014EB020076100300F209030032
:100E700010B5044692B04822002168460DF0B6F93C
:100E80000122204602A900F049FE034630B10121AB
:100E9000064A07480BF059F912B010BD0323684603
:100EA0008DF8003000F068FDF6E700BF280A030067
:100EB00014EB02000023064A13601371054A136005
:100EC0001371054A13601371044A1360137170475C
:100ED00047E400203DE4002042E4002038E4002004
:100EE00010B5044692B04822002168460DF07EF904
:100EF000204602A900F07AFF034630B101210A4AD8
:100F00000A480BF022F912B010BD029B039AA3F518
:100F10009C53083B1343F6D1062368468DF80030F6
:100F200000F02AFDEFE700BF4F0A030014EB0200B8
:100F300010B5044692B04822002168460DF056F9DB
:100F4000204602A901F0A0FB034630B10121104A5E
:100F500010480BF0FAF812B010BD9DF808305A1E78
:100F6000032A01D9072BF6D1DDE90421A2F59C5310
:100F7000083B0B4308D00A4308D00A2368468DF883
:100F8000003000F0F9FCE6E70823F7E70923F5E76E
:100F9000830A030014EB020010B5044692B0482205
:100FA000002168460DF022F9204602A901F0CAFB93
:100FB000034630B10121064A06480BF0C6F812B0CC
:100FC00010BD0B2368468DF8003000F0D5FCF6E725
:100FD000BF0A030014EB02001FB50024074B4FF4B7
:100FE0008062029302AB009305490E2305480394E7
:100FF00005F0A0FD204604B010BD00BFEF0A0300BD
:1010000068E8002060D00020072810B5144605D0FD
:1010100009280CD0BDE81040FFF74CBF07480DF081
:10102000FCF821460648BDE810400DF0F6B805482A
:101030000DF0F3F821460448F5E700BF47E400202F
:101040003DE4002042E4002038E4002010B596B0D2
:1010500004464822002104A80DF0C8F800236A467F
:1010600000938DF8043002938DF80C30204602ABCB
:1010700006A9F8F7D1FA034630B101210C4A0D4810
:101080000BF063F816B010BD69469DF8180002AA6F
:10109000FFF7BAFF9DF818301BB1074907480CF05D
:1010A00002FD022304A88DF8103000F065FCE9E78A
:1010B000FD0A030014EB020024C6002060D00020CB
:1010C00008B550B9054B1B783BB1FFF7F3FEBDE8FF
:1010D0000840034903480CF0E6BC08BD56E4002074
:1010E00014C6002060D0002008B50121034A04483E
:1010F0000BF029F86FF0150008BD00BF190B0300B5
:1011000014EB02002DE9F0410025A4B002AF044623
:101110004822002107F140000DF068F830222946EE
:1011200007F11000BD710DF061F84FF0FF3307F1CA
:101130000808C7E90233FB1D009301212046CDF8C2
:10114000048007F11003BA1D00F034FDB8B16E46FB
:101150008AB002AA3D4BD461C2E9053040F20133A6
:1011600013843B4B42F8103F4FF411512B46394842
:10117000FAF78AFFB5468837BD46BDE8F081BB79EE
:1011800003F0FB03012B04D1BB69013356D10423C7
:10119000BB7100F0BDFB0028EDD12F4ABB7911785F
:1011A000994208D087F8400007F14000137087F893
:1011B000483000F0E1FB294BB9699A68914203D1AC
:1011C000DB68FA699A421DD00423244D07F110040C
:1011D00087F840300FCC0FC50FCC0FC594E80F0037
:1011E00085E80F0007F1480607F110050FCD0FC67F
:1011F0000FCD0FC694E80F0086E80F0007F14000FE
:1012000000F0BAFB164AFB791178994209D01370A5
:10121000052207F1400087F8402087F8483000F0A9
:10122000ABFBBB7903F0FB03012BA4D1BB680133FB
:1012300008D10C490C480CF036FC9CE70B4805F033
:10124000F1FAA6E74046FFF789FD94E72F0B03006C
:101250000400000114EB020035E4002030D000202F
:1012600057E4002034C6002060D0002048C9002088
:1012700030B5A5B000214822054668460CF0B6FFFF
:1012800000F046FB0146A0B9374C2378032B3AD92E
:1012900048220DEB02000CF0A9FF607870B13021FC
:1012A0000CF062FF044650B9304A012130480AF080
:1012B0004AFF304805F0B6FA25B030BD044629464D
:1012C000294814AA239400F061FFC11D034607D0EA
:1012D00001280BD90121284A25480AF036FF0BE0E6
:1012E0000A230221254A22480AF02FFF072312A8C9
:1012F0008DF8483000F040FB20460CF02AFF219882
:101300000CF027FFD5E7284600F0C4FD044630B1B5
:1013100010210CF029FF044608B9194AC5E72846F0
:1013200002A90F9400F0D6FDC21D034607D0012884
:1013300010D90121104A0E480AF007FF10E00221DF
:10134000104A0B480AF0FFFE0A2302210E4A084801
:101350000AF0FBFE072368468DF8003000F00CFB16
:10136000002CA6D02046CBE736E400205B0B030020
:1013700014EB020090C90020E90B0300870B030067
:10138000130C0300400C0300AF0B030038B50C46F0
:10139000054640B931B30846F8F7ACF8082816D02E
:1013A0006FF0150012E0F8F7A5F80828F8D18CB115
:1013B0002046F8F79FF80828F2D129460B480CF090
:1013C0002CFF21460A480CF028FF002038BD074BAF
:1013D0001D70F6E7294605480CF01FFF0022044B5C
:1013E0001A70F2E7014B1970F8E700BFAFC7002091
:1013F000B8C7002010B538B31448F8F77BF8044696
:101400001348F8F777F8082C15D108280ED1104AA0
:101410000E49104803F074F938B1034601210E4813
:101420000E4A0AF092FE6FF00D0010BD07490C48FD
:1014300003F066F9F0E7082802D105490948F7E703
:10144000094803F05DF9E7E70848FAE7AFC700206D
:10145000B8C70020670C030014EB0200AE0C0300B9
:101460007E0C0300900C0300A30C0300811003000A
:101470000023F0B58DB00D460646CDE90333CDE926
:101480000633CDE909338DF814308DF820308DF80E
:101490002C3000285ED000295CD0304CA0212046A2
:1014A0002F4A237003F090F9034648B101212D4AD9
:1014B0002D480AF04AFE6FF00D0420460DB0F0BD35
:1014C00020462C210CF09CFE044648B96FF04C04D9
:1014D000F3E734B90121254A23480AF034FEF5E741
:1014E0000C27601C2C210CF08BFE013F0446F0D130
:1014F0000028EFD0811C082203A80CF0A8FE601C75
:101500002C210CF07DFE04460028E3D0811C08222B
:1015100006A80CF09CFE2C21601C0CF071FE00282B
:10152000D8D0811C082209A80CF091FE01AB09AAB1
:1015300006A903A800F064FA044630B1034601216D
:101540000B4A09480AF001FEB7E7019B3360029B92
:101550002B60B2E76FF01504AFE700BF95E3002002
:10156000DD0C0300EA0C030014EB0200070D03007E
:10157000210D03004FF0FF3307B5684601A9CDE9FF
:101580000033FFF775FF48B14D300AD00121064AFC
:10159000064803B05DF804EB0AF0D5BD6846FFF7D6
:1015A000DDFB03B05DF804FB4E0D030014EB0200FD
:1015B000002208B511460346034803F0A1F80028AD
:1015C00018BF6FF00D0008BD6C0D03002DE9F74F3B
:1015D00005230422CDE90023224B187090B922483C
:1015E00003F08EF8034648B1204A214801210AF051
:1015F000ACFD6FF00D0003B0BDE8F08FFFF75AFCB3
:101600000020F8E76D4600241A4E1B4FDFF86C806F
:1016100055F8049B1A4BB9F1040F14BFB246BA46F1
:10162000504614BFC3469B46F7F764FF042813D106
:1016300051465846F7F754FF40B1524649461148C3
:1016400003F05EF8034618B10F4ACEE7FFF7ACFB94
:10165000002CD5D10124DBE749460C4803F050F8B3
:10166000F0E700BF56E40020810D03008D0D03005C
:1016700014EB0200C1C70020C6C7002042E40020CE
:1016800047E40020B80D0300DB0D0300CC0D030080
:10169000014B1878FFF79ABF56E40020002313B5DA
:1016A00004460193D0B101AB0E490F480DF102027F
:1016B00003F050F9031E08DC0C4801210C4A0AF023
:1016C00044FD6FF00D0002B010BD019B00200133FE
:1016D0000CBF04239DF802302370F4E76FF015006F
:1016E000F1E700BF050E0300220E030014EB020019
:1016F0002C0E030038B5431E062B05460C4608D9B0
:101700000346124A124801210AF01FFD6FF015002E
:1017100038BD042902D90B460E4AF3E70E4B5A5C3A
:101720000E4B53F820100E4802F0EAFF40B103467A
:10173000012107480B4A0AF008FD6FF00D00E7E7AA
:10174000094B1D70094B1C70E2E700BF590E0300E6
:1017500014EB02007B0E03007110030000F1020085
:10176000A00E0300B60E0300AEC70020ADC70020D8
:1017700013B50446B0B10D490D480DF1060203F052
:10178000E9F80128034608D00A4801210A4A0AF06C
:10179000DCFC6FF00D0002B010BDBDF8063000207B
:1017A0002370F8E76FF01500F5E700BFDB0E0300CC
:1017B000E60E030014EB0200EF0E0300042838B518
:1017C000044619D804281CD8DFE800F0240A241B9A
:1017D00024000123154AAB4013421BD1012D10D127
:1017E000FFF724FB0346A8B10121114A11480AF072
:1017F000ACFC6FF00D0038BDA0F11405EDB2182D52
:10180000E7D90C48234601210B4A0AF09EFC6FF0F1
:101810001500F0E72146094802F072FF0028EAD0DF
:101820000121074A03480AF08EFCE2E7010C30016F
:101830002A0F030014EB0200540F0300700F030083
:101840007B0F0300F7B507460124294ED6E8EF3F8A
:10185000C6E8E24F002AF9D1002B46D10DF107006E
:10186000FFF71CFF054660B12146224A22480AF0D4
:101870006AFC6FF00D049DF80600FFF79FFF2546F8
:1018800029E09DF8073003F0FB03012B23D00DF175
:101890000600FFF76DFF0028EBD1184805F00CF8A3
:1018A0002046FFF78BFF04460028E4D19FB14FF09C
:1018B00096720023114804F0D9FF10F10B0F044673
:1018C00007D103210E4A0C480AF03DFC6FF0730467
:1018D000D1E70028CFD10023D6E8EF2FC6E8E13FBB
:1018E0000029F9D1284603B0F0BD6FF07605F9E77D
:1018F00038D80020B40F030014EB020048C90020C0
:10190000DE0F0300014804F01FBF00BFF8C800202D
:10191000024B1868B0FA80F04009704744D80020A4
:1019200070B50646124D4FF0FF324FF0FF331148AD
:1019300004F092FE2C6844B908200CF011FC48B960
:10194000FFF7E0FF6FF068000DE063689E4207D08C
:101950002468F0E7046046606B682BB9C5E90000B5
:10196000FFF7D0FF002070BD18606860F8E700BF87
:1019700044D80020F8C8002038B50F4C054623682D
:10198000C3B14FF0FF334FF0FF320C4804F064FE58
:1019900023680BB11C681BB9BDE83840FFF7B2BF24
:1019A00028465B6898471CB1226823461446F2E734
:1019B0002246FAE738BD00BF44D80020F8C800200E
:1019C00070B50E461446054600B132B901210A4AE7
:1019D0000A480AF0D6FB002070BD1046F7F78AFDD2
:1019E000B042F8D83246214628460CF0E2FBB0FA65
:1019F00080F04009F0E700BF8B10030014EB0200F9
:101A00002DE9F3411D46002307460E461446019377
:101A1000F7F770FD08281CD13046F7F76BFD082852
:101A200017D124B12046F7F765FD082811D1328877
:101A3000B378ADF804200021022201A88DF8063009
:101A400006F0E4FA072809D92C4A01212C480AF0AB
:101A500098FB6FF0150002B0BDE8F081294B02221F
:101A600053F820800021F01C06F0D0FAB8F1000FE6
:101A700012D14FF0FF332B609CB12288A378ADF8D0
:101A800004200021022201A88DF8063006F0BEFADB
:101A9000072815D91C4AD8E708FB00F02860013058
:101AA000EAD03A88BB78ADF804200021022201A8D0
:101AB0008DF8063006F0AAFA07280FD9134AC4E7B2
:101AC000134B53F820600EB9124ABEE702220021E0
:101AD000E01C06F09BFA70432860E2E70E4B0222FE
:101AE00053F820400021F81C06F090FA1CB1444342
:101AF00000206C60AFE74FF0FF34F9E7B01103004E
:101B000014EB020048F10200E5110300311203005A
:101B100068F102001112030068F102000023F0B521
:101B200085B007460D4602A804211646CDE90233CA
:101B30000AF0C9F9044640B103460121184A194880
:101B40000AF021FB204605B0F0BD014602AA384646
:101B50000AF094F9044648B10346134A012111489A
:101B60000AF011FB02A80AF0D8F9EBE7314601AA06
:101B700002A80AF084FA044610B103460B4AEDE7C6
:101B8000019B1BB1012B03D12B70EBE70346FBE755
:101B90000121074A03480AF0F6FA6FF01504E1E75D
:101BA000A410030014EB0200541203007F12030080
:101BB000A81203002DE9F0471D46002390B00393BF
:101BC000ADF810308DF812301646DDE9189807226E
:101BD000092382460F4605A80B21CDE900230AF010
:101BE00072F9044648B103460121784A78480AF060
:101BF000CAFA204610B0BDE8F087014605AA504653
:101C00000AF03CF9044648B10346724A0121704883
:101C10000AF0B9FA05A80AF080F9EAE701466B462E
:101C200003AA05A80AF057FA044610B103466A4A07
:101C3000ECE76A4A009903A8FFF7C2FE00284BD0E0
:101C40000DAAC7F1020105A80AF019FA041E6AD10B
:101C50000D9C052C44DC002C5ADB002E3ED1002DBF
:101C600068D125460024B9F1000F43D125F00405C1
:101C7000012DCFD1B8F1000FCCD000230825CDE93C
:101C80000733CDE90A338DF824308DF830304FF02A
:101C9000FF330295C8E90033002F40F08D802946BC
:101CA0000DEB050307AA05A80AF015FA0921044659
:101CB0000AAA02AB05A80AF00EFA50EA04020BD1F8
:101CC00043460AA907A8FFF79BFE034620B101215E
:101CD000434A3F480AF057FA00249BE73470BEE7B6
:101CE0005A2C15D106B13470002D5AD1B9F1000F1C
:101CF000F2D05A250AAAC7F1050105A80AF0BFF9D2
:101D0000002857D19DF82830002489F80030ADE72D
:101D100023460121334A2E480AF035FA6FF01504A4
:101D20002346314A72E7FBDB06B13470002D98D0B0
:101D30005A2C36D005A80AF0F1F9032836D9C7F194
:101D4000030101AB0DAA05A80AF0C5F90146D0B9F7
:101D5000019B102240336B4403F80C0C0DA806F0D5
:101D600055F90923E8600193C7F1040101AB0DAAFD
:101D700005A80AF0B0F9014640B14FF0FF33AB605F
:101D8000254604466FE74FF0FF30EAE7019B10223B
:101D900040336B4403F80C0C0DA806F037F9A8602B
:101DA0005FE74FF0FF33C5E902339FE74FF0FF30A5
:101DB000E860F4E70023A7E7072102AB07AA05A81C
:101DC0000AF089F92946044672E700BFA41003000F
:101DD00014EB0200C4120300F112030039100300D7
:101DE000210D03001A1303002C0E0300002373B50A
:101DF00006460D46CDE9003300293BD0002839D0F6
:101E0000042168460AF05FF8044640B10346012108
:101E10001A4A1B480AF0B7F9204602B070BD0146C5
:101E20006A4630460AF02AF8044648B10346154A85
:101E3000012113480AF0A7F968460AF06EF8EBE7AB
:101E40002A46022168460AF032F9044610B10346D8
:101E50000D4AEDE70D49D5E9003299424FF00803EC
:101E60009341E9D202210A4A05480AF08AF96FF043
:101E70001504E1E76FF01504CEE700BFA4100300DE
:101E800014EB0200421303006F13030000E09950AB
:101E90009C13030008B530B901210C4A0C480AF024
:101EA00070F9002008BD0023013810F8012F2C2AFA
:101EB00001D10133F9E7002AF7D10A2BF1D9A3F1B7
:101EC00009000523B0FBF3F0ECE700BFC9130300E2
:101ED00014EB02002DE9F0430B230D4600210746C9
:101EE0008DB0CDE909110493CDF82B10421E12F8E4
:101EF000013F2C2B01D10131F9E7002BF7D185F8F7
:101F000030304FF0FF330331AB6007A809F0DBFF3F
:101F1000044648B103460121974A98480AF033F92C
:101F200020460DB0BDE8F083014607AA384609F007
:101F3000A5FF044658B1C31D15D00346904A0121A0
:101F40008E480AF020F907A809F0E7FFE8E70646FF
:101F5000002104AB09AA07A80AF0BDF8044620B185
:101F60000346884AEBE70126F2E7874A049909A865
:101F7000FFF726FD002800F0A580012101AA07A88F
:101F80000AF07DF804460028DDD1019B002B40F0CB
:101F9000F080022102AA07A80AF01DF904460028D1
:101FA000D1D1029B4FF00708B3F1805FA4BF4FF07F
:101FB000FF330293029B0321AB6005AA03AB07A882
:101FC000CDF80C800AF087F804460028BBD1039BAB
:101FD0000A2130336B4403F81C0C2A1D0DF1170045
:101FE0000AF0D3F804460028ADD18DF817002A4630
:101FF0000A2105A80AF0C9F804460028A3D1042143
:1020000002AA07A80AF0E7F8044600289BD1029B21
:102010000521EB6002AA07A80AF031F8044600285F
:1020200091D1029B0621AB8205F1100207A80AF0AC
:1020300026F80446002886D1414605F1280207A863
:1020400009F0E9FF044600287FF47DAF082102AAC9
:1020500007A80AF014F8044600287FF474AF029B26
:1020600009216B8502AA07A80AF009F8044600288E
:102070007FF469AF029B0A21AB8505F1200207A816
:102080000AF015F8044600287FF45DAF3846FFF7E4
:1020900001FF85F83000C0B200EB800000F10B04B6
:1020A00007A80AF03BF884420ED2214605F1180237
:1020B00007A809F0FCFF044600287FF444AF95F818
:1020C000303033B900243EE700220023C5E906235F
:1020D000F5E76B6B002BF5D00F274FF0000895F854
:1020E0003030984504D3002EECD06FF006042AE778
:1020F0006A6B391F02EB081207A809F0C0FF4FEA0C
:102100000819044600287FF41EAF6A6BF91E4A4482
:10211000083207A809F07FFF044600287FF413AFB8
:1021200002AAB91E07A809F0AAFF044600287FF4F6
:102130000AAF6B6B029A4B445A81791E02AA07A818
:1021400009F09DFF044600287FF4FDAE6B6B029AF8
:102150004B449A816A6B39464A44043207A809F015
:102160008EFF0537044600287FF4EDAE08F1010824
:10217000B5E70124E7E600BFA410030014EB02005A
:10218000F3130300F11203001710030000232DE9DD
:10219000F04F16460B220D469946A1B002AFC7E993
:1021A0000F33BA62F860C7F843304A1E12F8013F95
:1021B0002C2B02D109F10109F8E7002BF6D14FF0E1
:1021C000FF32302409F1030886F8383086F83030C1
:1021D000B260F9684978994215D8414607F1340050
:1021E00009F071FE0446C0B10346AF4A0121AF4871
:1021F00009F0C9FF07F1340009F08FFE20467C3753
:10220000BD46BDE8F08F04FB03F0F16B01330144E0
:102210008A60F16B01448A82DBE7014607F13402F0
:10222000284609F02BFE044648B3C31D02D00346DE
:102230009F4ADBE7EA468AB002AA9E4BC2E907053D
:10224000C2E9053840F2024393849B4B42F8103FA9
:1022500000234FF432519548F9F716FF0123D54674
:102260007B61002107F1280307F13C0207F13400EC
:1022700009F031FF044620B10346904AB6E7786181
:10228000EFE78F4AB96A07F13C00FFF799FB386125
:1022900030B901218B4A854809F073FF0024A9E772
:1022A000012107F11C0207F1340009F0E8FE0446A1
:1022B00000289FD1FC69012C9CD0022C04D121461E
:1022C000814A7A4809F05DFF4FF0000A0125D046A7
:1022D000A9F10A037B607B68AB4203D9FB685B789A
:1022E00043450CD87B69002BD8D06FF00603012141
:1022F000764A6E4809F047FF6FF006047AE705F169
:102300000109494607F1200207F1340009F063FF93
:10231000044690B16D468AB002AA6D4BC2E90780AF
:10232000C2E90539052342F8103F00234FF421513B
:102330005E48F9F7A9FEAD465CE73B6AB3F1805F02
:1023400007DB0221634A594809F01DFF4FF0FF33B4
:102350003B623B6A07F12C023B650723A91C7B62A9
:1023600007F1340007F1240309F0B5FE044610B16B
:102370000346594A3AE77B6A07F11802603313446F
:1023800003F84C0C0A2107F14C0207F12F0009F069
:10239000FCFE044610B12346504A27E787F82F0079
:1023A0000A2107F1480207F12C0009F0EEFE04466D
:1023B0000028F0D107F12002E91C07F1340009F0F0
:1023C0000AFF044638B1012100904346444A374889
:1023D00007F0C8FA0EE73B6A07F12002291D07F152
:1023E00034007B6509F04BFE044610B103463D4ABC
:1023F000FCE63B6A07F16002691D07F13400A7F8AB
:102400005C3009F054FE044610B10346364AEDE64E
:1024100007F15802A91D07F1340009F030FE044607
:1024200010B10346314AE1E607F17002E91D07F1F8
:10243000340009F0F0FD044610B103462C4AD5E6FD
:1024400007F1720205F1080107F1340009F0E3FD1C
:10245000044610B10346274AC8E607F1740205F1A5
:10246000090107F1340009F0D6FD044610B1034616
:10247000214ABBE607F1680205F10A0107F13400C1
:1024800009F015FE044610B103461C4AAEE607F1FA
:102490001A0205F10B0107F1340009F0BCFD0446F6
:1024A00080B30346164AA1E62514030014EB02008C
:1024B000F31303005C14030005000001F112030094
:1024C0001710030099140300B814030070180300D8
:1024D000EF140300211503006415030084150300A5
:1024E0009D150300D3150300FD15030031160300ED
:1024F000531603007B1603009B160300BB16030054
:10250000E01603000C35294607F11A0207F13400E2
:10251000B7F91A9009F07FFD044610B10346514AFD
:1025200064E6B9F1000F00F08580B44607F1480E6B
:10253000BEE80F00ACE80F00BEE80F00ACE80F00EB
:102540009EE80F0097F81A908CE80F00B9F1000F81
:102550001DD0B9F10A0F15D90A240A230221424AD3
:10256000424809F010FE3B697B61102120460BF0C8
:10257000FBFD48B902213E4A3C4809F002FE08F141
:102580000108A8E64C46F0E7706386F830404FF04B
:102590000009BC60BB684B45F1D0726B691C02EB53
:1025A000091207F1340009F06AFD4FEA091B0446DD
:1025B00010B103462F4A19E6726BA91C5A4408321F
:1025C00007F1340009F027FD044610B103462A4AFA
:1025D0000CE607F12002E91C07F1340009F04FFD79
:1025E000044610B10346254A00E6736B3A6A5B4421
:1025F0005A81291D07F1200207F1340009F03FFD3F
:10260000044610B103461E4AF0E5736B3A6A5B4418
:102610009A81726B05355A442946043207F1340019
:1026200009F02DFD044610B10346164ADEE509F116
:102630000109AFE73023F46B07F1480C03FB0A44B0
:10264000BCE80F000FC4BCE80F000FC49CE80F00EB
:1026500084E80F0096F838300AF1010A013386F851
:1026600038308CE7031703002D17030014EB02002A
:1026700085170300B9170300DD17030007180300CF
:10268000291803004B1803007FB5002306460D46AA
:10269000CDE90233002947D0002845D0042102A803
:1026A00009F011FC044640B103460121204A2148AB
:1026B00009F069FD204604B070BD014602AA30460B
:1026C00009F0DCFB044630B103461B4A01211948DE
:1026D00009F059FD18E001210DF1060202A809F0E8
:1026E000B6FC044610B10346144AEFE7BDF80630C5
:1026F00002A82B7009F012FD022809D84FF0FF3212
:102700004FF0FF33C5E9022302A809F006FCD1E728
:10271000022105F1080202A809F0C9FC04460028BC
:10272000F2D00346064AD1E76FF01504C2E700BFB6
:10273000A410030014EB02009C180300CE18030041
:10274000F7180300F8B50E460446F0B1E9B10821C8
:102750000F4AFFF735F938B90E4801210E4A09F042
:1027600010FD6FF00400F8BD00250C4F0834214621
:1027700057F8040BF6F7B4FE08B93570F3E70135E6
:102780000A2DF4D16FF03C00EDE76FF01500EAE799
:102790002C19030014EB02003519030020F102008C
:1027A00070B5064C064EC5B2B44200D370BDD4E934
:1027B0000031284698470834F6E700BF241F03007D
:1027C000241F030010B515491548FEF7DFFD034629
:1027D00030B1144A0121BDE81040134807F0B8B8E1
:1027E000FEF708FE044610B1104A0346F2E7FEF772
:1027F000DFFE01210E4801F083FF2046FEF7E6FED2
:10280000034608B10B4AE5E701460B4801F078FFA3
:10281000034608B1094ADDE710BD00BFF419030003
:10282000FD190300061A030014EB0200271A030027
:10283000471A03005A1A03007B1A0300861A030082
:10284000034610B530B10A4A0121BDE810400948DD
:1028500007F07EB8084B1978084B1878FEF74AFF46
:10286000034608B1064AEFE7BDE81040FFF7AABFEC
:10287000A61A030014EB0200ADC70020AEC700206B
:10288000DB1A030010B50749074809F0CBFC0446E2
:1028900028B101210346054A054807F059F82046AA
:1028A00010BD00BF012B02004CD80020111B0300FB
:1028B00044EB02002DE9F041DFF8D4810D46D8F851
:1028C000704000AF072C00F008065BD0132C00F01E
:1028D000A080052C40F0B980D8F854806D496E482E
:1028E00009F09CFC18F4805F41D06C496A4809F0FB
:1028F00095FC172418F4006F04D06949664809F064
:102900008DFC182418F4007F0ED06649624809F047
:1029100085FC654B18F4004F9B6B04D00121634A82
:102920005D4807F015F8192418F4806F04D0604949
:10293000594809F073FC1A2418F4807F19D05D49B6
:10294000554809F06BFC1B24EB69002E40F09B807E
:10295000C3F3080222B96FEA53236FEA4323EB6102
:1029600029462046F9F75CFEBD46BDE8F0811624F5
:10297000C0E718F4005FE7D04F49474809F04EFC24
:102980001C24E1E7D8F85C4043484C4909F046FC78
:10299000600606D5D8F868300121494A3E4806F05D
:1029A000D7FFE10705D547493B4809F037FC262406
:1029B000CAE7A20705D54449374809F02FFC272468
:1029C000C2E7630705D54149334809F027FC2824AD
:1029D000BAE7200705D53E492F4809F01FFC2924F6
:1029E000B2E7E10605D53B492B4809F017FC2A243C
:1029F000AAE7A20605D53849274809F00FFC2B2481
:102A0000A2E723063DD53549234809F007FC2C24CD
:102A10009AE7D8F86C8032491F4809F0FFFB18F09C
:102A2000020F03D02F491C4809F0F8FB18F0010FE2
:102A300003D02D49184809F0F1FB18F0040F83D09A
:102A40002A49154809F0EAFB7EE7294A294BE8465E
:102A50008AB00F2CC8BF13466A462749103CC2E90A
:102A600005134FF400731384244BD46142F8103FD4
:102A700000234FF411510848F9F706FB0024C5461E
:102A800062E7252460E723F4FF7323F0010366E780
:102A90004CD800202401030044EB02003A0103005B
:102AA0009EFF02004B01030000ED00E06401030003
:102AB0007901030094010300FEFF02004B1B030099
:102AC000641B0300741B03008A1B0300A81B030084
:102AD000C31B0300E01B0300F51B03000F1C0300D6
:102AE000221C03003C1C03006C1C03009A1C030006
:102AF000C1010300AC010300A202030004000001B5
:102B000000B5104B89B05A6AD86C00929A6A20F0CE
:102B100005000192DA6A694602921A6B03925A6BB7
:102B200004929A6B0592DA6B06921A6C1B6D0792EF
:102B30009B0748BF40F00400FFF7BCFE09B05DF8FA
:102B400004FB00BF4CD800202DE9F0411F46164B76
:102B5000044693F800800D461646A2B0B8F1000F67
:102B600015D1684606F0BDFF3A4631462846289BF7
:102B7000A0470446684606F0B5FFB8F1000F02D042
:102B80000A4803F0E1FD204622B0BDE8F0814FF095
:102B9000FF324FF0FF33054803F05EFD0028E0D020
:102BA0006FF08304EFE700BF64E4002034C9002025
:102BB000002300B589B0CDE9063303AB04930423A9
:102BC00003900593A9B10B6806934B680793022302
:102BD000111E18BF01210848CDE9002140F2F5314E
:102BE00004AA00F02BF80028B8BF012009B05DF856
:102BF00004FB0123ECE700BF0501004070B5382657
:102C000094B006AB05460C463246002118460BF040
:102C1000EDFACDE90454CDE9020654B1012304AA2A
:102C2000009200210448019302AA00F007F814B0B2
:102C300070BD2046FBE700BF0001004010B4B1F5B5
:102C4000004F029C0ED2042B0CD8042C0AD824046A
:102C500044EA0364134644EA0102014610BC0348F7
:102C6000FFF772BF6FF0800010BC7047217C01003D
:102C700030B50468ACB1B4FA84F30122C3F11F0388
:102C8000DBB29A4024EA0202D0E8EF5FA54204D109
:102C9000C0E8EC2FBCF1000FF6D1EAD102480B706E
:102CA00030BD0248FCE700BF0000AD0B0200AD0BD9
:102CB00010B50368CB40DB0710D401238B400268BA
:102CC00043EA0201D0E8EF4F944204D1C0E8EC1F80
:102CD000BCF1000FF6D1F2D1014810BD0148FCE76C
:102CE0000000AD0B0400AD0B014BC3F804057047A9
:102CF00000700140F7B5044618B1012822D003B096
:102D0000F0BD0222264B0646C3F808230122DA60F2
:102D1000C3F80401D3F80431012342F21075204FA7
:102D20008DF80730D4B1012CE9D1D7F80C3403F475
:102D3000803386BB002BE2D0012009F0A0FA013DD0
:102D4000F3D1DCE70022164B0DF10706C3F80803A8
:102D50005860C3F80021D3F80031DDE7D7F8183404
:102D600003F480333EB9002BC9D0012009F087FA63
:102D7000013DF3D1C3E7D7F8182402F00302327003
:102D8000002BBCD09DF807000128B8D109F077FAD4
:102D9000013DC7D1B3E7D7F80C2402F00102EEE7FA
:102DA00000500040044B1A7922B9012218601A71B0
:102DB0000248704702487047C0D800200000AD0BA1
:102DC0000C00AD0B08B5074B1B6833B10520F9F7B4
:102DD000DDFF10B90520F9F7B7FF0122024BC3F858
:102DE000182508BDC0D800200050004010B510B113
:102DF000012848D010BD294BD3F81814D3F8182453
:102E0000C90324D502F00303022B05D0012B02D005
:102E10000020FFF76FFF0123204A0220C2F8183577
:102E200008224FF48273002103F1804303F5A0438D
:102E300019601C68012402F1804202F5A04214606E
:102E4000174A12681AB3154BC3F80403D2E7D3F834
:102E50001424D207DFD5D3F81C2402F00302013A70
:102E6000012AD5D80E4A12681AB10222C3F80423E7
:102E7000C0E7D3F80421002AFBD00022C3F80421C4
:102E8000D3F80431B6E700224FF48073CBE71A6819
:102E9000002AFCD019601B68ACE700BF005000405E
:102EA000C0D8002010B5164BD3F8002152B1002035
:102EB000C3F80001D3F800210122C3F80823114B05
:102EC0001B6898470E4BD3F8042182B10022C3F847
:102ED0000421D3F80421D3F81824D3F818240221AC
:102EE00002F00302012A03D1C3F818159A6010BD3D
:102EF000C3F80813034B0120BDE810401B681847B6
:102F000000500040C0D8002001460148FFF7B0BE85
:102F100044C60020036803F01F025B0902600248F8
:102F200018BF0020704700BF0025844070B43224D1
:102F30000279184B624352FA81F2083233F8124098
:102F4000E10524D5C4F3432124F4F85423F81240B6
:102F500064240026027904FB02340E3434F8025F44
:102F600015F4807F03D0C5F34325A9420FD0013665
:102F7000202EF3D164240025624302EBC1029D5050
:102F8000027904FB023070BC5830FFF791BE70BC70
:102F9000704700BF48C6002032235843034B50FA05
:102FA00081F1083133F81100400B704748C600200A
:102FB00032235843054B50FA81F1083133F81100A0
:102FC00080F00200C0F34000704700BF48C60020F8
:102FD00032235843044B50FA81F1083133F8110081
:102FE000C0F34010704700BF48C60020024611F0F1
:102FF000010004D003490B6A13600B6203B900207F
:10300000704700BF00258440F0B50546002001262A
:10301000044607468C420BD1114BD3F87C2132B1C8
:103020000022C3F87C21D3F87C3140F00040F0BD91
:10303000E3B29B0003F580729B0806FA03F31D427E
:103040000BD002F1804202F54432D2F800C0BCF14C
:10305000000F02D01760126818430134DAE700BF8E
:10306000001003402DE9F3470546544B296DD3F872
:103070000403C0B240F00040FFF7C6FF061E18DA96
:1030800000236846E96D00934FF00108FFF7AEFF9B
:1030900095F85C30DA0758D4296D4FF00040FFF7FF
:1030A000B3FF6846E96DFFF7A1FF0028F0D126F0D5
:1030B00000460124002E68D102B0BDE8F08794FAE2
:1030C000A4F4B4FA84F4E00804F1080335F813908A
:1030D00004F007021DF8003008FA02F223EA0203A6
:1030E0000DF8003001A80194FFF714FF019B4FEA8F
:1030F0009901803350F82370C9F3820A4B07D146F7
:10310000C7F3014725D552462846214609F01AF94A
:1031100001A80194FFF7FEFE019BFFB2803350F837
:103120002330C3F301439F4207D10021204609F019
:10313000FAF83946204609F0F6F801A80194FFF79D
:10314000E9FE019B08FA03F30362009C002CB6D150
:10315000A2E7022F0DD10321204609F0E4F80AF07E
:103160000503012BE9D14A462146284609F0EAF831
:10317000E3E70221204609F0D6F8BAF1030FF2D0B6
:10318000032FDAD1BAF1020FECE796FAA6F3B3FAFD
:1031900083F304FA03F29B0003F1804303F5443305
:1031A000D3F8101526EA0206D3F810252846C2F3F4
:1031B0000142C1F3042109F0C5F87BE70010034088
:1031C00032222DE9F3410379214F534353FA81F31E
:1031D000083337F813300546DB070C46CEB234D53A
:1031E00009F0CDF895F8048021464046FFF7F0FE3F
:1031F00060B121464046FFF7CFFE2A6800B202EBDD
:1032000080030022C3F81025C3F810252846214664
:10321000FFF78CFE32222B7901A802FB0366002304
:10322000083627F816300194FFF774FE019B00EB77
:103230008300D0F80022074B134043F00203C0F88C
:103240000032054802B0BDE8F0810448FAE700BF4B
:1032500048C60020F0F8FCFF0000AD0B0400AD0BE9
:103260002DE9F043D2F8009004460D46164685B08D
:10327000B9F1000F34D032220079DFF8D081424317
:1032800052FA81F2083238F81230CFB29B0703D5D8
:10329000FFF79EFE00283BD100230DF10F02CDE980
:1032A00000338DF80E308DF80F300DF10E014B46C6
:1032B000284608F0EFFF3221237901FB037308331E
:1032C00038F8132022F0020228F81320237901FB9A
:1032D0000377083738F8173043F0010328F8173020
:1032E0007368002B43D04FF0320C22791F780CFB0F
:1032F00002F2D3F804E052FA85F2544B083233F864
:103300001200E9B210F0020F04D0BEF1000F18D085
:103310004F482FE020F4604020F0200023F81200F6
:10332000BEF1000F0DD0032FF2D8726850682268EA
:1033300090F800E002EB8E02FFB9C2F81075C2F8F7
:1033400010754FF0320C22790CFB0212083233F860
:10335000120020F01C0023F8120022790CFB02114D
:10336000083133F8112042EA870223F81120B368AC
:1033700063BB384805B0BDE8F083D2F8108528F06B
:103380000308C2F81085226802EB8E00D0F81025E1
:1033900022F4473222F44072C0F810252A02D0F8F5
:1033A000108502F4F85242EA074242EA0802C0F8E5
:1033B000102522790CFB0212083233F8120040EA81
:1033C0004E3040F0200023F81200BAE72946D3E936
:1033D00000872046FFF7AAFDB8F1000FC9D064238B
:1033E00020791A4E4343F218F358984504D1536894
:1033F0009F4201D100210CE0642303FB00600DF12A
:103400000F015830FFF734FC124B9842B2D19DF8AF
:103410000F1064222379534303EBC10346F8038062
:1034200023795343322203EBC10333445F60237992
:10343000534353FA85F3083336F8132042EA412206
:1034400042F4807226F8132093E700BF48C600209C
:103450000400AD0B0000AD0B2DE9F04305460C4612
:103460001F4685B09AB306793046FFF7A1FD20B11B
:1034700021463046FFF7ACFD80BB32235E43DFF8C8
:10348000FC9056FA84F6083639F816305FFA84F85C
:1034900013F01C0F02D05378012B1FD001238DF89D
:1034A0000F3000232046CDE900230DF10F01931CBE
:1034B000013208F0EFFE32222B7902FB038808F17B
:1034C000080839F8183043F0030329F81830002FA2
:1034D00051D021462879FFF76BFD18B1284805B077
:1034E000BDE8F0833E782B68244903EB8603C3F8DC
:1034F0001005C3F8100532202B794FEA860C4343A0
:1035000053FA84F3083331F813E0E2B22EF4604E3C
:103510002EF0200E21F813E097F801E0BEF1000F25
:1035200029D02B68BF789C44DCF810354FEA0E4E4A
:1035300023F4981323F4F853CCF81035230203F442
:10354000F8530EF4403E3F05DCF8108543EA0E03C5
:1035500007F480173B4343EA0803CCF810352B7976
:1035600000FB0322083231F8123043EA463343F0BD
:10357000200321F812300348B1E700BF48C60020FD
:103580000400AD0B0000AD0B30B564250479044B8D
:1035900005FB0434A160017905FB0133DA6030BD1D
:1035A00048C6002038B505790C462846FFF710FDBF
:1035B00058B132235D43064B55FA84F4083433F88E
:1035C000143004485B0B137038BD0348FCE700BFA0
:1035D00048C600200000AD0B0400AD0B2DE9F04102
:1035E000064607796420184D00FB075898F860409C
:1035F00044BB40462146402210300AF0F7FD2146E8
:103600003068D8F850608E4212D10023C0F87C3167
:10361000D0F87C3140F30730F9F796FB642303FBC5
:1036200007550123094885F86030AB65BDE8F08196
:10363000CBB29B0003F580727C2B04BF845083586F
:103640000131E0E70248F1E748C600200000AD0B79
:103650000C00AD0B64210279044B01FB023393F89B
:103660006000003818BF0120704700BF48C6002026
:1036700064235422007913FB002302481844FFF707
:1036800017BB00BF48C6002064235422007913FBF7
:10369000002302481844FFF7EBBA00BF48C60020D9
:1036A00073B503680D46D3F8041306460029A4BF7A
:1036B0004FF00041C3F80413047929462046FFF770
:1036C00087FC00B329462046FFF772FCD8B1294693
:1036D0002046FFF761FC002501B23468890001F53E
:1036E0008073E550E35833680B44D3F8101541F06C
:1036F0000101C3F8101522B1012332688340C2F8DA
:10370000043302B070BD32235C43104B54FA85F48D
:10371000083433F81430C3F38203042B11D0052B83
:1037200011D001A80195FFF7F5FB019A0369D34079
:1037300003F00103991C284602B0BDE8704008F070
:10374000F2BD0321F7E70221F5E700BF48C60020DC
:103750000148FFF787BC00BFACC6002070B5084C1D
:103760000E462379154643B92A20F9F7EDFA0123CD
:10377000044823712660A56070BD0348FCE700BFC4
:10378000C8D800200000AD0B0C00AD0B002330B5F5
:103790000D4A50F8234003F5A2710133082B42F87B
:1037A0002140F6D10023084A00F11C0103F5B27450
:1037B00051F8045F0133082B42F82450F6D1036C12
:1037C000C2F8043330BD00BF00A0024038B5002469
:1037D000154D2A20C5F81045C5F81445C5F81845FB
:1037E000C5F81C45C5F82045C5F82445C5F8284549
:1037F000C5F82C45C5F89045C5F89445C5F89845D9
:10380000C5F89C45C5F8A045C5F8A445C5F8A84528
:10381000C5F8AC45F9F7A6FA4FF0FF33C5F8083301
:10382000024B1C7138BD00BF00A00240C8D8002068
:103830000123024A8340C2F80433704700A00240CB
:103840000123024A8340C2F80833704700A00240B7
:10385000F8B5012600270B4B0B4DD3F80C4304B9E8
:10386000F8BD94FAA4F0B0FA80F006FA00F324EA66
:103870000304064B82009F502B68002BEFD0A968F1
:103880009847ECE700A00240C8D8002000A1024001
:1038900010B4CC7B8A6803682CB9D1E90041C3F825
:1038A0000845C3F80C15C3F824252822037953438F
:1038B000054AD3582BB1006810BC40F30730F9F724
:1038C00043BA10BC704700BFD4D8002070B5817BCC
:1038D000E9B9046804F01F0364091AD140F20C65C9
:1038E000104A114E02EB8303D3F8001231402943F2
:1038F000C3F80012416801F01F0349090DD102EB22
:103900008303D3F8002232402A43C3F80022012067
:1039100070BD803351F82330FFDE803354F82330FC
:10392000FAE700BF00258440F0F8FCFF2DE9F041E4
:10393000074690F80480282000FB08F0144E0C463F
:10394000351895F82210F1B9A96032506B6085F8EE
:10395000251085F824106CB1A37B204685F827300C
:10396000FFF7B4FF88B1637B2146384685F82630DF
:10397000FFF78EFF282303FB08660123054886F81E
:103980002230BDE8F0810448FBE70448F9E700BFB6
:10399000D4D800200000AD0B0C00AD0B0400AD0B23
:1039A000062103680279C3F800152821034B01FBA7
:1039B0000233022283F82220704700BFD4D80020AF
:1039C000282102790B4B01FB023300219960026828
:1039D0000948C2F80803D2F8000220F4BC50C2F82B
:1039E0000002C2F80015012283F8241083F8222077
:1039F000704700BFD4D8002002029C012DE9F84F87
:103A000028239046002290F80490AE4D046803FBF2
:103A1000095383F823204B680E4633B1CB6803F07B
:103A20006043B3F1005F40F085813378023B012BA6
:103A300006D8336903F06043B3F1005F40F07A8148
:103A4000A14BC4F80833282303FB095393F824102F
:103A500001F0FF0239B19B68DFF870B2C4F804339B
:103A60005846BDE8F88F18F0140F0CBF0121002153
:103A700083F82410317809EB890783F820107178D6
:103A800005EBC70783F82110F168D96071681961E7
:103A900031695961B168C3F81C809961C8F300119C
:103AA00083F825107378C4F88835C4F86021D4F8F9
:103AB0006031C4F84821D4F84831C4F82421D4F83E
:103AC0002431C4F80421D4F8043118F0010318BFDC
:103AD0000123C4F8503518F0020318BF0123C4F8BD
:103AE00040353378032B00F2A480DFE803F07999A6
:103AF00062024FF48073C4F80032D7E90323C4F89C
:103B00004425C4F848350123A3604FF480112046B2
:103B100008F0A2FC0028F8D1D7E90523C4F8442511
:103B2000C4F8483528234FF4802203FB09539A60D8
:103B3000DFF89CB1282202FB09F218F0080AAB5802
:103B400005EB020013D13178032910D0012940F090
:103B500086802160002B6FD0282202FB09F2716859
:103B6000AA5821B9002A00F0BB80012262612822F4
:103B700002FB09F2A918AA58002A00F0B18018F037
:103B8000040F1CBF00228A6018F0400F06D12822C3
:103B900002FB0952916841F002019160282202FB68
:103BA0000952916841F4007191609268C4F804234D
:103BB00056E7D7E90323C4F84425C4F84835D7E9C4
:103BC0000523C4F83425C4F838354FF48453C4F8B9
:103BD0000032012323622823022203FB0953A6E7B4
:103BE00018F0200FD7E90323C4F8442514BF4FF47D
:103BF00080724FF40072C4F848354FF0280315BFA7
:103C0000C4F80022C4F800224FF48022022214BF1C
:103C100003FB095303FB09539A600123236287E7DF
:103C2000D7E90323C4F83425C4F838354FF480535A
:103C3000CDE7DFF8A0B07DE7026902B961612649EE
:103C4000DFF898A0204608F007FC012210F4007F5E
:103C500018BF626110EA0A0F1F49F3D07CE7012107
:103C6000A160002B7FF478AF006918B31B4B1AEAF0
:103C7000030F7FF471AF2046174908F0EDFB10F4F5
:103C8000007F8246F2D04FF08071204608F0E4FBBE
:103C9000D4F8001280B111F4007003D101228246E1
:103CA00022626261CB05E1D54FF48021204608F005
:103CB000D3FB04E06161D9E70122226262614FF027
:103CC000000AD3E7D4D8002002029C010B00AD0B00
:103CD0000000AD0B0400AD0B020204000200040062
:103CE000282101FB09550021D4F8C424C4F8C424B8
:103CF00085F824108AB11149114B12F0010F14BF3D
:103D00008B469B46013112F0020F18BF8B4612F012
:103D1000040F0C4A18BF9346A2E618F0400F7FF438
:103D20009FAE3946204608F055FB054A002808BFDB
:103D3000934695E6DFF810B092E600BF0000AE0BA8
:103D40000100AD0B0200AE0B0A00AD0B70B55D4D6E
:103D5000022186B0284608F07FFB4FF4007106462A
:103D6000284608F079FB584CD8B1E6B9A3684FF063
:103D70008071C5F808330223A360A3682846C5F8FC
:103D8000043308F069FB18B1D5F800329B0503D461
:103D900001224C4B1A625A61012384F8233006B089
:103DA00070BD002E58D0E5696E060AD494F8233011
:103DB0003BB94549434808F00DFB80F0010084F809
:103DC000230015F0040525D13E4B94F82520C3F8B7
:103DD0006051D3F86011C3F85C51D3F85C1112B193
:103DE00094F823205AB10022C3F80022A260374A77
:103DF000C3F808234FF48062354BC3F88021238C2D
:103E0000ADF80430E3680493236902936369059372
:103E1000A36903932B4AD2F8C4349807C2F8C43478
:103E20004AD459074AD4DA074AD494F823309B007D
:103E3000DBB28DF8003094F825300BB984F82430CB
:103E4000E3695B0703D594F82330002BA7D0D4E9AE
:103E5000003168469847A2E74FF48021284608F0D1
:103E6000FBFA94F82030ABB994F8253053B94FF4ED
:103E70008062C5F80032A360144BC5F80833144BB8
:103E8000C3F8802100238DF8043094F821308DF898
:103E90000530B7E74FF40073C5F8003240F2022353
:103EA000A36003F1CE73C5F80833A368C5F80433E3
:103EB0000123AB602B6272E70123BAE70223B8E764
:103EC0000323B6E700A00040D4D8002002029C01E2
:103ED00000E100E0036803F01F025B090260024892
:103EE00018BF0020704700BF00258440F7B5064684
:103EF00008F0DCFA084608F0D9FA01A80196FFF7A5
:103F0000E9FF0C4640F20D61019B2B4D00EB830055
:103F1000D0F8003201942B400B43C0F8003201A8C6
:103F2000FFF7D8FF019B012700EB8300D0F8003298
:103F30002B400B43C0F80032042008F0A0F90925FB
:103F400001A80194FFF7C6FF019A0369D340DB077C
:103F500014D401A80196FFF7BDFF019B013D07FAAC
:103F600003F3C360042008F08AF9304608F09EFA93
:103F7000042008F084F915F0FF05E1D101A80194AF
:103F8000FFF7A8FF0123019A9340C360042008F0C3
:103F900076F9204608F08AFA042008F070F901A8A2
:103FA0000194FFF797FF019A03690448D34003F097
:103FB0000103C01A03B0F0BDF0F8FCFF0100AD0B27
:103FC00070B503680446033BDBB2052B03D8094AEE
:103FD00052F823502DB9A06858B1BDE8704000F0E8
:103FE0001DB808F0BFFA21682B46BDE87040090CE7
:103FF000184770BD88F10200014B5B69184700BF8C
:1040000010C70020014B1B68184700BF10C70020D5
:10401000014B5B68184700BF10C70020014B1B69AC
:10402000184700BF10C70020014B9B68184700BF0E
:1040300010C70020014B1B6A184700BF10C70020A3
:10404000014B5B6A184700BF10C70020014B1B687B
:10405000D8687047FCD80020002230B50B4B196897
:104060000C6894420FD001EBC2039D68A8420BD1AB
:104070004FF003020433D3E8CF1F002903D1C3E874
:10408000C02F0028F7D130BD0132EAE714D9002053
:104090002DE9F041002406460F462046DFF8548003
:1040A0003368A34201D8BDE8F08106EBC4056B6814
:1040B000DBB2012B16D16A68B8F80030B3EB124FAF
:1040C00010D1022FA8680FD1FFF77AFF01206B688B
:1040D00023F0FF0343F003036B60B8F800300133B3
:1040E000A8F800300134DBE70168090C08F0EAF9B0
:1040F000ECE700BF5CDD002010B5074C02216068D2
:10410000FFF7C6FF0028F9D101212068FFF7C0FFA3
:104110000028F3D110BD00BF1CD9002070B50728BE
:1041200060D8DFE800F00B5F475F435F3C0402F0BC
:1041300075F80320BDE87040FBF794BC03202A4BC0
:10414000D3F81446D3F81866284B1D781870EDB2D2
:1041500002F032F8012D10D1254B264A9C4212D094
:10416000230C1B04B3F1886F0DD0A4F58033203BE2
:10417000022B0FD96FF0040313603146C4F30B0018
:1041800002F00EF800E014601B4B186807F0F4FB17
:104190000020CFE7194931F913301360F4E7002408
:1041A000124B20461C7002F007F8EDE7FFF7A4FF62
:1041B0000220BFE70D4B1A78012AD0B20ED1104A67
:1041C0001168104A8C6854604968116002221A70A4
:1041D00001F0F2FF084B186807F0CEFBFFF78CFFE9
:1041E0000120A7E770BD00BF00A0024059E40020F5
:1041F0000100500518D9002004D900204AF502001A
:1042000000D900201CD900200A23F7B54FF47A7595
:104210000C4E0D4F01933168386808F07EF9044662
:1042200040B907F0A7FB40B9012001A9FBF71EFB2D
:104230006E30F0D1204603B0F0BD0198684307F01E
:1042400091FBE8E708D9002010D90020054B1B7826
:104250002BB9054B1968054B186808F05EB90020AA
:10426000704700BF58E400200CD9002014D900206A
:1042700070B5164B42681B6822F0FF0242F0020242
:10428000C31A42601248134A0168C3F38913D2E883
:10429000DF4F651CC2E8D65F002EF8D101EBC301E9
:1042A0004A6892B242EA04424A600268032002EB82
:1042B000C302536823F0FF0343F00103536007F088
:1042C00051FB0122044BDA6070BD00BF0CD9002005
:1042D00014D900205EDD002000A002402DE9F04F3F
:1042E00095B038220021064603A809F07FFF02237B
:1042F0000493082306932023089304230D9310238B
:1043000040250F9380230122CDE91153D5230021AD
:1043100057480B921393FBF769FB0546002840F0C2
:10432000A380024653493079FFF718FA03A8FFF734
:104330002DFA34686268B2F59D6F40F09280616931
:10434000E3680B44E16903F59D630B44B3F5003F5B
:1043500000F287802068294609F048FF33681C680E
:10436000D3F81C9004F53A72019204F16007424AB6
:1043700004F1A40804F1200BB9F1000F5BD1C2F8DD
:1043800000B000254FF0010A2570657084F802A086
:10439000E570336840461B69636033685B69C4F845
:1043A00014B0A360354BC4F81890C3F80080344BA8
:1043B000E7601F600823C4F8108084F8A43088F8F0
:1043C000015088F8025088F8035084F860307D70FE
:1043D000BD70FD7008F084F8384608F081F8294B6C
:1043E00004F53A721A60284B04F1E80231681A6049
:1043F000264B274E1960274B2749C3F81046C3F8B0
:104400001456264B264C1D80264B86F800A01D8096
:10441000254B029525601D611B690293029B144B7D
:10442000186807F0ABFA98B103236FF07304337088
:10443000FFF7CCF911E09B6904F14009636433682C
:104440004846DB69C2F800B0236401F0C3FE98E778
:104450002468002CECD1154B1C70204615B0BDE82B
:10446000F08F6FF01504E3E76FF02D04F5E700BF60
:1044700004D900201D41020000D9002014D90020D9
:1044800010D900200CD9002008D90020FCD8002029
:1044900059E4002000A00240F04902005EDD002047
:1044A00018D900205CDD00200056004058E40020B0
:1044B00070B5164B42681B6822F0FF0242F0010201
:1044C000C31A42601248134A0168C3F38913D2E841
:1044D000DF4F651CC2E8D65F002EF8D101EBC301A7
:1044E0004A6892B242EA04424A600268032002EB40
:1044F000C302536823F0FF0343F00103536007F046
:1045000031FA0122044B5A6070BD00BF08D9002067
:1045100010D900205EDD002000A0024010B5FFF79A
:1045200073FE012400220321047081704270C27066
:10453000FFF7BEFF054B1C7007F0E5FFBDE810401C
:10454000034B47F23051186807F018BA58E40020BE
:1045500004D9002038B50A4B04461B78022BDDB283
:104560000DD1FFF751FE50B100220121846001708E
:1045700042708570C270BDE83840FFF799BF38BD02
:1045800059E40020034A126812B1002800DB1047EA
:10459000704700BF30D900202DE9F7430025814640
:1045A0000F461048294690461E46019303F038FDF9
:1045B000041E11DB0134204607F0FDFFC9F800009E
:1045C00068B1334642462146019603F029FD28464C
:1045D0003C6003B0BDE8F0836FF01500F9E76FF0C1
:1045E0000B00F6E7C8EB020010B50E4B04461B6843
:1045F000A3B1F4F77FFF082810D9237A3F2B0DD001
:1046000009490822204603F047FB014630B904F16E
:1046100008000A22BDE8104003F0F8BC4FF0FF305C
:1046200010BD00BF30D90020CE1C03002DE9F3419E
:1046300005460020174688461E4607F095FF0246AD
:1046400040B915B1284607F0B8FF6FF00B0002B073
:10465000BDE8F0816FF05803002403730423056064
:104660000E4D037244738473C47344728472C472B3
:10467000C0F80480394603202C7007F091FF4FF0FA
:10468000FF3301932B78B34201D10020DFE70220F2
:1046900001A9FBF7EBF80028F4D0D8E75AE4002092
:1046A000F8B5054600240F4F57F8046B28463146ED
:1046B00009F0ECFD28B90134042CF5D14FF4803019
:1046C0000DE06CB1A31E012BF8D83046F4F712FFB1
:1046D0000A220021284403F07FFB40EA0440F8BD91
:1046E0002046FCE7A0F10200014B18600020704753
:1046F00034D90020014B1860704700BF30D900202A
:104700000FB42DE9FF410A9C01F05CFD00284AD05E
:10471000002C4BD0284E294F3168386807F050F9EB
:10472000002846D1264D3168286807F027F900286F
:1047300036D122460BAB03A902A80193FFF72CFF49
:10474000044658B1286807F017F9386807F036F9B9
:10475000204604B0BDE8F04104B07047029C2046FA
:10476000FFF742FF02230646012220460399FFF786
:104770005DFF04460028E5D1DFF84880D8F8000046
:10478000FFF78EFF0446D8F8000007F010FF2868F6
:1047900007F0F2F8002CD8D13046FFF7F3FED4E74B
:1047A0006FF00A04D1E74FF0FF34D1E76FF00D044A
:1047B000CEE76FF00A04CBE748D9002040D90020AB
:1047C00044D9002038D900200CB42DE9F04F89B02D
:1047D00080460F46129C01F0F5FC002800F0A280F4
:1047E000B8F1000F00F0A180002C00F09E80002F97
:1047F00000F09E80514DDFF848B12968DBF80000D9
:1048000007F0DEF8002840F096804E4E29683068A8
:1048100007F0B4F8002840F08280224613AB07A9C5
:1048200006A80593FFF7B8FE044618B1306807F0F4
:10483000A3F823E0DDE906930193434B1D68002DA7
:1048400039D00C228246414B1B6802FB0353029372
:10485000029B9D421CD1BAF1000F2CD0306807F0AA
:104860008BF84A4639464046D047044618B9404678
:10487000FFF716FF0446484607F09FFEDBF80000EE
:1048800007F09CF8204609B0BDE8F04F02B0704731
:10489000AB68A3420DD9019A48469A4228BF1A46EE
:1048A0002968039303F0F8F918B9039BD5F804A01D
:1048B0001C460C35CCE74846FFF796FE022305461A
:1048C000012248460199FFF7B1FE04460028ADD108
:1048D000DFF87C904046D9E9004ABA455246214665
:1048E00028BF3A4609F075FCBA45204607D907F0BB
:1048F0005EFE306807F040F86FF00604BEE7FFF791
:10490000CFFE0446D9F8000007F051FE306807F0EA
:1049100033F8002CB2D12846FFF734FEAEE76FF033
:104920000A04ABE74FF0FF34ACE76FF00D04A9E7E2
:104930006FF01504A6E76FF00A04A3E748D900203A
:1049400040D9002044D9002028D9002024D90020B3
:1049500038D900200EB42DE9F343DDF824808146D8
:1049600001F030FC00285DD0B9F1000F5DD0B8F146
:10497000000F5AD0304C314F2168386807F020F8CA
:10498000002855D12E4E2168306806F0F7FF002828
:1049900045D14846F4F7AEFD451C284607F00BFE0E
:1049A000044668B9306806F0E7FF6FF00B0438681A
:1049B00007F004F8204602B0BDE8F04303B07047AA
:1049C00049462A4609F043FC2046FFF70DFE022324
:1049D0008146012220462946FFF728FE044630681A
:1049E00014B106F0C9FFE2E706F0C6FFB9F1000F07
:1049F000144D06DB2868FFF753FE10B94846FFF751
:104A0000C1FD0AAA41462868019203F03BFB041E3F
:104A1000286808BF6FF04C0407F0C9FDC7E76FF0C6
:104A20000A04C4E74FF0FF34C4E76FF00D04C1E798
:104A30006FF00A04BEE700BF48D9002040D900202B
:104A400044D9002038D9002038B5C3680446A72BC4
:104A500001D0206810E0032907D0042926D00229BC
:104A600002D10122154B1A7038BD144B00681A7818
:104A7000022A05D10028F7D0BDE8384007F097BDDD
:104A80000F4D2A6862B12B689847002320682B607D
:104A900007F08DFD0B4B1868BDE8384006F06CBF81
:104AA000094A1060616851600222DCE7074B1B680D
:104AB000002BCED000689847CBE700BF5AE4002017
:104AC0002CD9002044D9002038D9002034D9002026
:104AD000012210B511460B48FAF788FF70B90A4851
:104AE000FAF7A6FF014648B94FF0FF32074B1A60AC
:104AF000BDE8104001230522FFF798BD6FF02D009F
:104B000010BD00BF44D9002040D9002048D9002062
:104B100010B400F11C03D3E8EF2F511EC3E8E41FCB
:104B2000002CF8D1012A0CDC074BD0E8EF2FC0E8AD
:104B3000E13F0029F9D16422002110BC043009F0C2
:104B400055BB10BC704700BF1EF1010010B500241A
:104B50000A4B4FF45072214609481C7009F046FB7D
:104B600021462246064B074801310829C3E90002C5
:104B70009A6003F16803F7D110BD00BF5BE4002029
:104B80004CD900201EF10100164830B50022034622
:104B90004FF0FF34144DD0E8EF1FA94204D1C0E814
:104BA000EC4FBCF1000FF6D10CBF0121002112D156
:104BB000682101FB023301220C49DA61097893F87C
:104BC000202061F3451283F820200222A3F8482018
:104BD00083F84A2030BD0132082A00F16800DAD19A
:104BE0000846F7E74CD900201EF101005BE40020E5
:104BF00030B5024600236825054905FB03F460181B
:104C00000C59944203D00133082BF6D1002030BD5B
:104C10004CD9002010B50446043007F0C2FE606C89
:104C200008B1FAF743FF064BD4E8EF2FC4E8E13FA1
:104C30000029F9D12046BDE81040FFF769BF00BF49
:104C40001EF1ADDE70B50825064C074E2368B34251
:104C500002D02046FFF7DEFF013D04F16804F5D1E4
:104C600070BD00BF4CD900201EF101002DE9F843B2
:104C70000F4C06460025A0464FF068090D4B0E4F1D
:104C800018702368BB420CD009FB058393F82020E1
:104C900066F3451283F82020A36B13B1204607F07A
:104CA000EEFC0135082D04F16804EAD1BDE8F88373
:104CB0004CD900205BE400201EF10100112806DC25
:104CC00000280DDB084BC34003F001007047B0F52E
:104CD000817F07D040F21113C31A584258417047E0
:104CE000002070470120704741000200034B02681A
:104CF0005A6082699A6042691A6070478CDC0020B1
:104D0000012208B511460448FAF770FE002818BFC2
:104D10006FF02D0008BD00BF98DC00202DE9F04F9A
:104D200085B082460F4616461D4601F04BFA28B95B
:104D3000012006F019FE6FF00A041CE05AEA07038E
:104D400000F051811EB3336823F4A05323F0020313
:104D5000002B40F04B81706838B9B06878B107F02B
:104D6000C3FD60B96FF0060405E007F0B7FD002849
:104D7000F3D16FF00504204605B0BDE8F08FF06870
:104D800028B1B16807F0C4FD08B96B20D1E79A4B90
:104D90004FF47A61186806F0F1FD0446002840F0EF
:104DA0002881002F64D0F6B1336803F4A053B3F523
:104DB000805F18D13368DB0445D44FF0FF3770684B
:104DC00008B100F093FD8D4B8D4A1860B368002B3D
:104DD00008BF01231360F3688A4A002B08BF06232B
:104DE000136033681CE00A220021384603F00EF9F4
:104DF0004FF6FE73421E9A4200F2F280824A03028C
:104E000043EA10231380002ED4D1002301217B4AD2
:104E10004FF0FF3713607A4A11600621794A11601A
:104E2000DFF8E8815046C8F80030BAF1000F65D1CC
:104E300007F09AFB064600BB6FF009046E4B18683A
:104E400006F09AFD97E73A21384609F0D9F900B102
:104E5000471C38466E4909F019FA0A2228B1002188
:104E6000033002F0B9FF0746A9E701463846F8E7E4
:104E7000654B1880002EC8D09FE707615F4BDFF8B5
:104E800080B11B68DFF87CA1B361DBF800303246EB
:104E9000F361DAF8003047F20D013362D8F80030E0
:104EA0000420736107F07CFB4FF0FF33594F5A4EDB
:104EB00003933E603868B04231D0002840F08C80C7
:104EC0002020D7F80490FAF7E9FD286070B109F1C5
:104ED00018034D4A019318461288B9F8141007F0C8
:104EE00074FB064638BB2868FAF7E0FD6FF009044A
:104EF00078680028A2D007F05AFB9FE7F4F7FAFA87
:104F000007F032FB0646002896D007615046F4F7BA
:104F1000F1FA51460246306809F05BF9AEE702202B
:104F200003A9FAF7A3FC0028C4D06E2006F01CFDEC
:104F30006FF00A0482E7D9F808102A6801290AD01C
:104F400002291FD01046FAF7B1FD3046FAF7AEFD40
:104F50006FF00504CCE708211161D8F8001011F0BA
:104F6000020137D00192B9F816000130FAF796FD28
:104F7000019A90612A68906930B91046FAF796FD57
:104F80003046B1E71621E7E7B9F8141009F1180324
:104F90000B441946B9F8162009F01BF900202968BE
:104FA000B9F81620896988542A680192D9F808004E
:104FB00008F0BFF9019A2B685060DBF800205E61B1
:104FC0009A60DAF80020DA60D8F800201A6000222F
:104FD000DA618DE79161E7E708F0F1F9044687E7C8
:104FE0006FF007042AE76FF00104C4E64FF0FF34C6
:104FF000C1E66FF00204BEE698DC0020A4DC0020CD
:10500000A0DC00209CDC002060DD0020A8DC00206B
:10501000EF1C03008CDC0020EEC100BCF8B548F2A8
:105020000F03994205460E4640D022D848F20D03A0
:10503000994233D048F20E03994233D00069FFF70A
:10504000D7FD044610B3B6F5004F1FD9A6F50046AC
:10505000013E0B2E1AD8DFE816F0AE00E800B600CD
:10506000B600B6003A013A01B600C40019001900B2
:105070000B0149F2040399421CD0B1F5104F3FD9FE
:10508000C068FFF7B5FD0446002848D1286800280D
:1050900000F02D81BDE8F84007F089BABDE8F8407E
:1050A000FFF724BEBDE8F84007F09CBCBDE8F8401F
:1050B00007F085BC0369082B00F21981DFE813F0C3
:1050C0001000160009000E00160017011701180045
:1050D0001E000020BDE8F840FFF7C8BD0120F9E739
:1050E0000021E868BDE8F84007F0BCBB0121F8E703
:1050F0000021E868BDE8F84007F0C0BB0121F8E7EF
:105100000069FFF775FD04460028BFD048F281030F
:105110009E42BBD10146284600F038FB56E049F2DA
:1051200002039E4200F0CD8037D807F023FB0746EC
:10513000E0B91020FAF7B2FC0646B8B139461022A1
:1051400009F054F82B6873606B683381698A002911
:1051500000F0C8802A8A05F1140007F036FAF060E2
:10516000002840F0BF803046FAF7A0FC286807F01E
:105170001EFA204607F0C0FA58B1204607F0FAFAA6
:1051800038B994F8203043F0800384F820300C23A1
:10519000A361204607F0B5FA18E049F203039E42E6
:1051A0003DD049F282039E427FF470AF014628460B
:1051B00000F004FB0AE06B692BB9284608F019F9E6
:1051C000AA6943681A60284608F015F9204607F0D6
:1051D000E1FA002800F08B802046BDE8F84007F097
:1051E0004EBA90F8203043F0010380F8203007F0E9
:1051F000A8FA18B13E4B186806F0BEFB94F82030B0
:10520000204623F00A0384F8203007F0C3FA10B1D7
:10521000204607F034FA2046FFF7FCFCD3E7286964
:1052200069280BD16823A361D0E790F82030EE689D
:105230006FF3410380F82030686918B100F06AFB11
:10524000A061C3E7204607F066FA28B994F8203039
:1052500043F0040384F82030204607F05CFA00286D
:10526000B4D0002EB2D00021204600F0C5FAADE740
:105270006B69F3B9284608F0BCF8AA6943681A605C
:10528000426892F8203043F0040382F820304368EB
:1052900022691A61436862695A6183684BB105F1FA
:1052A000180205F1300152F8040B8A4243F8040B4E
:1052B000F9D194F82230002B85D0013B84F82230BC
:1052C00081E790F82230013380F822307EE72846CB
:1052D00008F08FF86B6913B9AB69436073E74FF05F
:1052E000FF33FAE73146204607F0E6F96EE7F8BDEE
:1052F000ACDC002030B585B00546FFF779FC0446EC
:1053000028B9092006F030FB4FF0FF300EE000F026
:1053100059FF68B9204607F014FA18B10D4B186808
:1053200006F02AFB2046FFF775FC002005B030BDD3
:10533000002007F019F9014608B96920E2E7056184
:1053400001AA47F2090000F0FDFA0028EDD0162866
:10535000EBD0D7E7ACDC00202DE9F04385B08146E7
:10536000884615461C460C9FFFF742FC40B90920B1
:1053700006F0FAFA4FF0FF33184605B0BDE8F083A7
:1053800014B90FB11620F3E7B8F1290F00F0ED8042
:105390000CDCB8F1010F12D0B8F1060F00F0E1807B
:1053A000B8F1000F00F0DF806D20E1E7B8F58D7FE8
:1053B00000F08880B8F5007FF6D11E2D08E03D2D65
:1053C000F2DC202D0EDC142D4ED0152D53D0022DE5
:1053D000EAD1384607F0C8F80646002840F0C780F2
:1053E0006920C5E7A5F121031C2BDDD801A252F8E5
:1053F00023F000BFD3530200D3530200A95302008D
:10540000A9530200A9530200A9530200A9530200A4
:10541000D3530200A9530200A9530200A95302006A
:10542000A9530200A9530200A9530200A953020084
:10543000A9530200A9530200935402009B54020096
:105440009F540200A3540200B3540200A953020067
:10545000A9530200A9530200A9530200A953020054
:1054600085540200B75402003A46214605B0BDE813
:10547000F04307F0C4BF3A46214605B0BDE8F0430B
:1054800007F0CBBF3A46214605B0BDE8F04307F030
:10549000D2BF01230422019305E00223FAE703238C
:1054A000F8E7042201920DEB020107F0E4FF034646
:1054B00062E70523EEE73A46214605B0BDE8F04332
:1054C00007F0D9BF6B1E112B3FF66EAF01A252F849
:1054D00023F000BF2B55020055550200D3530200A4
:1054E000A9530200475502001D550200A9530200AE
:1054F000A9530200A9530200A9530200A9530200B4
:1055000039550200D3530200D3530200D353020093
:10551000A9530200D3530200D35302003A46214656
:1055200005B0BDE8F04307F0C9BF3A46214605B0D3
:10553000BDE8F04307F0D6BF3A46214605B0BDE8C6
:10554000F04307F0E4BF3A46214605B0BDE8F0431A
:1055500007F0EFBF3A46214605B0BDE8F04307F03B
:10556000F7BF372D34E71F2D32E7202D30E700231A
:105570000822437202728372C372C0F810904046D0
:1055800007F000FF7061284600F0B8F9B06124B15F
:105590003A462146306808F01CFE314647F20300C7
:1055A000776001AA00F0CEF9034600283FF4E4AE8C
:1055B000DEE600BF2DE9F04385B0814688461746F8
:1055C0001D460C9EFFF714FB40B9092006F0CCF9EC
:1055D0004FF0FF37384605B0BDE8F08305B10EB98E
:1055E0000E20F3E7B8F1290F00F08F800CDCB8F142
:1055F000010F11D0B8F1060F00F08380B8F1000F51
:1056000000F081806D20E1E7B8F58D7F2AD0B8F5F4
:10561000007FF7D11E2F0EE0152F1CD00ADC042FBF
:1056200012D0142FEED13246294605B0BDE8F04322
:1056300007F0C5BF212FE5D1306806F095FF04467D
:10564000002864D16920C1E73246294605B0BDE88B
:10565000F04307F0A4BF3246294605B0BDE8F04349
:1056600007F0BCBF7A1E122ACCD801A151F822F053
:10567000E7560200F556020039560200395602007C
:10568000D9560200BD56020005560200055602001A
:10569000055602000556020005560200CB560200D0
:1056A00005560200395602003956020039560200EA
:1056B00005560200055602003956020032462946B8
:1056C00005B0BDE8F04307F098BF3246294605B063
:1056D000BDE8F04307F0A3BF3246294605B0BDE858
:1056E000F04307F0AEBF3246294605B0BDE8F043AF
:1056F00007F0B9BF3246294605B0BDE8F04307F0D0
:10570000C4BF372F97E71F2F95E7202F93E700237C
:105710000822437202728372C372C0F8109040462E
:1057200007F030FE6061384600F0E8F82146A061DD
:1057300001AA47F20400D4F8008000F003F90746FC
:1057400020B1404606F039FF38463FE762683368CB
:1057500041469A4228BF1A462846326008F039FD71
:10576000404606F02AFF35E708B5FFF7EFF9FFF7E7
:10577000C7FA40B9012204481146FAF737F9002860
:1057800018BF6FF02D0008BDACDC002010B54369D8
:105790000C467BB191F820306FF3C30381F82030C1
:1057A000406900F0B7F8044BA061BDE810401868EC
:1057B00006F0E2B810BD00BFACDC002010B591F8D7
:1057C00020300C466FF3C30381F82030006960B9C4
:1057D000DBB223F0140343F0140381F82030054BAF
:1057E000BDE81040186806F0C7B800F093F8A06153
:1057F000F5E700BFACDC00202DE9F341DFF8E880DD
:105800000546D8F80000019106F0B8F8074650B1F7
:10581000019B002B65D11023AB614FF0FF37384659
:1058200002B0BDE8F081686CA8B1F3F763FE461CD6
:10583000304606F099FE044678B9284606F086FF01
:1058400008B16923AB61D8F8000006F095F869202B
:1058500006F08AF8E1E73E46EAE72B680422036196
:105860000023027243728372C37295F84B2005F1D4
:105870004801013292008260143008F0AAFCF6B1AF
:105880003246696C206808F0E2FC666095F82030CA
:10589000042043F00803224647F2810185F82030B6
:1058A00006F07EFE284606F051FF0028B7D12846B4
:1058B00006F047FF40B9A8690028B0D0C8E72670B5
:1058C0006670A670E670E0E7022001A9F9F7CEFF46
:1058D00010F10B0F05D00028E9D00028B8BF4042D6
:1058E000B6E77420B4E700BFACDC002003289CBFFF
:1058F000014B1856704700BFF31C030002383528CF
:105900009ABF034B53F820004FF0FF30704700BFA1
:1059100088F3020070289ABF024B53F82000024817
:10592000704700BFC4F10200ADBAADBA0138042817
:105930009ABF034B53F820004FF0FF30704700BF71
:10594000B0F102004FF0FF3337B50D4DCA60144679
:1059500015600A4601460420019306F021FE2068E6
:10596000A84202D0FFF7D6FF08E0022001A9F9F70C
:105970007DFF0028F3D00028B8BF404203B030BDFF
:10598000EEC100BC431C07D0064B984207D83C230D
:10599000B0FBF3F080B270474FF6FF7070474FF6E0
:1059A000FE70704787FF3B002DE9F34105460E4628
:1059B000144600F007FC002800F0C1800023614F6E
:1059C0003246294607207B6006F0EAFD4FF0FF33A0
:1059D0000193022001A9F9F749FFD7F80480064690
:1059E000B8F1000F06D110F16E0FF2D1304602B0BF
:1059F000BDE8F08110F16E0FF8D0D8F80450022DF8
:105A000000F0948047F6FF739D4200F09280002DD5
:105A100040F0928044B142F209023B88934209D09F
:105A200042F20912934240D078680028DED006F096
:105A3000BEFDDBE74FF443722946204608F0D6FB53
:105A4000B8F8083001222360D8F80A01FFF79AFF5E
:105A5000A080D8F80E01FFF795FFE080D8F812017A
:105A6000FFF790FF2081D8F81601FFF78BFF6081C8
:105A7000D8F81A01FFF786FF20231546A081A373EB
:105A8000511E2274657408EB8101D1F80A00FFF7FA
:105A900079FF6082D1F88A00FFF774FF0132212A72
:105AA000A08204F10604EBD1BEE7294620464FF45C
:105AB000437208F09BFB0621B8F80830103444F814
:105AC000103CB8F80A3024F80C3CB8F80C3024F834
:105AD0000A3CB8F80E3024F8083CB8F8103024F826
:105AE000063CB8F8123024F8043C98F8143004F856
:105AF000023C08F1150398F814200633954204F18E
:105B0000060491DA13F8062C04F8062C13F8052C79
:105B100004F8052C01FB0582B2F81700013524F8C2
:105B2000040CB2F8192024F8022CE4E76FF00C06FC
:105B30007AE76FF05E0677E76FF0150674E74FF0CF
:105B4000FF3653E7C0DC002070B50446002800F0A3
:105B50000881022A00F0B980032A00F0C480012ADB
:105B600040F0FF80E72940F2FF80824D2B68002B38
:105B700000F0FD80FEF75EFAE8220021204608F0E2
:105B800035FB7D4B1B78032B2B6858689968C4E95B
:105B90000001D8681969C4E902015A6922619A6949
:105BA0006261DA69A2611A6AE2615A6A22629A6AD9
:105BB0006262DA6AA2621A6BE2625A6B226393F83B
:105BC000512084F85020D3F841202264D3F8452096
:105BD0006264D3F84920A264D3F84D20E2641A8F9E
:105BE000A28693F83A2084F8362093F83B2084F874
:105BF000372093F83C2084F8382093F83D2084F82F
:105C0000392093F83E2084F83A20B3F83F20A28749
:105C100032D1D3F852200A25C4F8E42000225234AD
:105C200003F1590193F85600824205DA0C2A04F177
:105C30000C0401F10A0103D1FEF702FA002070BD45
:105C400005FB0230B0F85760013224F80C6C11F8F3
:105C50000A6C04F80A6CB0F85A6024F8086CB0F9C1
:105C60005C6024F8066CB0F95E0024F8040C11F8AE
:105C7000030C04F8020CD5E7D3F8CA201946C4F87F
:105C8000E4200A26002206FB0230B0F8525001320E
:105C9000A4F8525091F854500C2A84F85450B0F89B
:105CA000555004F10C04A4F84A50B0F9575001F1D2
:105CB0000A01A4F84C50B0F95900A4F84E0091F82C
:105CC000510084F85000DED1B6E752294CD92B4D53
:105CD0002B68002B4BD0FEF7ADF9532220462968E4
:105CE00008F077FAA8E767293ED9254D2B68002BE5
:105CF0003DD0FEF79FF9234B1B78012B23D168225F
:105D00000021204608F072FA0022296808340B8826
:105D1000C81C44F8083C8B7804F8043C8B78183491
:105D20009A4289DA02EB0213C55C0B4404F8185C52
:105D30005E6853F8085F013244E904655D689B685A
:105D400044E90253EAE72B681A8922600122227192
:105D5000227200221968C4E904125B68C4E90632A1
:105D60006AE76FF015006AE76FF0790067E76FF098
:105D7000220064E7BCDC00205DE40020B8DC0020E9
:105D8000B4DC00205CE400202DE9F04100F01AFAB8
:105D9000054600285FD0314E4FF0FF31306805F0E6
:105DA000EDFD044600284DD12D4C2378B3BB00F007
:105DB00009FA002849D100F005FAA8B14FF002080D
:105DC0004746152007F07DFC014650B105220368C7
:105DD00041F204001A71C3F805700022FFF7E4FDD8
:105DE00018B1B8F1020FE6D1002500F0EBF9A8B127
:105DF000152007F066FC014680B1036800226FF0B1
:105E00007F00012718715A7141F203209A71DA71EB
:105E10009F74FFF7C9FD0DB100B92770152007F079
:105E200050FC0146A0B101250368002241F20400A4
:105E30001D71FFF7B9FD044608B90A4B1D703068A3
:105E400005F09AFD2046BDE8F0810327B846B8E783
:105E50006FF00B04F3E74FF0FF34F3E7C8DC0020EA
:105E60005FE4002060E40020014B186000207047D0
:105E7000B0DC00202DE9F041056807460C463DB135
:105E800001F47043B3F5005F04D1404BC3E9001542
:105E9000BDE8F0813E4E336863B144F204029142A2
:105EA00064D00CD844F2020399424ED044F203036A
:105EB000994253D03868BDE8F04106F078BB44F20F
:105EC000012221F4807393420FD044F203139942CC
:105ED000F0D1304C206808B106F069FB01222E4B4E
:105EE0001A7025600420336826E0DFF8B080D8F807
:105EF000000008B106F05BFB44F201339C420CBF8A
:105F00000322022295F85170254B264C1A70C8F8CE
:105F1000005017F008053368227810D01AB9052010
:105F200098470123237007F04107012F02D1022077
:105F30003368984701203368BDE8F0411847002ACC
:105F4000F1D0062098472570EDE7174C206808B17E
:105F500006F02DFB032033682560EDE70D4C20682B
:105F600008B106F024FB00220B4BB9E72A78032A7C
:105F7000A0D8DFE802F0020507090720984799E753
:105F80000820FBE70920F9E70A20F7E7C0DC00203A
:105F9000B0DC0020B4DC00205CE40020BCDC00208D
:105FA0005DE400205EE40020B8DC002008B500239A
:105FB000094A0A4813700A4A13700A4A13700A4AB7
:105FC00013700A4A136001221146F9F70FFD0028E9
:105FD00018BF6FF02D0008BD5EE40020C8DC002073
:105FE00060E400205FE400205DE40020B0DC0020DD
:105FF00010B50B4C206818B106F0D9FA00232360C5
:10600000084C206818B106F0D2FA00232360064C31
:10601000206818B106F0CBFA00232360002010BDE1
:10602000BCDC0020B8DC0020B4DC002030B4074B1E
:106030001C6844B143688589A4460268C1899BB243
:10604000E8B230BC604730BC704700BFCCDC0020F9
:1060500037B50125074C4FF4FA70656105F082FCF5
:10606000002363610193256123690193019B03B0C0
:1060700030BD00BF0056004030B50D4D89B0036AF9
:1060800003AC01908DF808300FCD0FC42B6801A828
:10609000236006F023FA40B9044603AD55F8043BEB
:1060A000984710B90134052CF8D109B030BD00BFB4
:1060B0008CEB0200034BD3E8EF2FC3E8E10F00297C
:1060C000F9D17047D0DC002038B50546002850D003
:1060D000436A002B50D0836A002B4DD00124294BFA
:1060E000D3E8EF2F002A03D1C3E8E14F0029F7D10D
:1060F00045D1686A00F04EF8F9F7ECFC224BC82055
:106100009C6605F02FFC2846FFF7B6FF044640B911
:1061100001221D4B0220DA66FFF7CCFF0024204647
:1061200038BDFFF795FF002C11DBAB6A204698477E
:10613000164B9C421AD013DCA4F18864033C012C5A
:1061400011D82846FFF798FF04460028E0D0012226
:106150000D4BDA66F9F7D6FC0020FFF7ABFFDEE760
:106160000B4B9C42EDD06FF00404F0E76FF00A0493
:10617000EDE76FF00D04D2E76FF01504CFE74FF0B5
:10618000FF34CCE7D0DC0020005000400500400484
:1061900001005005014B1860704700BFD4DC00209F
:1061A00007B5044BCDE900011B686846984703B06A
:1061B0005DF804FBD4DC0020014B1870704700BF71
:1061C00061E40020024B1878431E58425841704742
:1061D00061E400200021074B01221970064B197061
:1061E000064B1960064B1960064B18600648F9F714
:1061F000FDBB00BF62E4002063E40020DCDC002083
:10620000E0DC0020F0DC0020D8DC0020024B186825
:1062100008B105F0B1BB7047D8DC002070B4284B42
:106220001B68196958691A7C00221A745C7C5A74BC
:106230009C7C9A74DC7CDA741C7D1A755C7D5A75C2
:106240009C7D03299A75DC7DDA7529D0042929D033
:1062500001290FD185681B4E954210D11A7A012170
:1062600000221972597A5A72997A9A72DA7A6FF010
:106270005F02DA72144B70BC186805F07DBB911C8C
:1062800000EB81014C682178622907D0633918BF7F
:106290000121490046F821400132DDE70121F9E7FB
:1062A000187ADEE7187A1972597A5A72997A9A72BC
:1062B000DA7A6FF05F02DA720122044B1A70D9E7C2
:1062C000F0DC0020E4DC0020D8DC002063E40020C7
:1062D000014B986864307047F4DC002010B5044628
:1062E000F5F7F2FD03480121034A03F028FB20469D
:1062F00007F04EFA44EB0200F71C03002DE9F843C7
:1063000004460D4600AFEFF31188202383F3128873
:10631000BFF36F8F0428294A98BF294BE9468AB0FA
:106320009668117C98BF53F820306A4688BF254B89
:10633000C2E9073140F2013323489384234BC2E979
:10634000050442F8103F00234FF431512048F5F77F
:106350009BFECD4645B1EB69C3F3080323B1012190
:106360001C4A1B4803F0EBFA2EB1304607F0C4FB81
:1063700008B1037803B91848E9468AB06A46174B52
:10638000D061C2E9053640F201331384144B42F860
:10639000103F00234FF411510D48F5F775FE2946C3
:1063A000CD462046FFF79AFF88F31188BFF36F8F21
:1063B0003046F6F745FCBD46BDE8F883F4DC002026
:1063C00060F40200061D03001C1D0300050000010F
:1063D00044EB0200441D0300141D0300651D03006F
:1063E0000400000138B5094B53F82040013053F840
:1063F0002050A54200D838BD636823B1204607F07D
:10640000CFF90834F5E723689847FAE774F40200F7
:10641000012270B5294B032086B01A70FFF7E2FF06
:10642000F6F7F0F80420FFF7DDFF254C254D264652
:10643000AE4204F1300410D300F040FE204C224E56
:10644000AC4226D300F04EFEF4F7DCF81F4A137B73
:1064500023F00103137306B070BD54F80C3C059390
:1064600054F8103C049354F8143C039354F8183C2B
:10647000029354F81C3C019354F8203C009354E9D7
:106480000A2354E90C0100F0F7FB54F8303C5E6538
:10649000CDE7D4E90A23B3F1FF3F08BFB2F1FF3FD4
:1064A00005D052EA0301206803D107F027FB3034FE
:1064B000C6E73146183000F0DBFFF8E764E400205F
:1064C000B4EA0200B4EA02003DDC020090D10020F0
:1064D00008B50348034A0021121A07F079F908BDEC
:1064E00030CA002068E40020882370B5134E0122D2
:1064F00003FB0066002386B0CDE904230F2201933D
:10650000CDE9023214234FF4A0720D4D0D4903FB67
:106510000055044602FB00110B4B3046009500F07D
:10652000ABFB737B2C7423F004037373074B0134B0
:1065300003EBC423EE606B6006B070BD08D1002091
:10654000F4DC002068F40020B7D8020068EC0020DA
:10655000BFB50020FFF746FF2E4B03F5006282F324
:10656000088883F30A880024E0232B4D2B4E85F8FE
:106570002230EC772C766C76AC7685F820406B6A0E
:10658000274F43F4E0236B6285F82340F6F7DAFAED
:10659000F6F77AFC4FF0FF33AB62EB62F6F718FECA
:1065A000F6F796FCF5F700FC40F201131D4D284666
:1065B000AB81C5E91A4401F087F9B56007F0DCF852
:1065C0000120FFF70FFF0220174DFFF70BFF00F030
:1065D000A9FD164B75610593012315494FF48052AF
:1065E000CDE9034328463B46CDE90144009400F041
:1065F00043FB06466A7B284622F004026A7307F0D2
:10660000C2FA2046FFF770FF3A4631462846F6F7B1
:106610001DFC00BF68EC002000ED00E0F4DC002071
:1066200011640200C0D2002090D10020C71D0300D9
:10663000A8F5002038B5064C064DAC4201D3002029
:1066400038BD2046D4E9011207F0C6F81434F4E747
:1066500080C80020A8C800202DE9F3410446174651
:106660001E46EFF31188202383F31288BFF36F8F48
:10667000C368334A7BB180689168884219D057EA71
:10668000060318D188F31188BFF36F8F6FF00F00E6
:1066900002B0BDE8F081916891F90E100133E3601A
:1066A00093682161A36088F31188BFF36F8F002086
:1066B000EEE72169F2E791F90E1090F90E306FF0D4
:1066C0007E029942A8BF19469142B8BF11468B423B
:1066D0002DDD07F0FBF8054622464146CDE9007660
:1066E000184800F037FC0028E1D0EFF31186202392
:1066F00083F31288BFF36F8FA068D0B1236821693C
:106700009C420AD04BB193F90E309942A8BF19466A
:106710006FF07E039942B8BF194607F0D7F840B131
:106720003146084800F086FC6FF00A00B0E700250B
:10673000D2E7002DF4D186F31188BFF36F8FF3E712
:10674000F4DC002065E4002038B58368044663B3B8
:10675000194A926893422BD1C368012B03D9013B9C
:10676000C360002038BDEFF31185202383F3128826
:10677000BFF36F8F0169806807F0A8F8204607F023
:1067800077FAA06058B190F90E2022610022C2670A
:1067900007F0F9F92946094800F04CFCE1E7E06010
:1067A00085F31188BFF36F8FDBE76FF01500D9E732
:1067B0004FF0FF30D6E700BFF4DC002065E4002096
:1067C00037B51146EFF31185202282F31288BFF30B
:1067D0006F8F04689CB12368426823F003039442DE
:1067E000036008BF43600121204607F0E3F8044638
:1067F00085F31188BFF36F8F204603B030BD51EA97
:106800000302F5D000F10802CDE900131046294635
:1068100000F0A0FB0028EFD1014B9B685C69EBE71F
:10682000F4DC002038B50446EFF31185202383F310
:106830001288BFF36F8F07F01BFA48B10022C267BE
:1068400007F0A1F92946BDE83840074800F0F2BB3F
:10685000D4E902329A4218BF01330221A36004F145
:10686000100007F03FFCEDE765E4002013B5EFF3FF
:106870001181202484F31288BFF36F8F846844B1A0
:10688000013C846081F31188BFF36F8F002002B058
:1068900010BD52EA030406D181F31188BFF36F8F54
:1068A0006FF00F00F3E7CDE900230246014800F046
:1068B00051FBECE765E4002070B50446EFF3118569
:1068C000202383F31288BFF36F8F6FF00A062046F0
:1068D00007F0CEF918B1C66707F055F9F7E7A060E1
:1068E000022104F1100007F0FDFB2946BDE87040CD
:1068F000014800F09FBB00BF65E400201FB5094AB6
:1069000002AB92E803004FF4906283E80300009327
:1069100005494FF0FF33054800F00CF9002005B0A1
:106920005DF804FBB4EB0200A805012018D200209A
:106930002DE9F04305464FF0FF364FF0FF37DFF803
:106940002C8185B0EFF31189202383F31288BFF3E4
:106950006F8FD5F888408CB9022105F1A00007F0AF
:1069600050F8002860D100234946CDE90067029322
:1069700005F190023E4800F083FCE3E7D5F88C2057
:1069800023689442C5F8883008BFC5F88C30D5F824
:10699000A03043F00203C5F8A030E36823F00403FD
:1069A00043F00103E360636889F31188BFF36F8FDD
:1069B00020469847EFF31189202383F31288BFF311
:1069C0006F8FE368D90623F0010237D4E260E368F1
:1069D0009A071AD5D8F8000023F00203E360A0B1AB
:1069E0000021026888B143689C4237D1036869BBC3
:1069F000D8F80420C8F80030824201D1C8F8043029
:106A0000002340F8083BFFF70DFFD5F8A03023F036
:106A10000203C5F8A03089F31188BFF36F8FDB053F
:106A200090D400F087FB8DE705F198040022012146
:106A3000204607F081F90028F8D194E723F01103EC
:106A4000E36004F11000FFF7EDFEC0E70B60D8F83B
:106A50000430834208BFC8F80410D1E722B113689C
:106A6000014610461A46BDE71346F9E714DD00203B
:106A700065E40020F8B5C36804469A070F46C3F3DF
:106A800040062CD45B071AD40B680BB983680B60E3
:106A9000E368DD0742BFA36802263B603D6858BF3C
:106AA0000126002D3AD01F4B9B68AB420AD0D5F887
:106AB000A030D807C3F3800214D46FF0120600236D
:106AC0003B6025E007F00FF8D5F8A0300028F0D1A2
:106AD000D907C3F3C002F0D552B15B0708D46FF0F9
:106AE0000F06ECE7002AFAD1C3F3C003002BF6D15E
:106AF00000232360D5F88C3063B9C5E922442846C9
:106B000006F099FFE36843F00403E3603B68A36089
:106B10003046F8BD1C60C5F88C40F0E76FF01506F4
:106B2000CDE700BFF4DC00200146014806F0BBBF02
:106B300018D20020F0B50446002089B0C4E9220034
:106B40000E9D04F19000C4E9240004F19800C4E90A
:106B500026004DB32879002840F2011008BF01201B
:106B6000C4F8A00000204FF0FF364FF0FF37CDE90A
:106B70000330CDE90100CDE9066720460B4B0094B8
:106B800000F0AAF855B1296811B1204606F0B1FF0E
:106B90006B791BB1237B43F001032373204609B0BB
:106BA000BDE8F04006F0AABF0120D9E73169020034
:106BB00037B501900846EFF31184202181F3128844
:106BC000BFF36F8FC16811F01E0F16D153EA020593
:106BD00008D101A9FFF74EFF84F31188BFF36F8F2F
:106BE00003B030BD41F00801C160019910308161EE
:106BF000034900F03DFC0120EEE70020ECE700BF78
:106C000045DA020001460148FFF7D2BF18D2002042
:106C1000F7B50C4616461D460190EFF31187202369
:106C200083F31288BFF36F8F084606F0F5FE55EA2E
:106C3000060309D1204601A9FFF71CFF87F311883D
:106C4000BFF36F8F03B0F0BDE36804F1100043F0B1
:106C50000803E360019B3246A36203492B4600F020
:106C600007FC0120EAE700BF45DA020001460148BF
:106C7000FFF7CEBF18D200202DE9FF410E9E00F194
:106C8000580506730426C0E91655002504464673C8
:106C90000D9EC0E906558673D61D0C9A26F0070690
:106CA000C0E91A168560C573056702920B9A01EB5D
:106CB000060801920A9A00924246F6F7A7F8054B99
:106CC00065659B6803B15B6F4046636704B0BDE8D0
:106CD000F08100BFF4DC0020F0B5002587B00595F9
:106CE000109DDDE9127604950F9D044603950E9DD7
:106CF00002950D9D01950C9D0095FFF7BDFFB6F126
:106D0000FF3F08BFB7F1FF3F05D056EA070305D1A3
:106D1000204600F0A1F9204607B0F0BD3A463346C0
:106D2000024904F1180000F0A3FBF4E73DDC020087
:106D300038B50D4D2B4653F8184F9C4200D004B97E
:106D4000EC68AB6838B95A7BD20604D1A26912B993
:106D5000DA897F2A05D89C4202D0204600F0D0FA7A
:106D600023466B6138BD00BFF4DC002008B590F904
:106D70000D200146002A437B04DA03F07F034373AE
:106D800006F0BEFE044B9868431A58425841BDE8CD
:106D90000840FFF7CDBF00BFF4DC002070B490F9CD
:106DA0000D30427B002B29DBD30627D183692BBB17
:106DB000134962F07F0242730A4652F8184F944218
:106DC00018BF2346CC6923B9C0E900242060C861FC
:106DD0000CE090F90E5093F90E60B5420AD0AE4225
:106DE00008DD5A68C0E9003210605860002070BCAD
:106DF000FFF79EBF9C42E7D01B68E4E770BC70477A
:106E0000F4DC0020002A2DE9F0410E460CBF1021D1
:106E10000821427B044611420FD141EA0203D20904
:106E200018D1437308291BD00120FFF781FFBFF35E
:106E30005F8F637B23F060036373274B9B68A342E0
:106E400043D1EFF30583002B3FD13046BDE8F0413D
:106E5000F5F70CBF03F07F03437306F051FEE1E743
:106E6000A36813B1204606F053FE04F1180006F0A3
:106E700085FF4FF0000804F15807A56DBD4200D012
:106E8000B5B9154FBB689C42CED1EFF30583002BFB
:106E9000CAD00120FFF74CFF40F201130F4DAB8128
:106EA00000232846C5E91A3300F00EFDBD60BEE799
:106EB000284606F02DFE05F1180006F05FFF284673
:106EC000C5F87C80FFF76AFFD7E786F31188BFF328
:106ED0006F8FBDE8F08100BFF4DC0020C0D200203D
:106EE00070B590F90D200146002A437B04DA03F0C7
:106EF0007F03437306F004FE154A4B7B104663F094
:106F00007F034B7350F8183FD469834208BF0023B6
:106F100023B9C1E900042160D1610CE091F90E5060
:106F200093F90E60B5420ED0AE420CDD5868C1E94F
:106F30000030016059609068BDE87040431A5842C3
:106F40005841FFF7F5BE9C42E3D01B68E0E700BF65
:106F5000F4DC0020F8B5124B0C46DDE9067611464C
:106F60009868104A1060EFF31182202282F3128891
:106F7000BFF36F8F9D68284606F0D4FDB6F1FF3F42
:106F800008BFB7F1FF3F06D03A463346064905F140
:106F9000180000F06DFA2046BDE8F840F5F766BE2F
:106FA000F4DC00201CDD00203DDC0200F8B50446C6
:106FB000EFF31186202383F31288BFF36F8F437B97
:106FC00049B2DA0619D18569BDB903F07F0343736D
:106FD00006F096FD437B164A63F07F034373134626
:106FE000817353F8180F984218BF0546D0695DB9F0
:106FF000C4E900300460D46111E00020A17386F37D
:107000001188BFF36F8FF8BD95F90E70B9420BD0A0
:107010008F4209DD6B68C4E900531C606C6001207D
:10702000FFF786FE0120EAE7A842E1D02D68DEE7FF
:10703000F4DC002049B9EFF3058030B9054B5A69FB
:107040009B689A4201D0F5F711BE81F31188BFF316
:107050006F8F7047F4DC002010B5EFF3118420220D
:1070600082F31288BFF36F8F427B510704D484F3FD
:107070001188BFF36F8F10BD22F004024273FFF737
:107080008DFE2146BDE810400148FFF7D3BF00BF89
:1070900065E40020034648B9EFF3058232B9064A99
:1070A00051699268914201D0F5F7E0BD83F31188F0
:1070B000BFF36F8F704700BFF4DC0020EFF3118146
:1070C000202383F31288BFF36F8F054B9A68D37B1D
:1070D000013BD37381F31188BFF36F8F704700BFFB
:1070E000F4DC002038B5EFF31185202484F31288F6
:1070F000BFF36F8F0A4B00209A68D37B0133D373A1
:10710000FFF716FE85F31188BFF36F8FEFF3118041
:1071100084F31288BFF36F8FBDE83840FFF7BABF22
:10712000F4DC0020024B03F11802C3E90622704789
:10713000F4DC0020F8B5EFF31185202383F31288E7
:10714000BFF36F8F19498868437B03F07F03437354
:1071500006F0D6FC08468B685A7B62F07F025A73B1
:1071600050F8182FCC69824208BF002222B9C3E927
:1071700000042360CB610CE093F90E6092F90E706D
:10718000BE420ED0B7420CDD5168C3E900210B604E
:1071900053600120FFF7CCFD2846BDE8F840F5F725
:1071A00065BDA242E3D01268E0E700BFF4DC002036
:1071B00050EA01032DE9F04105460E4603D1FFF7E1
:1071C000B9FF00202BE0831C71F1FF3329DB06F0AF
:1071D000EAFD2C18EFF31188202383F31288BFF304
:1071E0006F8F124F124BB8681860FFF7BFFDB86879
:1071F00010492A463346183000F03AF9BA6840463A
:10720000537B43F010035373F5F730FD06F0CBFDCD
:10721000201A63EB0303012873F10003D1DBBDE8FF
:10722000F0816FF00104241AD4E700BFF4DC0020E1
:107230001CDD00203DDC0200B1F1FF3F08BFB0F1D2
:10724000FF3F08B506D10A4B986806F0ABFC4FF03B
:10725000FF3008BDFFF7ACFF4FF47A7147F6FF73BC
:107260000022C0FB0132D80B40EA4240F1E700BFE8
:10727000F4DC0020014B9868704700BFF4DC00206C
:10728000D3B5DDE90667089CCDE90067FFF762FE2C
:107290001CB1034B9B685B69236002B0D0BD00BF8B
:1072A000F4DC00200122044BC01A044BC0105843E8
:1072B000034B1A54704700BF48D30020ABAAAAAAB8
:1072C00065E40020C3897F2B12D80A4B1B6863B189
:1072D000094B90F90E201B689A4209DB437BDB06C1
:1072E00006D1064BC31A18BF012303F001007047F3
:1072F0000023FAE724DD002020DD002008D1002053
:1073000070B50E4B0E4C1E7C054606EB460304EB97
:10731000C304204606F032FD00220A4B28469A5547
:10732000FFF7D0FF48B1084B2046BDE870401A680F
:107330000649013AD31700F09BB870BDF4DC002079
:1073400048D3002065E4002024DD0020A57202005F
:1073500038B5EFF31185202383F31288BFF36F8FC5
:10736000104B114A9C681068A04206D1FFF7C8FF75
:1073700085F31188BFF36F8F38BD00211B7C11602E
:107380000A4AD35C002BF3D02046FFF79BFF00286E
:10739000EED0637BDB0602D12046FFF7A1FD20463D
:1073A000E4E700BFF4DC00201CDD002065E40020E1
:1073B00008B50648064A0749121A06F00BFABDE856
:1073C0000840054A0549064806F004BA80C5002071
:1073D00030CA0020641F0300000000004C1F03009F
:1073E00080C50020034B1B680BB9F8F7C7B9002014
:1073F000704700BF28DD002030B570B10B4B5B68D3
:1074000098420AD0036843B1D3E90421D0E9044586
:10741000121941EB0501C3E90421D0E900321360E0
:107420005A600023C0E9003330BD00BF38C70020D8
:1074300010B50E4B1C689C4204D1FFF7D3FF6FF0D0
:10744000004010BDFFF7CEFF002CF8D0D4E9043285
:107450001B1A62EBE072B3F1004F72F10001EEDA39
:10746000002AACBF18460020EBE700BF38C7002059
:10747000B3F1FF3F08BFB2F1FF3FF8B504461D4628
:1074800016465ED08160EFF31187202383F31288C4
:10749000BFF36F8F013275F1FF3324DA6FF0010310
:1074A0002D49D1E900209B1A4FF0FF3262EB00001A
:1074B0009E1B60EB0500012E70F1000301DA01262E
:1074C0000020C4E90460254ED6F800C07568B445B4
:1074D00008BF4FF0000CBCF1000F0DD1C4E90065EE
:1074E0002C6074601CE0FFF77DFF013645F100055C
:1074F000361845EBE070E4E7DCE90420D4E9043118
:10750000934271EB000E1DDAD21ADCF8043060EB06
:107510000100CCE90420C4E900C31C60CCF804409D
:107520003368B34209D09C4207D10D4B1C6824B983
:10753000FFF77EFF2146F8F7F3F887F31188BFF3D2
:107540006F8FF8BD9B1A61EB0001AC45C4E90431B3
:10755000C4D0DCF800C0BEE760D3002038C70020EC
:1075600028DD00202DE9F84FEFF3118C202383F361
:107570001288BFF36F8FDFF8B0A0DFF8B09000245F
:10758000C9F80000DAF800000025504508BF0020C7
:10759000274FE046D7E90021D9F8003078B3D0E989
:1075A000046C4FEAE37EB3427EEB0C0B05DAF61A6D
:1075B0006CEB0E04C0E9046421E0B21841EBE67103
:1075C000C0E90445C7E90021FFF716FF88F31188D9
:1075D000BFF36F8F83689847EFF31188202383F3FD
:1075E0001288BFF36F8FD9F80030DAF800009B1BC8
:1075F0005045C446C9F80030CBD1D7E9002100245A
:107600009A1841EBE373C7E90023C9F80040FFF77C
:107610000FFF2146F8F784F888F31188BFF36F8FC6
:10762000BDE8F84FFFF794BE38C7002028DD0020E2
:1076300060D3002010B5EFF31184202383F3128868
:10764000BFF36F8FFFF7CEFE0346054AD2E9000174
:10765000181841EBE37184F31188BFF36F8F10BDED
:1076600060D30020F8B50446EFF31187202383F39D
:107670001288BFF36F8F026822B187F31188BFF3BE
:107680006F8FF8BDD0E90A36581C46F10001022878
:1076900071F1000127D3012B76F10001BCBF01235A
:1076A00016465D1E46F1FF3606F081FB013041F1C2
:1076B0000001401946EB0101012871F1000139DB9D
:1076C00006F075FB013041F100016FF00102401935
:1076D00046EB01034FF0FF31121A61EB0303204622
:1076E0001749FFF7C5FE236B01332363236A6BB190
:1076F00087F31188BFF36F8F2046236A9847EFF313
:107700001187202383F31288BFF36F8F54F8185F1B
:10771000A542B2D0002DB0D0284606F05DFA002375
:10772000EB6787F31188BFF36F8F2846BDE8F840F9
:1077300006F029BA6FF001024FF0FF33CFE700BF28
:10774000657602002DE9F04105461C4690461F462D
:10775000EFF31186202383F31288BFF36F8FB4F108
:10776000FF3F08BFB2F1FF3F05D186F31188BFF399
:107770006F8FBDE8F081531C74F1FF3309DB012AE0
:1077800074F10003BCBF0122002412F1FF3844F160
:10779000FF37284606F0F2FADDE906010023C5E9C5
:1077A0000A012B6342463B4628460249FFF760FE2A
:1077B000DBE700BF657602002DE9F74F1D46274B3A
:1077C00016469F68012387F8603087F8613052EAD7
:1077D00005030CBF0123002307F16002804606F079
:1077E000B4FB8146EFF3118B4FF0200A8AF3128825
:1077F000BFF36F8F97F860404CB901465A46404638
:1078000006F044FB8BF31188BFF36F8F0BE000236E
:1078100087F8603056EA050309D18BF31188BFF36E
:107820006F8F6FF00A04204603B0BDE8F08F594611
:10783000CDE900650A4A0B48FFF78CFB0446EFF3DD
:1078400011858AF31288BFF36F8F2A464946404656
:1078500006F01CFB85F31188D6E700BFF4DC00209E
:1078600040C7002066E4002038B50346EFF31185D9
:10787000202282F31288BFF36F8FC16001218160E3
:107880000068834206D185F31188BFF36F8F00240F
:10789000204638BDD0E9003213605A600023C0E9A9
:1078A000003306F0CAFB294604460248FFF7C2FB34
:1078B000EEE700BF66E400200A460146014806F0F4
:1078C00035BC00BF80C80020014B4367704700BF34
:1078D00080C8002038B504460D4606F004F920B9EA
:1078E000064B9B685B6F0BB938BD054B2A4621469A
:1078F0001846BDE8384006F019BC00BFF4DC002093
:1079000080C80020F8B504460D46F2F719F9174B68
:1079100006460F4693F9003001331AD022462B4613
:1079200020462946F1F73AFC98B900220023204668
:107930002946F1F729FC60B9002200232046294698
:10794000F1F7FAFB40B102F028F900262223084F94
:10795000036030463946F8BD02F01FF92123036069
:107960000448BDE8F84000F0A9B800BFCBC700202C
:107970000000F0FFBA19030070B506460D4600F08E
:107980001DF80D4B044693F90030013312D02946FF
:107990003046F1F741FC68B900212846F1F7B4FA06
:1079A00040B102F0FAF82123002103600846F1F704
:1079B000CBF90446204670BDCBC70020F8B521F0B6
:1079C00000450E466B1EB3F1FF4F05D220F0004775
:1079D0000346B7F1FF4F05D3F1F702F90146F1F77E
:1079E000B3F9F8BDAF42FCDB00F0004404D1E40F72
:1079F000314B53F82400F4E710F0FF4F3FD13A0227
:107A00006FF07D01002A37DC16F0FF4F3DD12802D0
:107A10006FF07D02002835DA11F17E0FB5BF6FF0EF
:107A20007D03C3F316035B1A43F40003A1EB0201C9
:107A3000B8BF07FA03F312F17E0FB5BF6FF07D00F8
:107A4000C6F31606801A46F40005B8BF8540581BD9
:107A5000F1B913EA200338BF0346002BC7D0B3F5B2
:107A6000000F1DDB12F17E0F1DDBA3F500007F323E
:107A7000204340EAC250B4E701395200C2E7F91589
:107A80007F39C1E7013A4000C4E7EA157F3AC3E70E
:107A9000002802DA5B000139D9E7A8D04300FAE7F1
:107AA0005B00013ADBE7C2F1FF2202F57F0282327E
:107AB00043FA02F0204394E78CF4020000200149CD
:107AC000704700BF0000F87F38B50546002941D057
:107AD00051F8043C0C1F002BB8BFE41800F0DCFA8E
:107AE0001D4A136833B9636014602846BDE8384006
:107AF00000F0D8BAA34208D9206821188B4201BFF0
:107B000019685B6809182160EDE71A465B680BB1DC
:107B1000A342FAD911685018A0420BD12068014441
:107B2000501811608342E0D118685B6808445360C4
:107B30001060DAE702D90C232B60D6E72068211801
:107B40008B4202BF19685B680918636008BF216037
:107B50005460CAE738BD00BF30DD0020F8B5CD1C49
:107B6000064625F0030508350C2D38BF0C25002DE1
:107B700001DBA94203D90C2333600020F8BD00F0DB
:107B80008BFA21490A6814469CB9204F3B6823B9F7
:107B90002146304600F03CF838602946304600F077
:107BA00037F8431C23D10C233046336000F07AFAB7
:107BB000E3E723685B1B17D40B2B03D923601C441A
:107BC000256004E06368A2420CBF0B60536030463E
:107BD00000F068FA04F10B00231D20F00700C21A20
:107BE0001CBF1B1AA350C9E722466468CCE7C41C1B
:107BF00024F00304A042E3D0211A304600F008F834
:107C00000130DDD1CFE700BF30DD00202CDD0020CA
:107C100038B50023054D044608462B60F5F76CFB8C
:107C2000431C02D12B6803B1236038BD34DD002032
:107C30000CB4184B30B50C1E9DB01D6808DA8B23B0
:107C40004FF0FF302B601DB0BDE8304002B07047F0
:107C50004FF402730290069002A9ADF8143014BFDD
:107C600004F1FF332346209A2846049307934FF6E6
:107C7000FF73ADF8163021AB019300F019FA431CE5
:107C8000BCBF8B232B60002CDDD0029B00221A701E
:107C9000D9E700BF48C7002070B50A4405460E4E1C
:107CA000914201D1002011E015F8013B11F8014B80
:107CB000F05C00F003000128305D00F0030008BF15
:107CC0002033012803D12034181BE9D070BD181BC4
:107CD000FCD1002CE4D1F9E7D91D0300242B2DE9B8
:107CE000F0478646904601D8012B06D101F055FF9A
:107CF000162303600020BDE8F0870D4635482A466C
:107D000015F8014B065D16F00806F8D12D2C24D18C
:107D10002C780126951C2BBB302C30D00A2306F181
:107D2000004C00220CF1FF3C1046BCFBF3F903FBB6
:107D300019CAA4F13007092F28D83C46A34234DDE4
:107D4000571C07D081452DD301D1A2452ADB00FB6A
:107D50000340012215F8014BEBE72B2C04BF2C78D4
:107D6000951CD8E7102BDAD1302CD8D12A7802F024
:107D7000DF02582AD3D16C7810230235CFE72B7855
:107D800003F0DF03582BF6D00823C8E7A4F141071E
:107D9000192F01D8373CD1E7A4F16107192F04D876
:107DA000573CCBE74FF0FF32D4E7531C08D12223D6
:107DB0006046CEF80030B8F1000F9CD0691E06E096
:107DC00006B14042B8F1000F95D0002AF6D1C8F8AC
:107DD000001090E7D91D030013460A4601460248E9
:107DE0000068FFF77BBF00BF48C700202DE9F04FB8
:107DF000904685B089461E460D46454A02902B4660
:107E000015F8014B175D17F00807F8D12D2C41D15B
:107E10002C7801279D1C002E41D1302C4CD00A26F5
:107E200007F1004A07F1FF3BF31732460AF1FF3A28
:107E3000584603935146F1F70FF9019200228E46FE
:107E4000844611461046A4F13003092B05D9A4F14C
:107E50004103192B37D8A4F137039E423DDD541C52
:107E600015D084457EEB010234D38E4508BF84458E
:107E700002D1019A9A422DDB039A714300FB021151
:107E8000A6FB00020A44181842EBE371012215F820
:107E9000014BD8E72B2C04BF2C789D1CBBE7102E80
:107EA000BED1302CBCD12B7803F0DF03582BB7D1D7
:107EB0006C7810260235B3E72B7803F0DF03582BDC
:107EC000F6D00826ACE7A4F16103192B05D8A4F17C
:107ED0005703C2E74FF0FF32D9E7531C0AD12223E0
:107EE000029A584651461360B8F1000F0AD105B006
:107EF000BDE8F08F17B1404261EB4101B8F1000FCE
:107F0000F5D00AB105F1FF39C8F80090EFE700BFDE
:107F1000D91D030013460A46014602480068FFF7D0
:107F200065BF00BF48C700202DE9F04386460D46D7
:107F3000354E284615F8014B375D17F00807F8D184
:107F40002D2C26D12C780127851C3BBB302C32D020
:107F50000A234FF0FF380026B8FBF3F803FB08F9BB
:107F600030466FEA0909A4F1300CBCF1090F29D899
:107F70006446A34237DDB6F1FF3F07D080452FD3DB
:107F800001D1A1452CDB00FB0340012615F8014B74
:107F9000E9E72B2C04BF2C78851CD6E7102BD8D111
:107FA000302CD6D1287800F0DF005828D1D16C7859
:107FB00010230235CDE72B7803F0DF03582BF6D0E2
:107FC0000823C6E7A4F1410CBCF1190F01D8373CD6
:107FD000CFE7A4F1610CBCF1190F04D8573CC8E7F6
:107FE0004FF0FF36D2E7731C06D122233046CEF87D
:107FF000003032B9BDE8F08307B14042002AF9D021
:1080000006B1691E1160F5E7D91D030013460A4643
:10801000014602480068FFF787BF00BF48C700203D
:1080200007B5009313460A4601460348006806F068
:1080300047F903B05DF804FB48C7002070B51E4641
:108040009AB04FF40173044608461546ADF80C305B
:1080500000910491F1F74EFA094B2A4669460190C6
:1080600009930023059020460D9312934FF6FF735A
:10807000ADF80E30334600F017F91AB070BD00BFEE
:10808000FDE1020013460A46014602480068FFF778
:10809000D5BF00BF48C70020014801F076BD00BF32
:1080A000A8C80020014801F076BD00BFA8C8002084
:1080B0002DE9F04F98468B899DB007461B060D466B
:1080C000144610D50B6973B94021FFF747FD2860AE
:1080D000286130B90C233B604FF0FF301DB0BDE884
:1080E000F08F40236B610023CDF80C804FF0010925
:1080F000DFF8A081099320238DF8293030238DF8F3
:108100002A3023469A4613F8012B0AB1252AF9D1C1
:10811000BAEB040B0BD05B4622462946384606F0E4
:10812000FAF8013000F0A780099A5A4409929AF8A7
:108130000030002B00F09F8000234FF0FF320AF147
:10814000010A049307938DF853301A93CDE9052360
:10815000544605224F4814F8011B06F01CF8049AF7
:10816000D8B9D00644BF20238DF85330110744BF3F
:108170002B238DF853309AF800302A2B15D0079A0C
:10818000544600204FF00A0C214611F8013B303BC9
:10819000092B4BD9B0B1079214E0A0EB0803A2461B
:1081A00009FA03F313430493D2E7039B191D1B68D9
:1081B000002B0391BBBF5B4242F00202079307937F
:1081C000B8BF049223782E2B0AD163782A2B32D1A0
:1081D000039B02341A1D1B6843EAE3730392059361
:1081E000DFF8B4A003222178504605F0D4FF38B15F
:1081F000A0EB0A004022049B013482401343049305
:1082000014F8011B062225488DF8281005F0C3FF3D
:10821000002836D0224B1BBB039B073323F00703F8
:1082200008330393099B334409936AE70CFB02323A
:108230000C460120A8E7002301344FF00A0C194630
:108240000593204610F8012B303A092A03D9002B58
:10825000C6D00591C4E70CFB012104460123F0E7D9
:1082600003AB2A4604A9384600930E4BAFF30080B7
:10827000421C0646D6D1AB895B063FF52DAF099867
:108280002CE703AB2A4604A938460093054B00F0BF
:1082900083F9EDE7D91E0300DF1E0300E31E030090
:1082A0000000000017E302002DE9F0470C46ADF591
:1082B000227D002106460DF10408A74F0093CDF85A
:1082C0001881CDE94411A549A091A549A191137840
:1082D000002B00F05C81F95C551C11F0080119D0ED
:1082E0006368002B0FDD23681A78BA5C120701D48B
:1082F0002A46ECE7459A01330132236045926268D1
:10830000013A6260ECE7A19B21463046984700287D
:10831000E9D0EDE7252B12D099466368002B40F396
:108320009480226813784B4540F0318163680132B4
:10833000013B22606360459B01334593D8E741913F
:10834000439153782A2B04BF1023951C4FF00A0247
:1083500008BF4193A94619F8011BA1F13003092B6D
:108360001ED9DFF800A20322504605F014FF38B1F1
:10837000A0EB0A000123419A4D46834013434193E9
:1083800015F8013B782B06D8572B10D8252BC3D0D6
:1083900056D8002B64D0032347930A2342936AE004
:1083A000439B4D4602FB031130394391D2E7A3F1C1
:1083B0005802202AEFD801A151F822F0AB84020024
:1083C0009783020097830200CD8402009783020006
:1083D000978302009783020097830200978302002D
:1083E0009783020097830200E3840200C98402009D
:1083F00047840200478402004784020097830200FA
:10840000BD840200978302009783020097830200D5
:1084100097830200F3840200C5840200678402008F
:108420009783020097830200EF8402009783020083
:10843000C98402009783020097830200AB84020084
:10844000453B022BA7D8052314E0A19B21463046CB
:10845000984700283FF465AF4498002840F08F808B
:108460004FF0FF308FE0419B43F40873419310239A
:108470004293042347936368002B4ADD419B5906CE
:1084800004D423681A78BA5C120749D4479B022B9C
:1084900058DC6B46224641A9304600F0ABF9012872
:1084A00075D002287FF424AFD6E7419A42F40072D7
:1084B000419210226E2B429202D9DAE700234293B6
:1084C0000323D7E70823D3E70A22F3E729464046E8
:1084D00006F046F8419B054643F0400341930123D3
:1084E000C8E7419B43F0400341930023C2E70223C6
:1084F000C0E74198C3063FF5FBAE009B10F0010FAB
:10850000459A03F1040100911B6814BF1A801A6098
:10851000EEE6A19B2146304698470028AED09BE767
:10852000459A013245926268013A002A626002DD92
:1085300001332360A5E7A19B2146304698470028D8
:108540009FD089E7042B0FDC6B46224641A93046B9
:1085500000F0AAF9A3E700BFD91D0300CDE3020094
:1085600043E40200DF1E03000A4B002B3FF4C0AEC1
:108570006B46224641A93046AFF300808FE7A389BE
:108580005B063FF56DAF0DF5227DBDE8F0874498A1
:10859000F9E700BF000000002DE9FF470F7E91467C
:1085A00080460C46782F9A460C9D01F1430207D86D
:1085B000622F0AD8002F00F0E080582F00F0BB8017
:1085C00004F1420684F842703AE0A7F16303152BE8
:1085D000F6D801A151F823F0318602004586020049
:1085E000C1850200C1850200C1850200C18502006B
:1085F00045860200C1850200C1850200C1850200D6
:10860000C185020061870200D5860200178702003B
:10861000C1850200C185020083870200C185020076
:10862000D5860200C1850200C18502001F870200B5
:108630002B6804F142061A1D1B682A6084F8423038
:108640000123ABE0236829681F0601F104002860BC
:1086500001D50D6803E05E06FBD5B1F90050002D91
:1086600061687ADA2D200029A16084F843002DDAB0
:108670006D425E480A231646B5FBF3F103FB115722
:10868000C75D06F8017D2F460D46BB42F4D9082B85
:108690000BD12368DF0708D5236961689942DEBFE3
:1086A000302306F8013C06F1FF36921B22614B464F
:1086B00003AA21464046CDF800A005F0DFFE0130B8
:1086C00071D14FF0FF3004B0BDE8F08723F0040310
:1086D0002360CDE72B682068191D2960050601D5A8
:1086E0001D6802E04106FBD51D886F2F3F4814BF6F
:1086F0000A230823002184F843106668002EA66030
:10870000B9DB216821F004012160002DB3D1002ED6
:10871000B1D11646BBE7236843F0200323607827D6
:10872000334884F84570296823680E1D2E601E06A4
:1087300003D50D6804E02D48F3E75D06F9D50D88F3
:10874000D90744BF43F0200323600DB11023D1E7C4
:10875000236823F020032360F8E724480A23CCE7AA
:108760002B682668181D6169286035061B6801D5CD
:10877000196002E07006FBD51980002316462361BC
:1087800095E72B6800211A1D2A601E686268304632
:1087900005F001FD08B1801B606063682361002360
:1087A00084F8433083E72369324649464046D04740
:1087B000013086D023689B0714D4E068039B98425D
:1087C000B8BF18467FE70123324649464046D047A6
:1087D00001303FF476AF0135E36803995B1AAB4291
:1087E000F1DCEAE7002504F11906F5E7EA1E0300CB
:1087F000FB1E03002DE9F84315468A6880460C46A7
:1088000032B98A69002A14BF4FF0FF3201228A6010
:1088100022680027DFF88C90D1065FBF1A68111D0F
:1088200019601668A06988B1012807D12B681A78E9
:1088300063699B5C53B9002F31D022E0022820D11C
:108840002B681B7819F803301B071AD423680137EB
:10885000DA065EBF2B681B7806F8013B2A686B6856
:108860000132013B2A60A2686B60013AA26042B10A
:10887000002BD7DCD4F880312946404698470028A1
:10888000D0D0236813F0100305D1E2680132E26012
:10889000A26902B13370236900203B442361BDE823
:1088A000F88300BFD91D03002DE9F04F984687B02B
:1088B000784B0C468246164627464FF0000B93E84D
:1088C000070003AB83E80700734BA169734A0329D0
:1088D00008BF1A46A36801925A1EB2F5AE7F89BF3F
:1088E0006FF4AE754FF0000903EB050940F25D131C
:1088F00088BFA36057F81C3B43F450633D46236098
:10890000316803AB0222097853F82B0005F043FCD1
:10891000002840D0BBF1010F12D162682AB9226849
:10892000082142F4007261602260226822F4A06291
:108930002260A268511EA160DAB94FF0020BDFE796
:10894000BBF1020F06D0A268511EA1608AB94FF098
:10895000010BD5E7226802F4C061B1F5007F1FD199
:1089600042F4807210212260A2686160511EA160F1
:10897000B2B13268511C3160127805F8012B72686F
:10898000013A002A726006DCD4F880213146504654
:108990009047002874D10BF1010BBBF1030FAFD14D
:1089A00063680BB90A23636063684FF0000B3C49AE
:1089B0006069C91A05F0D4FDA368226873B33168F1
:1089C000606991F800C010F80C0038B3BCF1300FAA
:1089D00016D1100514D50BF1010BB9F1000F03D01E
:1089E000013309F1FF39A3607368013B002B736009
:1089F0000DDD336801333360A368013BA360DBE71F
:108A000022F4106222600B7805F8013BECE7D4F801
:108A100080313146504698470028EDD02368D9056B
:108A20000DD5BD4209D905F1FF3915F8011CD4F85F
:108A30007C3132464D4650469847BD4228D0226888
:108A400012F0100213D12A70394663685046019E15
:108A5000B047D8F8003021681A1D11F0200FC8F86F
:108A600000201B680FD01860E3680133E360ED1B42
:108A7000236900205D442B44236107B0BDE8F08FDB
:108A80004FF0000BCAE7CA074CBF18801860EBE72D
:108A90000120F2E7BCEB0200B9E20200BDE20200F5
:108AA0001C1F0300704700F053BF034690F82400DA
:108AB00020B99B6A0B6001238B8070476FF08500A3
:108AC000704700F03CBF00F043BF012903D1C3074A
:108AD00001D5F1F729BC7047836800EBC101B3F5FC
:108AE000004F2CBF51F8220031F81200704700EB04
:108AF000C1018068B0F5004F2CBF41F8223021F849
:108B000012307047012208B5FFF7E6FFD04008BDDC
:108B1000836800EBC101B3F5004F08D34B681AB16D
:108B200043F001034B60704723F00103FAE74B88E1
:108B30001AB143F001034B80704723F00103FAE7B9
:108B400053000122FFF7D3BF8368B3F5004F34BF52
:108B500004230823C91A081AC0087047B0F5004F4B
:108B600034BF04230823481C0833A0EBD300B0FA19
:108B700080F0C0F11F0070472DE9F0411746032235
:108B80000E460446FFF7A8FF8642054607F1040893
:108B90000AD10122E368BA4023EA0203E36000231A
:108BA00044F82830BDE8F081314602222046FFF724
:108BB00093FF06462B4601460322204644F82850E0
:108BC000FFF795FF334629462046BDE8F0410222D3
:108BD000FFF78DBF70B50D4686680446FFF792FF1C
:108BE000B6F5004F014601D3012809D03046FFF702
:108BF000B5FF294602462046BDE87040FFF7BCBFDE
:108C000070BD2DE9F04705468068FFF7A7FF05EB2B
:108C1000800ADAF8109088460646B9F1000F1BD09A
:108C20000327DAF8104028462146FFF76BFF40453E
:108C300007D3324621462846FFF79EFF2046BDE86F
:108C4000F087032221462846FFF746FF013FCAF876
:108C5000100001D08145E4D14FF0FF34EB680136BC
:108C6000B4401C40EAD094FAA4F2B2FA82F2131D86
:108C700055F82340DEE72DE9F04114460E4605463F
:108C8000FFF740FFA4EB0608371B07444246314676
:108C90002846FFF755FF3A4621462846FFF750FF82
:108CA0004346002221462846FFF721FF2146284659
:108CB000FFF728FF3B46211800222846BDE8F04177
:108CC000FFF715BF2DE9F041164604460F46FFF7A2
:108CD00019FF314605462046FFF714FF05442A4692
:108CE00039462046FFF72CFF31462046FFF70AFFA2
:108CF0002B46311800222046BDE8F041FFF7F7BEB1
:108D00002DE9F0410D4686680446FFF7FBFEB6F5F7
:108D1000004F014601D3012832D03046FFF71EFF35
:108D200004EB80010E6996B90122E3688240134387
:108D3000E36002220D612B4629462046FFF7D7FE4D
:108D4000032229462046BDE8F041FFF7D0BE0222AB
:108D500031462046FFF7C0FE074603462946204617
:108D6000FFF7C5FE0322334629462046FFF7BFFE24
:108D700039462B462046FFF7BAFE02223146E1E78C
:108D8000BDE8F081F8B50C460546FFF7BBFE261896
:108D9000012231462846FFF79FFEC3070CD4314617
:108DA0002846FFF717FF21462846FFF7ABFE21466E
:108DB00022182846FFF786FF002221462846FFF7A3
:108DC0008BFE271A012239462846FFF785FE10EA56
:108DD000020613D139462846FFF7FCFE21463246EB
:108DE0002846FFF779FE2246211A2846FFF76AFF38
:108DF000214632462846FFF76FFE241A21462846B0
:108E0000BDE8F840FFF77CBF38B571B105680022B6
:108E10002846FFF799FE044601462846FFF778FEEC
:108E20002146BDE83840FFF7ADBF38BD70B50668D4
:108E300009B9002070BDB368B3EBD10FF9D9B3F510
:108E4000004F34BF04230823CC1D1C44E4082146F2
:108E50003046FFF7D6FE05460028EAD001463046E8
:108E6000FFF750FEA04209D92C442946304622463D
:108E7000FFF701FF21463046FFF742FF304601224F
:108E80002946FFF745FEB368B3F5004F34BF04230E
:108E9000082303EBC5031844CCE72DE9F843066823
:108EA0001446B26801F1FF39B2F5004F34BF042314
:108EB000082319EA01090F460BD0494239408B4279
:108EC0004F4628BF0B46894654B900252846BDE8C1
:108ED000F8839942F8D82146BDE8F843FFF7A6BFCA
:108EE000B2EBD40FF1D9B2F5004F34BF04220822FF
:108EF000E11D3944C91A11443046C908FFF781FE03
:108F000080460028E1D0B36809EBC005B3F5004FF7
:108F100034BF042308231D4435447B1E1D44B5FB88
:108F2000F7F57D43A5EB090529463046FFF70CFE12
:108F30002C44073424F00704A41B804507464FEA5D
:108F4000E40408D2024641463046FFF794FE41460B
:108F50003046FFF7D5FE39463046FFF7D3FD38449B
:108F6000844208D2394630462246FFF784FE214625
:108F70003046FFF7C5FE012239463046FFF7C8FDEF
:108F8000A4E7B2F5802F2CBF082304232DE9F0417C
:108F90000026D21A8C18CD1D25F0070524F00704F1
:108FA000641BE408056021462046AC60EE60FFF7D4
:108FB000D5FD421D9200013002F107074FEAD707A5
:108FC0003146A2F1100205F11000B8BF324605F09B
:108FD0000DF93A4631462846FFF7B2FD3346324690
:108FE00031462846FFF783FDA4EB070828463146A3
:108FF0000122FFF78DFD42463946FFF7A1FD3B46B2
:10900000324639462846FFF772FD21462846FFF7CB
:1090100097FD4346324621462846FFF768FD214624
:1090200028460122FFF774FD3946BDE8F041FFF7FD
:1090300067BE2DE9F04706460D46174698462BB306
:109040004FF0000A98F8004093F80190DB78A400F4
:1090500004EB430498F802301C444444CA4509D345
:1090600039463046AC46D8F8042008F10803BDE87C
:10907000F047604714F8013B0AF1010A204648F81E
:109080002340F0F737FA01300444E7E76FF01500AA
:10909000BDE8F08770B5002502462846144614F84E
:1090A000013B0BB9184609E098B18D4207D1702BEE
:1090B00004D0A3F140023A2A0BD8002070BDA3F1DE
:1090C00040063A2E05D853780135941C002BE9D080
:1090D0000020252B224608BF80F00100DEE700209B
:1090E000704730B58A680C68551C14B14B689342C0
:1090F00001DC8D6030BD013B934208BF00228D60D2
:109100000CBFE254A054F5E70FB407B504A951F819
:10911000040B019100F09AFB03B05DF804EB04B07E
:1091200070470CB407B504AB53F8042B0193F1F767
:109130004DFF03B05DF804EB02B07047044608B57C
:10914000084611461A46A047FEF794F8F3F778FD53
:109150000CB4034607B5084605AA40F20511DB68C2
:109160000192984703B05DF804EB02B070472DE917
:10917000F0410746884615461E461446B44205D3BC
:109180000EB1601B08E02378002BFAD0414614F89A
:10919000010BB8470028F1DABDE8F08110B503698A
:1091A000024613F0080009D11368D4689C429BBFA3
:1091B0000120126AE31AD31A0B6010BD002318466F
:1091C000FAE713B501A90446FFF7E8FF20B1019BB8
:1091D000E268013B13440193206A019BC01A0138E5
:1091E00002B010BD10B5044650182269236AD20798
:1091F00002D5013B184010BD984228BFC01AFAE7BB
:1092000010B504460A46C168FFF7ECFF2369E06029
:1092100023F00803236110BD38B50D46C2698B00E9
:10922000016843F00203044642F8213001682A46EF
:10923000FFF7D8FFE3686168984208BF23692060A0
:1092400008BF43F008032A46204608BF2361FFF702
:10925000C9FF606038BD2DE9F74FC768C6699B46F6
:1092600016F82730044603F00303022B8846914684
:109270004FF0000306EB870A09D01360CBF80030EB
:109280002369990710D4002003B0BDE8F08F56F889
:10929000271013608908CBF80030F1D0FFF7B0FF3A
:1092A000E368A3600120EFE7A3695046984716F8EA
:1092B00027300546DA07E6D513F002031DD0B8F1D2
:1092C000000F03D041462046FFF7A6FF61682A46FB
:1092D0002046FFF787FFD4E902319942606004D14C
:1092E0002A462046FFF77EFFA060A3682360E36064
:1092F000236943F008032361D4E701462046019324
:10930000FFF77EFFE268A260B8F1000F04D0216889
:10931000E269019B42F8213005EB0802CBF80020FE
:1093200021682046FFF75EFF2369206043F00803B1
:10933000236116F827306FF3000306F82730C9F8C9
:1093400000A0AFE770B504461546FFF74BFF236852
:10935000834205D12369216023F00803236170BD96
:10936000E269AB0043F0020342F8213061682A460B
:109370002046FFF737FF6060F1E738B50369044620
:109380005B0706D5456AFFF71CFF85422CBF656267
:10939000606238BD38B50D4604461C22002104F039
:1093A00025FF0022EB68A361AB6863612B68E36172
:1093B0006B68626223622A6923B1591E194208BF91
:1093C00042F001022261012204F128000021BDE8DF
:1093D000384004F006BB2DE9F04F002587B000931C
:1093E000036A04468B420E469246A94603950595AC
:1093F00039D3EFF3118B202383F31288BFF36F8FE0
:10940000059AD8462AB129462046FFF79BFF00233C
:10941000059304A92046FFF7C1FE04990746B1420F
:109420002AD32268E369204613F8221003EB82094D
:1094300021F0030103F8221021683246FFF7D2FE23
:10944000E3682060984212D0002788F31188BFF3A8
:109450006F8F039929B162690AB1204690470023B2
:109460000393002FC5D1484607B0BDE8F08F2369AC
:1094700043F008032361E7E718B12046FFF7CCFE6D
:10948000E3E7009B5AEA030319D0019104F02BFB98
:109490000199A0B98BF31188BFF36F8F5246009BDF
:1094A00004F12800FDF7E2F9EFF31188202383F39C
:1094B0001288BFF36F8FB0FA80F77F09C5E72046A7
:1094C00005AB03AA2568FFF7C6FE0746BDE770B5E2
:1094D0000446836908460D4698470246EFF3118615
:1094E000202383F31288BFF36F8F2B78204643F03D
:1094F00001032B706168FFF775FE60602046FFF77F
:109500003CFF86F31188BFF36F8F70BD2DE9F041EA
:1095100004462027EFF3118687F31288BFF36F8F7D
:10952000236913F0080FA36802D16268934200D93F
:10953000226AD21AE16932B986F31188BFF36F8FBC
:109540004FF0000833E011F8232001EB830812F0FC
:109550000300F1D0022803D151F82350AD0805D102
:10956000D00712D44046A36998470546A1682A4609
:109570002046FFF737FE2946A0602046FFF740FE51
:1095800086F31188BFF36F8FC4E742F0020201F83F
:109590002320A3694046A5689847294602462046ED
:1095A000FFF720FEA06086F31188BFF36F8F40465F
:1095B000BDE8F081F8B50446836908460D46984732
:1095C0000646EFF31187202383F31288BFF36F8FD2
:1095D0002B786FF300032B7023699B0705D5E26896
:1095E000E36903EB82039D421AD12B786FF34103A9
:1095F0002B70D4E90231994204D132462046FFF75C
:10960000F1FDA06031462046FFF7FAFD87F311888F
:10961000BFF36F8F04F12800BDE8F840FDF702B9F1
:109620002B6860F39F032B60F0E7026983681207E1
:1096300002D442689A4200D2026AD31A181E18BF96
:1096400001207047038B13F0070305D10368002B3B
:109650000CBF002003207047022B05D1408BB0FACD
:1096600080F0400980007047012B05D10368002B72
:109670000CBF0020052070470020704710B50C4635
:1096800000B111B96FF0150010BD081D00F093F87E
:109690000028F9D1A368032BF6D9F3E72DE9F041AF
:1096A0000D4607461946281D90461E4600F097F8BD
:1096B000044638B13346424629463846A446BDE8FA
:1096C000F0416047BDE8F08110B4EFF3118220242F
:1096D00084F31288BFF36F8F416110BC0121F2F750
:1096E0003BB938B50C46054658B151B10B6843B18A
:1096F0004B6833B11C22002104F078FD00202C615E
:1097000038BD6FF01500FBE770B505460E46FFF754
:10971000B5FF041E14DBEFF31182202383F31288BC
:10972000BFF36F8F4FF6FF716B8B2C8B8B4204F066
:10973000070407D182F31188BFF36F8F6FF00A041B
:10974000204670BD022C0CD101336B8382F311884B
:10975000BFF36F8F0023224631462846FFF79EFF56
:10976000EEE7062C14D8DFE804F004131313041AF0
:109770000400002333606B683BB9C5E90066ACB9EF
:1097800002212846F2F7E8F8DAE71E606E60F6E795
:1097900082F31188BFF36F8F6FF00404D0E782F378
:1097A0001188BFF36F8F6FF08504C9E782F31188CA
:1097B000BFF36F8FC4E7034640B1426802F0030273
:1097C000022A06D0032A04D0012A05D06FF0150022
:1097D00070471A68002AF9D000209860704710B5C9
:1097E0004268034602F00302022A4FF0000481603F
:1097F00007D0032A02D05C60002001E018685C609A
:1098000010BD18685C600028F6D0FEF72DF8F3E76D
:10981000704703785B075FBF03684288C3F34A233E
:1098200003EB12105DBF173020F007008008002006
:1098300070470020704702F091B80346D3E8EF0F5D
:10984000421CC3E8E12F0029F8D170471FB500235F
:10985000CDE902011A4619461846CDE90033F2F760
:1098600097FC05B05DF804FB0120F2F755BA002023
:10987000704770B5D2E901369B1B8B420C461546EA
:109880000AD313680A460146981904F0A2FC204640
:10989000AB682344AB6070BD6FF01B00FBE770B595
:1098A0000E4615461946044618B9BDE87040F2F751
:1098B00033BA33B1C2F34A231030120D184404F006
:1098C00088FCC4E900562046BDE87040F2F7A8BB0A
:1098D0002DE9F3415F1C4FEA8708064608F117009F
:1098E00020F0070080080C461546F2F777FA0023AF
:1098F0008DF80470ADF805308DF8073068B1034677
:10990000019AA8F1040143F8102F2A46294452F87D
:10991000045B8A4243F8045FF9D100233146A20177
:1099200002F4E07242EA482222F07F4222F47002FE
:1099300022F03F0202B0BDE8F041FFF7B0BF07B52B
:109940000123019201AAFFF7C3FF03B05DF804FBF6
:1099500007B5CDE9002302236A46FFF7B9FF03B03C
:109960005DF804FB1FB5CDE90123069B01AA039313
:109970000323FFF7ADFF05B05DF804FBF8B506461D
:109980000D4614461F4604B9F8BD214628463A46FE
:10999000B047241A0544F6E713B500240094F1F704
:1099A00031FC02B010BD10B542680446D2E9002374
:1099B00081680068FFF7E2FF002263681A6010BD4B
:1099C00038B54B6805461A68CB680C469A4202D1F6
:1099D0000846FFF7E8FF6368D3E8EF2F511CC3E8A0
:1099E000E01F0028F8D1A36800209D5438BD0A2844
:1099F00038B504460D4602D10D20FFF7E1FF294698
:109A00002046FFF7DDFF002038BD2DE9F043054675
:109A100087B008460E8891F800900C46D1F808806F
:109A20001746F2F7FBFB011EC6F38216C9F3C20903
:109A30001EDB4846F2F706FB0346214651F8102B81
:109A40006088C2F34A22002A01EB020408BF002109
:109A50000022C0F30B10CDE90407CDE9021428461B
:109A6000414601960092F2F705FC07B0BDE8F0838D
:109A70000023E2E7436800201B685B689961704738
:109A800043681B681A685268536070470121436835
:109A90001B685A6811771868FFF785BF43681B6811
:109AA0001868F2F755BD70B543680C461D686B68C1
:109AB0009869F2F70DF9214603460F222868BDE8A0
:109AC0007040184701460068F2F7AABD08B5F2F7E2
:109AD00003FEBDE80840F2F703BE0A460121FFF786
:109AE0002EBF7047704700210120F2F799BD836EA9
:109AF00083F30B88704761B662B680F31188BFF3B9
:109B00006F8F704772B6002383F31188BFF36F8F96
:109B1000BFF34F8F30BF62B6BFF36F8F704772B61F
:109B2000002383F31188BFF36F8FBFF34F8F20BFE4
:109B300080F31188BFF36F8F62B6704740E800F37F
:109B400013F4803FD8B208BF6FF01500704730B5EE
:109B50000C684B6885B00A894D890094013B24F05C
:109B60001F04234402F01F0242EA451223F01F03A0
:109B700069468DF808200393F3F7E0F905B030BD8E
:109B8000002070474FF0FF3070474FF0FF324FF02A
:109B9000FF33FCF761BDFCF7D7BDFCF799BBF3F7CA
:109BA0001FBDF3F727BD0CB4034607B504AA08464A
:109BB00052F8041BDB680192984703B05DF804EB90
:109BC00002B07047FCF748BDFCF7BEBD37B569462B
:109BD00001AA0546F1F726FA044640B9FFF7DDFF72
:109BE00009234FF0FF340360204603B030BD4FF02F
:109BF000FF3201984FF0FF33FFF7E4FF009B204650
